:1000000090390020FD17000051180000FD16000077
:10001000FD160000FD160000FD160000FD16000094
:10002000FD160000FD160000FD16000099140000EA
:10003000FD160000FD16000055140000FD1600001E
:10004000C11700009BA20000C1170000C1170000EB
:10005000C1170000C1170000C1170000C117000040
:10006000C1170000C1170000C1170000C117000030
:10007000C1170000C1170000C1170000C117000020
:10008000C1170000C1170000C1170000C117000010
:10009000C1170000C1170000C1170000C117000000
:1000A000C1170000C1170000C1170000C1170000F0
:1000B000C1170000C1170000C1170000C1170000E0
:1000C000C1170000C1170000C1170000C1170000D0
:1000D000C1170000C1170000C1170000C1170000C0
:1000E000C1170000C1170000C1170000C1170000B0
:1000F000C1170000C1170000C1170000C1170000A0
:1001000000000000991100000000000071160000BE
:10011000F846002095EA000000000000711600007B
:1001200000000000711600000000000071160000C1
:100130000000000025E9000000000000711600002A
:1001400000000000711600000000000071160000A1
:1001500000000000711600000000000061A2000015
:10016000000000007116000004470020C9EE0000E6
:100170000000000071160000000000007116000071
:10018000000000007116000000000000C112000015
:100190000000000071160000000000007116000051
:1001A0000000000071160000000000007116000041
:1001B0000000000071160000000000007116000031
:1001C0000000000095A20000000000007116000071
:1001D0000000000071160000000000007116000011
:1001E0000000000071160000000000007116000001
:1001F00000000000711600000000000071160000F1
:1002000000000000711600000000000071160000E0
:1002100000000000711600000000000071160000D0
:1002200000000000711600000000000071160000C0
:1002300000000000711600000000000071160000B0
:1002400000000000711600000000000071160000A0
:100250000000000071160000000000007116000090
:100260000000000071160000000000007116000080
:100270000000000071160000000000007116000070
:100280007BB972B90029BEBF00204FF0004106E0E3
:1002900008BF00281CBF6FF000414FF0FF3000F096
:1002A000C5B9ADF1080C6DE904CE002909DB002BBE
:1002B0001ADB00F04DF8DDF804E0DDE9022304B0BC
:1002C0007047404261EB4101002B1BDB00F040F81E
:1002D000DDF804E0DDE9022304B0404261EB4101B6
:1002E000524263EB43037047524263EB430300F017
:1002F0002FF8DDF804E0DDE9022304B0404261EBB1
:1003000041017047524263EB430300F021F8DDF8EE
:1003100004E0DDE9022304B0524263EB430370477B
:1003200053B94AB9002908BF00281CBF4FF0FF315C
:100330004FF0FF3000F07AB9ADF1080C6DE904CE52
:1003400000F006F8DDF804E0DDE9022304B07047B0
:100350002DE9F0478C460D460446089E002B51D1EE
:100360008A4217466DD9B2FA82FEBEF1000F0BD059
:10037000CEF1200C01FA0EF520FA0CFC02FA0EF771
:100380004CEA050C00FA0EF44FEA174A250CBCFBA8
:10039000FAF81FFA87F90AFB18CC45EA0C4508FB66
:1003A00009F3AB420AD9ED1908F1FF3280F023813D
:1003B000AB4240F22081A8F102083D44ED1AA4B2FC
:1003C000B5FBFAF00AFB105544EA054400FB09F9B5
:1003D000A14509D9E41900F1FF3380F00A81A14554
:1003E00040F2078102383C44A4EB090440EA08408B
:1003F0000021002E61D024FA0EF4002334607360D3
:10040000BDE8F0878B4207D9002E54D0002186E842
:1004100021000846BDE8F087B3FA83F1002940F0D7
:100420008E80AB4202D3824200F2FA80841A65EBDE
:1004300003050120AC46002E3FD086E81010BDE831
:10044000F08712B90127B7FBF2F7B7FA87FEBEF1C2
:10045000000F34D1EB1B3A0C1FFA87FC0121B3FBD0
:10046000F2F8250C02FB183345EA03450CFB08F3B0
:10047000AB4207D9ED1908F1FF3002D2AB4200F2CE
:10048000D1808046ED1AA3B2B5FBF2F002FB105505
:1004900043EA05440CFB00FCA44507D9E41900F12C
:1004A000FF3302D2A44500F2B8801846A4EB0C0436
:1004B00040EA08409DE731463046BDE8F087CEF17E
:1004C000200405FA0EF307FA0EF720FA04F83A0CA6
:1004D00025FA04F448EA0308B4FBF2F14FEA1845A0
:1004E00002FB11441FFA87FC45EA044501FB0CF3AB
:1004F000AB4200FA0EF409D9ED1901F1FF3080F09A
:100500008A80AB4240F2878002393D44EB1A1FFAE1
:1005100088F5B3FBF2F002FB103345EA034500FB1C
:100520000CF3AB4207D9ED1900F1FF386FD2AB42A3
:100530006DD902383D44EB1A40EA01418FE7C1F121
:10054000200722FA07F88B4005FA01F448EA030372
:1005500020FA07FE4FEA134CFD404EEA040EB5FBAD
:10056000FCF94FEA1E440CFB19551FFA83F844EAC4
:10057000054509FB08F4AC4202FA01F200FA01FA5F
:1005800008D9ED1809F1FF3043D2AC4241D9A9F1A5
:1005900002091D442D1B1FFA8EFEB5FBFCF00CFB5F
:1005A00010554EEA054400FB08F8A04507D9E418A9
:1005B00000F1FF3529D2A04527D902381C4440EA72
:1005C0000940A4EB0804A0FB02894C45C6464D46F1
:1005D00015D312D056B1BAEB0E0364EB050404FA3E
:1005E00007F7CB401F43CC40376074600021BDE863
:1005F000F0871846F8E69046E0E6C245EAD2B8EB46
:10060000020E69EB03050138E4E72846D7E74046C8
:1006100091E78146BEE7014678E702383C4445E76A
:10062000084608E7A8F102083D442BE7704700BFE1
:1006300043689B6903B11847704743685B6A03B11D
:100640001847704743685B681847000038B5084C86
:100650004FF0FF3120460DF0AFFE054601F028FABD
:1006600010B128460DF0CEFE0FF060F9F0E700BFA4
:100670009047002010B50E480E4C0EF093FC206001
:1006800098B1FFF7DAFF2068FFF7D2FF22685368BE
:1006900023B11B6C13B10849104698472068436882
:1006A0001B6A03B19847002010BD6FF0150010BD04
:1006B000CA04010004000020F10600002DE9F04109
:1006C00007460E4615469846002425B17B681B69EF
:1006D00023B94445F9D32046BDE8F0812A46314686
:1006E000384698470028F4D02D1A04440644ECE715
:1006F0002DE9F0414F4D504C8AB02F462868436891
:10070000DB6B7BB1984768B1286843689B6B4BB142
:10071000984738B128684368DB6A33B9386843685A
:10072000DB6983BB0AB0BDE8F08198470028F5D0AB
:100730002668002E4FD1334601220DF103012868AF
:10074000FFF7BCFF0128D9D19DF80330012B1CD045
:10075000022BE7D104230DEB03011A463868FFF79B
:10076000ADFF002135480DF021FE064638B10223C9
:10077000042203750DEB020108300DF077FEBDF881
:100780000630236017E09847CCE703231A4601A9F7
:100790002868FFF793FF9DF806302948236031460B
:1007A0000DF004FE064630B100230375032201A9B3
:1007B00008300DF05BFE234B1E60224E306850B1B6
:1007C00008300DF06CFE2368984204D230680DF0BA
:1007D00019FE00233360DFF86C80D8F800307BB955
:1007E0003868226843681B69212A28BF21222BB15F
:1007F00001A9984723681B1A23607FE71846F9E789
:10080000986899892268014400233868FFF756FFE9
:10081000D8F8001026688B89361A03448B8126602D
:10082000002E7FF46BAF08480DF0DFFDC8F80060C4
:1008300064E700BF0400002008000020A04700205B
:10084000C04700200000002090470020F8B5054672
:100850000F464FF02002EFF3118382F31188234CEF
:100860002068FFF7EAFE2068FFF7E2FE002D37D090
:100870002B4600225E1B13F8011B69BB1544B61AF8
:1008800004212068FFF7DEFEFF212068FFF7DAFE73
:10089000B11DC9B22068FFF7D5FEAA212068FFF775
:1008A000D1FE36B1013D15F8011F2068D1B9FFF71F
:1008B000C9FEF9B22068FFF7C5FEC7F3072120681B
:1008C000FFF7C0FEC7F307412068FFF7BBFE390EF4
:1008D0002068FFF7B7FEFEE72F2908BF5A1BC9E7BC
:1008E0002E46CDE7FFF7AEFEDDE700BF0400002097
:1008F0002DE9F0411C481C4E1C4D86B001F0DEF87D
:1009000000236FF00802059304930392029301936E
:1009100000934FF42072164B164917480FF05EFAF9
:100920004FF0FF3130460DF047FD037D012B0446AB
:100930000DD0032B08D102212868FFF783FE04F1B4
:100940000807A3892BB920460DF05CFDE8E70421D8
:10095000F2E73846D5F800800DF099FD0146404693
:10096000FFF770FEEDE700BF804700200400002085
:100970004D060000D82D00200C00002008B50446CC
:10098000084611461A46A0470FF000F800F0F2FEA4
:1009900010B590F90B40C0688C424FF00C04B6BF04
:1009A000614304FB01014158202492FBF4F401EB64
:1009B0008401196002F01F0010BD07B501ABFFF7FD
:1009C000E7FF019A012303FA00F013680343136061
:1009D00003B05DF804FB07B501ABFFF7D9FF019A3F
:1009E000012303FA00F0136823EA0003136003B045
:1009F0005DF804FB2DE9F04743680589044600686B
:100A0000A77A5D43FF222844E27200214FF00C0ECA
:100A10004FF0200CB94205DB002523899D4223DBE2
:100A2000BDE8F087D4F80C90B5FBF3F20EFB01F8AB
:100A30001F2A09EB08064FEA930306F1040AC8BF10
:100A40001F3203F10303C6F804A0C6F808A0CABF0A
:100A500092FBFCF2E17249F8080023F00303C8BFDF
:100A600000EB82000131D5E76268E36820686A43E1
:100A70001E1D865081189A684A609A682046116047
:100A800099602A460021FFF798FF0135C5E72DE957
:100A9000F04F8BB0857A00AF0446BB60AB000A33E1
:100AA00023F00703ADEB030D4368FA6003336A4696
:100AB00023F0030342F80439E9464FF0FF360023E0
:100AC0004FF00C0E581EAB42786209DA2BB1106859
:100AD0008008033020F003005060506888420BD239
:100AE0007B6A013314D13A6D002313606FF00B0061
:100AF0002C37BD46BDE8F08FE0680EFB030000F127
:100B0000040C40680432604518BF1E460133D9E723
:100B1000711CE8D094F8108059F8261018F00108DC
:100B200005D04FF02003EFF3118883F31188E268BA
:100B30000C2303FB062353F8045F9D422CD095E859
:100B40000C001A602A68536022682046AA1A92FB99
:100B5000F1F23146FFF73FFF237CDA0701D588F336
:100B60001188002D6AD0A9EB890309EB860A3B6145
:100B70007B6A9E4212DBFB681A467B6A136023681D
:100B80007A6AEB1A59F8222093FBF2F3BA681360E1
:100B90003B6D00201D60ABE70025DDE7237C13F0F3
:100BA000010305D04FF02002EFF3118382F3118887
:100BB0003B6223685AF8042BEB1A93FBF2F33A6971
:100BC0009B00BB610AEB4A0313444FF0010B7B61AE
:100BD00006EB0B037B60DAF8008079680BFB08F307
:100BE000FB61EB183B60BB6920460BEB0302FFF790
:100BF000E4FE3B682268218908F1FF389844A8EB9D
:100C0000020862684A4390450AD2E2687969F86945
:100C10000A44111D29509168596091680B609360D6
:100C20000BF1010BBBF1040FD5D1237CDB0706F1DF
:100C300001069DD53B6A83F3118899E76FF00A009E
:100C400056E72DE9F04F87B0837A9B000A3323F0F3
:100C5000070300AFADEB030D4368033323F0030339
:100C60000446EB4600936D460120814260D20D465A
:100C7000164694F810805BF82590D4F800A018F080
:100C8000010805D04FF02003EFF3118883F311889A
:100C9000324629462046FFF790FE002D51D007F13D
:100CA0001403324629462046FFF772FE7A69042370
:100CB00090FBF3F083001068D84000F00F000F287D
:100CC0003FD126F00302FA6009F1FF320023BA6037
:100CD000FA687B6002EB030A524629462046FFF77A
:100CE0007AFE56457B6816D0B968B4F808E02268E9
:100CF00009FB0AFA0AEB0100616801FB0EF1884268
:100D000002EB0A0C07D2DCF8040052F80A1001606A
:100D100052F80A2050600133042BD9D1237CDA0722
:100D200001D588F311880423013D96FBF3F6A0E773
:100D30002B689B08033323F0030345F8043F01307D
:100D400093E709FB06F6226861680AEB060309F1DE
:100D5000FF399944A9EB02092289514389450BD2F5
:100D6000E1680C2202FB05152A1D4AF80620AA6834
:100D70005A60AA681360AB60237CDB0701D588F357
:100D800011881C37BD46BDE8F08F704710B54FF095
:100D90002003EFF3118483F3118800F025F8084A4B
:100DA0000123C2F840354FF08042C2F87835054B38
:100DB0004FF0FF329A62DA6284F31188002010BD8E
:100DC00000E0014000ED00E0054B1B68082B01BF6F
:100DD000044B1868B0FA80F0400918BF0020704733
:100DE000300100103401001008B54FF0804300229C
:100DF000C3F80C21C3F81021C3F838254FF08052F6
:100E000003F54043D2F80414C3F82015D2F80814AF
:100E1000C3F82415D2F80C14C3F82815D2F810140E
:100E2000C3F82C15D2F81414C3F83015D2F81814DE
:100E3000C3F83415D2F81C14C3F84015D2F82014A6
:100E4000C3F84415D2F82414C3F84815D2F828146E
:100E5000C3F84C15D2F82C14C3F85015D2F830143E
:100E6000C3F85415D2F83414C3F86015D2F8381406
:100E7000C3F86415D2F83C14C3F86815D2F84014CE
:100E8000C3F86C15D2F84424C3F87025FFF79CFF13
:100E900010B1334B334A1A60FFF796FF18B1324B4B
:100EA000FB22C3F81825FFF78FFF48B12F49304BBD
:100EB0000A681B6822F00F0203F00F0313430B6054
:100EC000FFF782FF18B12B4B4FF400721A604FF0FE
:100ED0008043D3F80024D20744BF6FF00102C3F867
:100EE00000244FF01023D3F80022002A03DBD3F8AC
:100EF0000432002B2FDA204B0122C3F80425D3F84B
:100F00000024002AFBD04FF010221221C2F8001258
:100F1000D3F80024002AFBD04FF010231222C3F88C
:100F20000422154B1A46D3F800140029FBD00021E7
:100F3000C3F80415D2F80034002BFBD0BFF34F8F59
:100F40000E490F4BCA6802F4E0621343CB60BFF353
:100F50004F8F00BFFDE70B4B0B4A1A6008BD00BF67
:100F60008C5600404881030000F00040E40E004031
:100F7000580200104096024000E0014000ED00E001
:100F80000400FA05F04400200090D00313B5114C82
:100F9000BFF35B8F2068BFF35B8F60B90E480EF024
:100FA00001F8BFF35B8F54E8003F44E80002002AD9
:100FB000F9D1BFF35B8F436804221B680DEB02017C
:100FC0009847002802DA00F0F9F90190019802B080
:100FD00010BD00BF7C0000200C05010010B54FF0D3
:100FE0002003EFF3118283F31188114C237823B986
:100FF00082F311886FF0440010BD013BDBB2237017
:1010000023B182F311886FF00F0010BD094B1878DF
:10101000012128B1217082F311886FF00A0010BD00
:10102000197082F31188044A1160187010BD00BF56
:1010300082000020810000200400004008B500224A
:101040001046012100F0FCFA002000F0C7FA002051
:1010500008BD0000F8B54FF02002EFF3118382F3D2
:101060001188264A1078441C147070B183F31188DB
:101070004FF08043D3F80C3403F00113B3F1011F98
:101080000CBF00206FF04300F8BD1D4D2F782FB12D
:10109000107083F311886FF00A00F8BD01262E70DE
:1010A00083F311884FF0804419B3384600F0A6FA54
:1010B000C4F80071D4F80433C4F804632660D4F88B
:1010C000002192B10022C4F800210E4A13F0010F52
:1010D0004FF0010308BFC4F808330020C2F8803184
:1010E00000F07CFA00232B70C2E720BF40BF20BF76
:1010F000E5E7C4F800112660F4E700BF8200002095
:101100008100002000E100E038B54FF02002EFF34D
:10111000118382F311881D4D2A788AB183F31188D7
:101120004FF08042D2F81C34D2F8182403F00303A5
:1011300043F48033934314BF6FF04300002038BD65
:1011400001242C7083F311884FF08043104DC3F8B5
:101150000421C3F818152C6011F003014FF0180595
:10116000C3F80853C3F80C21C3F81021D8D11022BA
:10117000C3F83825C3F80453C3F80443FFF76AFFE4
:101180000028CDD1034BC3F80041C9E780000020FF
:101190000800004000E100E0F8B54FF0804305464C
:1011A000D3F808E1D3F80423D3F80C44D3F8007142
:1011B000D3F80401D3F80C11D3F8106102F0010246
:1011C000BEF1000F03D04FF0000EC3F808E127B1C5
:1011D0004FF080430027C3F800713AB1E30341BFE9
:1011E0004FF080430122C3F808231A6120B14FF069
:1011F00080430022C3F8042149B14FF0804400210C
:10120000C4F80C112846FFF7E9FE0123636176B1AB
:101210004FF0804300210124C3F810112846C3F881
:101220000443FFF717FF10B9014BC3F80041F8BDA5
:1012300000E100E0084BC3F84005D3F80435C01ABC
:1012400020F07F40054B0238984282BF044B4FF498
:101250000032C3F80021704700100140FDFF7F00FD
:1012600000E100E038B5114B114CD3F804052268B9
:10127000104D801A2B6820F07F4098420FD3B0FBAE
:10128000F3F00D490968884228BF084600FB032394
:1012900023F07F432360094B18600EF0FBFB2068AE
:1012A0002B681844BDE83840FFF7C4BF0010014068
:1012B00088000020B846002084000020B4460020AA
:1012C000024B0022C3F84021FFF7CCBF00100140C1
:1012D000031E0A4A0A4804DB116890FBF1F18B42B5
:1012E00002DD136890FBF3F31068064A06491268A2
:1012F0000B6000FB0320FFF79DBF00BFB846002036
:10130000FFFF7F00880000208400002008B5074B05
:101310000022C3F84021064B4FF40032C3F880216D
:10132000FFF7A0FF034B01221A6008BD0010014027
:1013300000E100E08400002070B519480DF032FE95
:1013400050B34368174D1B6801219847164B002482
:101350001C60164B01261E60154BC5F808451B681E
:10136000C5F840354FF48033C5F84433C5F804332D
:10137000104BC5F840414FF40032C3F8802131468C
:101380002246112000F05CF9112000F027F90A4BE9
:1013900020461E602E6070BD4FF0FF3070BD00BF54
:1013A000300501000010014088000020840000206A
:1013B000B846002000E100E008100140064BD3E9E8
:1013C0000001064B1B685843054BD3F804351B1A24
:1013D00023F07F4318447047482D0020B846002072
:1013E0000010014007488168006A884208D000B5B3
:1013F0000EF070FA5DF804EB03494FF080520A607A
:1014000070470000102D002004ED00E00448002388
:101410002021C2180133302B82F80013F9D1704714
:1014200000E100E0084A094993680968D96608495B
:1014300098664B6843F080534B60002383F3118818
:101440009368D86E704700BF102D0020AC0A0100D1
:1014500000ED00E0202080F311880D498A682C20DF
:101460001044EFF3098C80E8F01F0A4F4FF000663C
:101470000A6A8A603E60906E0023936680F311884A
:1014800002F12C0090E8F01F8CF3098870470000EF
:10149000102D002004ED00E01EF0040F0CBFEFF350
:1014A0000880EFF30980816931F8021C11F0FF0117
:1014B0000229FFD000B500F040F900BD094B9A6A3F
:1014C0009A6A9A6A910708D55A6B9A6A120604D5E5
:1014D00018B19A6A22F080029A629A6A9B6A002086
:1014E000704700BF00ED00E00E4B9A6AD20416D49C
:1014F0009A6A110513D49A6A12F4007F9A6A09D085
:10150000120404D518B19A6A22F400429A62054B7B
:101510009B6A04E0510502D49A6AD205F8D50020EE
:10152000704700BF00ED00E0074B9A6A9A6A9A6A1A
:101530009A6A9A6A9A6A9A6A6FEA02426FEA124251
:101540009A620020704700BF00ED00E01B4A53681C
:10155000C3F30803033B10B50446032B2AD8DFE886
:1015600003F002252722D36A9B0723D4D06A10F008
:10157000804007D0124B1B784BB10120FFF79EFF34
:10158000062819D02146BDE8104000F0CBB80D4B1D
:101590001B781BB10120FFF7A7FFF1E70A4B188862
:1015A00080B20028EED0FFF7BFFFE9E70020E5E7B3
:1015B0000020F0E70020E5E710BD00BF00ED00E0EF
:1015C00028ED00E029ED00E02AED00E0024A536931
:1015D00043F010035361704700ED00E043B2002B6D
:1015E00008DB012200F01F0002FA00F05B09024A4A
:1015F00042F82300704700BF00E100E043B2002B37
:101600000DDB01225B0900F01F0002FA00F020331D
:10161000034A42F82300BFF34F8FBFF36F8F704729
:1016200000E100E04209054B00F01F0053F82220C2
:10163000012303FA00F01040704700BF00E100E012
:1016400043B2002BA8BF03F1604301F101014FEA4F
:101650004111ADBF03F5614300F00F00034BC9B268
:10166000B6BFC9B283F800131954704714ED00E0F7
:1016700000F044B808B572B6044BD86918B100221E
:10168000DA610DF0B7FC62B608BD00BF102D002076
:1016900070470000F8B50C4616461F4604220A9B08
:1016A000099905460EF022FCA6F1200121440C4ABE
:1016B000EC6521F00701002322F001022B656B6528
:1016C0002E668A61069A4A60079A8A60089ACA60FA
:1016D0000F604FF08072CA61E964AB66F8BD00BF6D
:1016E0007D090000014910220A60704710ED00E0FA
:1016F000404080F3118830BF704700BF404080F306
:101700001188DFF81CC0DCF800C01CF4006C0CBFB2
:10171000EFF30880EFF3098000B5FFF717FF00BD76
:1017200004ED00E038B504460D460EF02FF92946C9
:101730002046BDE8384000F005B801460068FFF7D4
:10174000F1BF0000052808B504D00EF0FDFA20B165
:101750000EF0FAFAFFF7CCFFFCE70EF005FB0028CD
:10176000F6D1034B9868BDE8084000F003B800BF0D
:10177000102D002038B505464FF02003EFF31184FB
:1017800083F311880EF048FB0B4B9B689D420DD1F3
:101790000A4B5A68C2F3080222B90EF09BF82046A1
:1017A000FFF740FE5A6842F080525A602046BDE87A
:1017B00038400DF043BF00BF102D002000ED00E0C9
:1017C00000B572B60B4AD06900281EBF0021D16156
:1017D0000DF010FC62B6EFF30580A0F110004FEAA7
:1017E000C0000549014409C998475DF804EBFFF7BB
:1017F000F9BD0000102D002000010000202080F322
:10180000118806484FF40061401880F309880220CF
:1018100080F31488BFF36F8F00F006F8D03A0020F1
:1018200030BFFFF7FDBF00BF08B5074B074A23F0E5
:101830007F039360BFF34F8FBFF36F8F0DF00AFCF0
:101840000DF012FC0DF030FC0000000000ED00E097
:1018500008B5FFF7E5FFBDE80840FFF7C3BD00008E
:10186000034B05225A60BFF34F8FBFF36F8F704752
:1018700090ED00E0114A10B51468082C1BD81049EF
:10188000506800234B609C4200F10C0003D1FFF72D
:10189000E7FF002010BD8B6050F80C2C22F01F02D7
:1018A00042F010021A43CA6050F8042C42F00102C0
:1018B0000A610133E7E74FF0FF3010BDD04400204C
:1018C00090ED00E00139034611F8012F0AB91A70B2
:1018D000704703F8012BF7E70138013910F8013F91
:1018E00011F8012F934202D1002BF7D11A46981A12
:1018F000704770B582B1013A0C46034603D11A789D
:101900002078101A70BD1E782578AE4200F10100D3
:1019100001F10101EFD0F2E7104670BD81EA00034A
:1019200013F0030F70B503460BD0013B0A449142FC
:101930001BD170BD002AFCD011F8014B03F8014BFC
:10194000013A9C07F6D11E1F0D46541B0C44032C74
:1019500006D822F003042144234402F00302E4E702
:1019600055F8044B46F8044FEFE711F8014B03F824
:10197000014FDCE770B5C9B203469C0711D141EABB
:10198000012444EA04441E46951B1D44032D0ED831
:1019900022F00304234402F003021A44934209D1C3
:1019A00070BD002AFCD003F8011B013AE5E746F8B8
:1019B000044BE9E703F8011BF0E730B585B00446B6
:1019C000154668460322FFF7A9FF0D2200210DF1FD
:1019D0000300FFF7CFFF20466A4669460AF000FB86
:1019E000044620B9032269462846FFF797FF2046A0
:1019F00005B030BD13B50C4601AA0331FFF7DDFF7A
:101A000048B9032201A92046FFF773FFB0FA80F01E
:101A1000400902B010BD0020FBE770B5CD1C0646A2
:101A20000C46284603210AF0BFFA60B9637903F037
:101A30003F0343F040036371224629463046BDE828
:101A40007040FFF7BABF70BD074A136833B9C16869
:101A500039B1016929B11060184670476FF0440030
:101A600070476FF015007047C02B002010B504467A
:101A700002480CF09BFC00B1047510BDE04700204B
:101A800008B5014603480CF091FC08B10123037529
:101A900008BD00BFE047002008B5034B01461868A9
:101AA0000CF0A3FC002008BD8C000020FFF7F4BF61
:101AB000014B1B681B691847C02B0020044B054ACB
:101AC0001B6810600BB1DB6818476FF0120070479D
:101AD000C02B00208C000020F7B51860C31D054600
:101AE00023F00303501E0E4680B214461A800021D4
:101AF000042206FB0050FFF73DFF023CA4B24FF664
:101B0000FF77BC4201D103B0F0BD04FB06602B1887
:101B10000422801B0DEB02012844013C0193A4B276
:101B2000FFF7FCFEEDE773B50568064695B1EB1DC2
:101B300023F0030304221C8829460DEB0200FFF763
:101B4000EDFE019B013CA4B21BB1DA1D22F00302A1
:101B500014803360284602B070BD70B50C6806462C
:101B60000D461CB1E31D23F003031C880422294603
:101B70003046FFF7D3FEF21D22F00302631C1380F0
:101B80002E6070BD18B1073020F003000088704748
:101B900002FB01007047401A80B2B0FBF2F07047C0
:101BA00010B5114401384FF6FF73013A92B29A42D0
:101BB00000D110BD11F8014D00F8014FF5E70144C7
:101BC000884201D10020704710F8013B002BF7D06C
:101BD0000120704710600860704710B514682060DD
:101BE00014686160106010BD884203D01AB1436868
:101BF00013607047002070470B68834209D022B100
:101C0000586810601A680A6001E0002BFAD1184683
:101C100070470023FBE700002DE9F047114FDFF884
:101C200048900426013EF6B2FF2E19D033B24FEA97
:101C3000830803EB43031D0104244FF00C0A0AE060
:101C40001AFB04510A1D04EB08003A44394409EB1D
:101C5000C000FFF7BFFF013CE4B2FF2CF0D1E1E789
:101C6000BDE8F0871001002090000020F0B4124B76
:101C700005460F460C26302472B1614306FB001462
:101C80002344597A187A814204BF013119722846D7
:101C90003946F0BC0CF04CBA4C4306FB00442344DC
:101CA0009C7ADA7AA24204D101329A72F0BC0CF02A
:101CB00079BAF0BC704700BF10010020F8B50546A6
:101CC0000E461C468AB1012362782078801A10F0F3
:101CD000030729D003B3012F39D00132D2B22270C9
:101CE000314628460CF05EFA1CE00CF049FA002858
:101CF000E9D0314628460CF02FFA0028E3D03023F3
:101D00000C22734302FB0533124A1A44937AD27AA7
:101D10009B1A18BF0123D7E70232D2B22270E368C0
:101D2000A06898470020F8BD002BF8D00132D2B24D
:101D300022700423302212FB06320C2313FB0523EE
:101D4000044A60681A442146FFF747FFC8E738464F
:101D5000F8BD00BF100100202DE9F04F00EB40035B
:101D600089B01B014FF00008434E0493054604243C
:101D7000CDF80480013CE4B2FF2C0BD1019B002B79
:101D800076D0B8F1000F73D14246294628460CF0B0
:101D9000CFF96DE00DF1200B00230C274BF8043D2B
:101DA0004FF0300907FB04F309FB053031185A46A0
:101DB000496830580293FFF717FF049B17FB04375D
:101DC000F31982460393BAF1000F19D130220C2384
:101DD0006A4303FB04223244917AD07A88421EBFC0
:101DE000D1720122019230226A4303FB042333445F
:101DF0001A7A597A91421CBF5A724FF00108B9E71A
:101E0000079B1F785A78BF1A07F00307012F04D1E8
:101E1000013A5A709868DA689047079A13785278AE
:101E2000DBB29A1A02F00302012A05930DD0029B3D
:101E3000039909FB0530304400224068FFF7DCFEBF
:101E4000079A059BC2F804A05370029B09FB053357
:101E5000F1185A464968F058FFF7C6FE012F82462E
:101E6000B1D10CB90028B1D0294628460CF09AF916
:101E700009B0BDE8F08F00BF1001002010B5421E70
:101E800000200139C9B2FF2900D110BD12F8013F6D
:101E9000002BF6D05C1E01302340C0B2F8E7F0B54D
:101EA000437F05681A460024FF2A01D10020F0BDB7
:101EB00002EB82078A4205EBC70615F8377004D09B
:101EC000B3681C4413463A46EEE7934200D1477785
:101ED0001BB203EB83033278B06805F83320337804
:101EE000FF2B06D003EB830305EBC3039A68024480
:101EF0009A602044F0BD30B5551A15F4000F836880
:101F0000446909D125F07F421A44A2420ED9121B1E
:101F100000248260446130BD8A1A22F07F429342DD
:101F200001D99A1AF1E72244D41A0022A41A0022F5
:101F3000EFE7034600221A709A6A596208460AB10E
:101F4000D96A104770472DE9F047857F0123044681
:101F5000C377002D4CD1437FFF2B02D1C577BDE85D
:101F6000F0870BF059FB6769667FD4F80080C71BC8
:101F700027F07F47FF2E06D006EB860608EBC6014A
:101F80008B689F4218D2A27AE37A934205D101333B
:101F9000DBB2022B08BF0023E372E37A04EB830376
:101FA0000122DD600023656AE377AC462346042105
:101FB0000320BDE8F0476047FF1A1D448A784B783C
:101FC00018F836609B1ADBB2012BD3D1D1F80C90F4
:101FD000013A8A70B9F1000FCCD048696369CA8BA5
:101FE000281A184420F07F400B69496AC847C1E7A6
:101FF000BDE8F0872DE9F04FC27F93B08346002AF9
:1020000040F0BA83436905930121837A8177C07ACE
:10201000984200F08F800B44DBB2022B08BF0023F4
:102020008BF80A300BEB83030191D3F80C80059BEE
:10203000434423F07F43CBF814309BF81D300393C7
:10204000DBF800300493DBF804300B939BF8093085
:10205000013BDBB20293002307934FF0FF0A029B80
:10206000FF2B6AD19BF81D30039A9B1A18BF0123DE
:102070000293019BE3B1DBF8003004934FF00009B9
:102080009BF81D60FF2E0CD037B2049B07EB87072F
:1020900003EBC704A568454540F23681A5EB08056A
:1020A000A560029B019A0399B14218BF134602939F
:1020B000DBF800300893DBF8043010939BF809300C
:1020C000013BDBB20193019BFF2B40F070819BF839
:1020D0001D30039A9342079B40F045835BB99BF800
:1020E0000940DBF804300193013CE4B24FF00008F2
:1020F000FF2C40F0A08200238BF81E30029B4BB1D6
:102100009BF81D30FF2B40F0E9820BF06BFA08B909
:10211000CBF818009BF81F30002B00F02D83DBF864
:1021200024405B46012203210420A44613B0BDE8ED
:10213000F04F6047019290467FE70B9B029A03EBBA
:10214000C2077B680693F978BE788E4200F0D7808C
:10215000069B387806EB460212019D18731CDBB211
:10216000984208BF0023BB70069B9A5C032AEBD9F8
:10217000052A17D8697801EB81030A930A98049B12
:1021800003EBC0046378A0781B1A13F0FF0309D097
:10219000042A0CD16A6852B9AA6842B9EA6832F0D6
:1021A0007F4204D101212846FFF7C3FECBE7012B74
:1021B00040F09B805846FFF772FE2B78A060042BFE
:1021C000064640F08480DBF8143008930BF024FAC4
:1021D000089B0990C31A23F07F4343449E42024662
:1021E0009EBF6269921B9B18626896BF6361F31A77
:1021F00000238AB1A98979B101F1FF3E1FFA8EFE51
:10220000A5F80CE09A422BD3DFF82493B4F81EC053
:10221000E64547D8A4F81CE0AA8808991344A360AF
:10222000EA88636913446361099A2046FFF763FEF5
:10223000A2692B891344A3616A8993428CBF9B1ABC
:102240000023A361AB7B03B1E370049B0A9A03F8FC
:1022500032A0637895F801A0013363700021A2E7F2
:10226000B4F81EC0E645CFD2616AAF4EAF488E19B2
:10227000864281BF01F1E87101F5D43101F5A57104
:102280006162666A216A8CBF4FF001094FF0000954
:10229000761A91440CF1FF3C6662A3EB0903A4F8A3
:1022A0001EC0AFE7666A216AA0480E449E497118B5
:1022B00081428EBF002101214E4411440CF1010CDA
:1022C0008CBF666266620B44A4F81EC09EE7A378CA
:1022D00063706B789BF81C209A4201BFFF238BF838
:1022E0001C300023CBF81830B8E704215B46DBF83C
:1022F000244001220846A0470123BE700793029B99
:10230000013BDBB20293AAE6DBF818309D4229BFFD
:10231000FF235B1B8BF81C300023CBF81830A3691C
:10232000A9441BB18BF81C60CBF818300022049B29
:10233000A26013F837308BF81D30D4F804E0BEF1FA
:10234000000F30D0A08BDFF8E4C1636A216A0B4430
:102350007549591861459FBFA3F1E873A3F5D433BC
:10236000A3F5A573636292BF019B6362002373446C
:1023700010F1FF301A44E8D2059BA260DBF814107C
:1023800003EB09022046FFF7B6FDA38BE38300238E
:10239000E370049B03F837A0637801336370A8EB04
:1023A0000508B2466CE6A37863705646F7E7109BC3
:1023B000019A03EBC20304935B680A93049B93F8AE
:1023C0000190BAF1FF0F00F08E800FFA8AF303EB51
:1023D0008303089AD04612F833A002EBC304002509
:1023E000DBF800300B93FF23A28B2370E38B934227
:1023F00086BF9B1A9BB200230C930FFA88F303EB62
:102400008303DB001193119BDBF80020DBF818003D
:10241000059002EB030EFF209BF81D30DEF808103C
:1024200009930690FF2B07D003EB830C02EBCC063D
:10243000B068814200F2A980DEF818000D9001EB2F
:10244000000C1E46FF2E40F0AE800D9830B105986E
:102450008142C0F0BF80FF2E40F08A810998CEF8FB
:102460000810834218BFBDF924008EF8003016BF53
:1024700000EB80008BF81D8002F83080FF2B06D027
:1024800003EB830302EBC3039A68511A9960A378A4
:10249000013363700021002D93D02846FFF749FDDA
:1024A0008FE709EB49030A9A1B01D51809F10102CC
:1024B0005FFA82F9049A12784A4508BF4FF0000982
:1024C0000A9AD35C032B0ED195F80180089B08EB88
:1024D000880403EBC4046278A3789A4209D00121EE
:1024E0002846FFF726FD049B9B784B45D9D1019BDD
:1024F000E6E5EB68DBF8141063602B692362AB8AB6
:10250000A383AB69A361EB69E3602B6A23610026B7
:10251000AB68A36066616A682046FFF7ECFC0123A4
:102520006662E683E3705BE75A2B17FF592B177F30
:10253000B6562EFE606800287BD0626A216A904BF6
:102540000A449049D3188B429CBFA2F1E872A2F5CD
:10255000D432A3688BBF6262A2F5A57200226262C8
:10256000034498BF01221344E28BA3600132E2834B
:10257000626993424FF0000189BF9B1AD31AA3608E
:1025800061619CBF6361A1603DE7B669091A46B904
:10259000059FB84200D23E1A0993059612F83C30C6
:1025A00040E70693F8E730B200EB800002EBC0078B
:1025B0000E97BF680F9767450AD20E9FBF69002F1D
:1025C0007FF443AF0F9EACEB060C12F8306039E796
:1025D000FF263AE7069B98453FF459AF069BFF2B31
:1025E000A8D01E4633B203EB83030593059A0B9BD9
:1025F00003EBC207FB8BBA8B934288BF9B1A7A68A6
:102600008CBF9BB20023002A94D00C9A934291D89D
:10261000FA78E3789A428DD231465846FFF73FFC6C
:10262000BB787B70059A0B9BB86003F832A0B2466A
:10263000E9E601212FE7019B03EBC4056E686B7887
:10264000EA789A4202D1013CE4B251E503EB43033C
:102650001B01F218F35C012B25D0022B2AD1D2F8F2
:1026600004C093689CF80000D2F80C90DBF800E0FE
:10267000FF2804D01968DBF81470B94223D0DBF8C6
:1026800014009BF81D1018600023FF2907D001EBF0
:10269000810A0EEBCA0087698068DFB103448CF8B9
:1026A0000010C9F80030936AC2F8248013B1D16ACF
:1026B000002098476B782A780133DBB29A4208BF32
:1026C00000236B70BBE700EB8000D9F800301EF8E8
:1026D0003010DAE703441EF83A10D6E7039BFF2BCD
:1026E00007D10AF099FF04460AF06EFF08B9CBF84B
:1026F00014409BF81D30DBF80020234E03EB8303CE
:1027000002EBC3030A279D680AF086FFDBF814403A
:10271000031B23F07F430333AB422CBFE41864193F
:1027200024F07F448046DBF82830204698470AF0A2
:1027300073FFA0EB080020F07F40A4EB08040330F7
:1027400024F07F44A04207F1FF377FF6E3AC002F6F
:10275000DAD140F202413046FEF778F8D4E70023A0
:102760008BF81E30CCE4002BF9D101230293B6E4A0
:10277000B0457FF437AF8AE613B0BDE8F08F00BFF5
:102780005A2B17FF592B177F60050100F0B51A4D22
:10279000059F9DF818402C26464305EB060EAA51CE
:1027A0008EF8081007998EF80930CEF80470013BB6
:1027B000DBB2FF2B11D1ECB92C2202FB005208999D
:1027C0001162099951620A99916253771377946162
:1027D00054619472D4722046F0BD1AB207EBC2065F
:1027E000716017F8322002EB4206A41A01EB0611C1
:1027F000E4B2DCE70120F0BDD0010020074A2C2123
:1028000000FB012310B45C6A2CB1A4460122032111
:10281000022010BC604710BC704700BFD0010020F0
:102820002DE9F047254F4FF02C08814608FB00703A
:102830000FFA81FCD0F804E00EEBCC061EF83CE069
:10284000F478651CEDB2AE4598BF002596F801E01E
:10285000AE452FD0D6F804C004EB44044FEA041E62
:102860000CEB0E044FF0030A0CF80EA06360089BFB
:10287000A360099BE3600A9B23610C9BA361BDF8E5
:102880002C30A3820D9BE3610E9B236202236362C3
:102890000F9BA362109B6270E362F570456A036A46
:1028A0000846984709FB087300220421A847606A7C
:1028B000BDE8F0870120BDE8F08700BFD00100200F
:1028C0002DE9F047DFF890804FF02C0A0AFB008ECC
:1028D0000FB2DEF80450814605EBC70015F83750FB
:1028E000C478661CF6B2B54298BF00264578B5425A
:1028F0002FD0D0F804C004EB440425010CEB0504F0
:1029000004270CF80570A380BDF82030E380BDF8E3
:1029100024302381BDF828306381BDF82C30A38199
:102920009DF83030A373022363620D9BA3620E9B5C
:102930006270E362C670DEF82030DEF8245008468C
:10294000984709FB0A8300223946A847606ABDE818
:10295000F0870120BDE8F087D00100202DE9F04785
:10296000DFF86C904FF02C0A0AFB009E8046DEF8E0
:1029700004000EB200EBC60710F83600FC78651CA8
:10298000EDB2A84298BF00257878A8421DD078689B
:1029900004EB4404240106194FF0050C00F804C0B0
:1029A0007270B3620222089B7262F362FD70DEF8FD
:1029B0002030DEF824400846984708FB0A9300229E
:1029C0000421A047706ABDE8F0870120BDE8F087C8
:1029D000D00100202DE9F047DFF878804FF02C0A75
:1029E00081460AFB00800FFA81FE456805EBCE07A1
:1029F00015F83E50FC78661CF6B2B54298BF00262A
:102A00007D78B54223D0D7F804C004EB44042501F7
:102A10000CEB05044FF0020E0CF805E0A360089BD8
:102A2000E360099BA362FF250A9B62606570C4F89E
:102A300024E0E362FE70456A036A0846984709FB92
:102A40000A8300220421A847606ABDE8F0870120BC
:102A5000BDE8F087D00100202DE9F047DFF86C9049
:102A60004FF02C0A0AFB009E8046DEF804000EB2EE
:102A700000EBC60710F83600FC78651CEDB2A842E2
:102A800098BF00257878A8421DD0786804EB4404EC
:102A9000240106194FF0010C00F804C0FF207070EB
:102AA00002207062B262F362FD70DEF82030DEF860
:102AB00024400846984708FB0A9300220421A047B7
:102AC000706ABDE8F0870120BDE8F087D0010020E2
:102AD0002DE9F041084C2C2505FB004306465F6AB2
:102AE0001B6A0846984706FB0543BC4600220421A2
:102AF000BDE8F041604700BFD00100200AF08CBD66
:102B0000401A20F07F40704708B50346012B084665
:102B10000ED833B119B106220649FEF7FFFE05486B
:102B200008BD19B106220449FEF7F8FE024808BDA7
:102B3000002008BD2E0200202802002070B50646A5
:102B40000D4606F0D1F9044610B10C24204670BDA4
:102B500006F0DEF910F0060FF7D1062229461EB165
:102B60000248FEF7DBFEF1E70148FAE72E020020FB
:102B700028020020002303700B70704720BF40BF65
:102B800020BF7047F0B50D4B89B005460E4601AA2F
:102B900003F1180718685968144603C40833BB4288
:102BA0002246F7D11B88238008AB1D4415F81C0C66
:102BB000831B5842584109B0F0BD00BFB00401006A
:102BC00008607047024B1868436800211B6818476B
:102BD0003402002018B90B6843F000430B607047C3
:102BE00018B90B6823F000430B60704770B5031DE4
:102BF000451E00249D4201D1204670BD15F8016F8D
:102C00000022A018082AC0B201D10446F2E716F04B
:102C1000010F03D00029F0D00139C9B27608013282
:102C2000EFE70000094B93F8420193F841219042ED
:102C30003BBF93F8412193F8403193F84131C018DC
:102C40002CBFC01A801AC0B2704700BF34020020E7
:102C500008B50146FFF7E6FF884221BF044B93F811
:102C60004121D3F83C3153F8220038BF002008BD81
:102C70003402002030B590F8743090F875409C42D2
:102C80005AD190F8C01090F8C1308B4254D190F9CD
:102C90001D30002B25DBC18C828CA0F87C10C18FED
:102CA000A0F87A2051437D224A434FF47A7192FB77
:102CB000F1F2A0F87E2090F87820012565F301025A
:102CC000D2B2002342F00402013C80F88850C0F8E0
:102CD000843080F8782080F8765080F87540184667
:102CE00030BD90F8C230DC0628D490F850309A06F7
:102CF00003D5D0F8A4309B0720D5C48C828CA0F8D3
:102D0000C640C48FA0F8C42054437D2262434FF4D0
:102D10007A7492FBF4F2A0F8C82090F8C220002345
:102D200002F0F80263F3C302013980F8C33080F87F
:102D3000C22080F8C110D2E7012030BD022030BD92
:102D400010B50C4620B142F611510548FDF77EFD45
:102D500094F850306FF3410384F8503010BD00BF39
:102D6000AC0501002DE9F843224D95F8424195F854
:102D7000549195F8403101348145E4B228BF814631
:102D800005F5A477A34208BF002405F59878B9F1AA
:102D9000000F03D095F841319C4201D1BDE8F88382
:102DA0003846FEF7C0FE06460028F7D04046FEF73C
:102DB000BAFE28B930461049BDE8F843FEF7CDBE4B
:102DC000066095F84221D5F83C3143F8220085F899
:102DD000424195F840310134E4B2A34208BF0024D7
:102DE00095F8543109F1FF39013B85F854315FFA08
:102DF00089F9CCE7340200207C03002038B5354C3B
:102E000094F81021002A61D004F586734FF4AA715A
:102E1000D4F80801FEF760FE2F4B94F83A21B4F87D
:102E20003811D4F82C01FEF757FE94F8401194F8AD
:102E300010212A4BD4F844010A440821FEF74CFE25
:102E4000274BD4F8580102222421FEF745FE94F8BE
:102E50007421244BB4F86811D4F86001013A92B29D
:102E6000FEF73AFE1D48FEF75EFE054620B940F229
:102E700033211D48FDF7EAFC1C4A2846111FFEF7C6
:102E8000A9FE94F8293043F0380384F829301F2331
:102E900084F81E31252384F81F311B23A4F8223126
:102EA0004FF4A473FF20A4F82431072384F81A01F7
:102EB00084F81B0184F81C0184F81D01A4F8263154
:102EC000A4F82831BDE83840FFF74CBFC4F80C2106
:102ED000A2E700BF34020020640300207C0300202E
:102EE0009003002098030020AC050100840300201B
:102EF0002DE9F84F0C78944281460F4690463DD01C
:102F00001F4ED6F8703133F83430038000254FF06F
:102F1000020B06F5B27A22B2D6F87001B9F800E0D9
:102F200000EBC20130F83220964520D148680128D4
:102F300020F003030AD9F3B1021D1CD04279D2B1AB
:102F4000027902F00302013A012A14D80122154441
:102F50004A60EDB213B15146FEF7FFFD013496F819
:102F60007421E4B2A24208BF00244445D3D13C708E
:102F70002846BDE8F88FC1F804B0EBE70025F7E775
:102F80003402002010B5094B93F810218242044608
:102F90000AD902464FF4AA71D3F80801FEF7F8FDEA
:102FA00010B1038CA34200D0002010BD34020020D9
:102FB0002DE9F04186B00223052805468846029394
:102FC0000ED0062800F0A08040F2A480073880B21E
:102FD000FFF7D8FF002800F0278190E8C0000FE03D
:102FE000924B9E69DF6902AB00930A46904B032126
:102FF0000020FFF7B3FC022879D0029B002B7AD186
:103000008A4CE37C23B142F21E718A48FDF71EFC14
:1030100006AB0222E57443F8102D032100932A46E3
:10302000834B0020FFF79AFC02287BD0029B002BE9
:1030300040F0EE80637C9D4203D0A37C9D4240F033
:10304000E38006AB022243F80C2D002200930321FB
:10305000774B1046FFF782FC02280CD10122114663
:103060000320FEF703FE039B022B04D142F26261B0
:103070007048FDF7EBFB039B002B40F08980022397
:103080000493637C23B942F26C616A48FDF7DEFB6E
:1030900004AB002000930122654B60740321FFF70D
:1030A0005DFC02280CD1012211460320FEF7DEFD53
:1030B000049B022B04D142F27B615E48FDF7C6FB04
:1030C000049A002A47D126F00046B74239D95A4B14
:1030D00011460320FEF7F2FD002800F0958042F231
:1030E0008F615448FDF7B2FB8EE0FFF747FD029B6E
:1030F000022BFAD081E7029B012B81D042F2FF61C3
:103100004C48FDF7A3FB7BE7484BD3F8D060D3F8DE
:10311000D47075E742F2197146480026FDF796FB18
:1031200037466DE7A37C9D4204D10122114603205E
:10313000FEF79CFD029B022B7FF478AFFFF71EFD8C
:10314000F8E73E4B11460320FEF7B8FD00285BD0A0
:1031500042F29661C5E7049B012B16D10022364B43
:1031600011460320FEF7AAFD20B142F29F613148CB
:10317000FDF76CFB0022314B11460320FEF79EFD4C
:10318000002841D042F2A561ABE742F2A761A8E76F
:10319000039D012D45D1B8F1FF0F23D006AB0222CC
:1031A00043F8042D032100934246214B0020FFF7F2
:1031B000D5FB02280CD12A4629460320FEF756FDEE
:1031C000059B022B04D14FF41B511A48FDF73EFB1F
:1031D000059B3BB1059B012B04D042F2C46115480D
:1031E000FDF734FB237D7BB1154B04229A6000224E
:1031F00011460320FEF762FD20B142F2D4610D4872
:10320000FDF724FB237D4BB9E37C0BB9012302932B
:103210000023E374029806B0BDE8F081FFF7AEFC2E
:10322000F0E742F2DC615CE70120F4E734020020C1
:10323000C12B0000AC05010034450020F4450020FE
:103240006445002010B5C4B2231F012B04D941F2FC
:1032500050510948FDF7FAFA084A537D3BB1043B47
:10326000012B04D95475BDE810400AF071BC0AF076
:10327000A1FC0028F7D010BDAC05010034020020ED
:10328000F8B590F83A40058E064604F007040F465C
:10329000204600210AF08AFB96F8F83013F0100F50
:1032A0004FEA440210D0291D42F00102C9B20820A1
:1032B0000AF0E8FB3A46214606F1F9000AF03CFE26
:1032C000BDE8F8400AF010BC082042F00102E9B263
:1032D0000AF0D8FB3846F3E7F8B5134C94F8785168
:1032E00094F874310135EDB2AB4208BF002594F873
:1032F0007731AB4207460E4604D142F242310B48C9
:10330000FDF7A4FA94F87821D4F8703123F83270DC
:1033100094F8782103EBC2035E6084F87851BDE82D
:10332000F84006F0CDBF00BF34020020AC0501001C
:103330002DE9F843244C064600272EB194F8753148
:1033400094F876219A4201D1BDE8F88394F875810A
:10335000D4F86C91D4F8080139F8382009EBC80387
:103360004FF4AA715D682F60FEF712FC034639F82E
:1033700038001A8C82421FD1D3F8482142B9D3F8C1
:103380003C21C3F848511AB9C3F83C51C3F84C2149
:10339000D3F84C2102B11560C3F84C5194F8753143
:1033A00094F874210133DBB29A4208BF0023013E36
:1033B00084F87531F6B2C0E72B7967F301032B71FE
:1033C0002946FFF789FFE9E73402002073B501229F
:1033D000044611460020FEF749FC94F8202042F2F2
:1033E0005F33002107320093D2B23F4B0846FFF70C
:1033F000B5FA30F0020304D042F261313B48FDF7E8
:1034000025FA3B4D6B7D052B27D1238C6A7C073336
:103410009A4222D1002142F2703300930122324BB2
:1034200069740846FFF79AFA30F0020304D042F2BA
:1034300072312E48FDF70AFA002242F277330093E8
:103440001146294B1046FFF789FA30F0020304D0E9
:1034500042F279312548FDF7F9F9D4F83C11D4F856
:103460004031994203D0D4F84831994201D1214EDC
:1034700012E00B796FF301030B710B68C4F83C3158
:10348000208CFFF729FFE8E70368C4F83C31C4F853
:1034900040313146FEF761FBD4F83C0118B1D4F855
:1034A00048319842F0D10023C4F84031C4F8443187
:1034B000D4F83C1151B94FF6FF732384D5F8883105
:1034C0009C4208BFC5F8881102B070BD0B796FF33C
:1034D00001030B710B68C4F83C31C4F84831208CEF
:1034E000FFF7FAFEE4E700BFB13E0000AC050100C3
:1034F0003402002090030020F8B50F4690F83810F1
:10350000C58DC1F3C2040646C90920460AF04EFA29
:1035100096F8F83013F0200F4FEA44020FD0291D1F
:10352000C9B2082042F001020AF0ACFA394606F5A9
:103530008D700AF057FDBDE8F8400AF0DBBA0820AC
:1035400042F00102E9B20AF09DFA3846F3E70000C2
:10355000262810B504460BD027280BD025280BD1E0
:1035600002200AF05FFA2046BDE810400AF060BA77
:103570001A20F6E75020F4E70A2802D8023040006B
:10358000EFE7272801D80330F9E741F2BF6102488D
:10359000FDF75CF9E7E700BFAC05010070B5314C01
:1035A00094F8793094F87A209A4251D00133DBB202
:1035B000022B08BF002384F87930012294F8C93027
:1035C00094F8CA10994207D00133DBB2022B08BF2E
:1035D000002384F8C930012294F8795027232B2145
:1035E00013FB0515661942B194F8C90003FB0040AE
:1035F0000622B11C7D30FEF791F930460AF07AFAC6
:10360000635D03F00F03022B24D0072B22D002238B
:10361000962063750AF094FB00200AF0F3FA94F800
:103620002830C3F30202D3B219460020CE0700F1BE
:10363000010514D5013B134094F82820C0B263F370
:10364000020284F828202530BDE87040FFF780BFD3
:103650000022B3E7032363750AF0EAFADFE74908BB
:103660002846E3E7340200202DE9F04F8FB0924660
:10367000049303680991002B8046426880F2B6806B
:10368000816823F0004391422CBF5A1A9A1A05927E
:10369000D8F80C203D320024FF27D31807938DF86B
:1036A0002970ADF82A400C940B940697A146A346C6
:1036B000254602230D930DAB02937B4B01930BAB7D
:1036C00000930DF129020CAB01210020FFF782F9D4
:1036D000022800F094800D9B23B141F24E417348C3
:1036E000FDF7B4F89DF82930FF2B64D0FF2F07D0E9
:1036F0000C9B994504D041F257416C48FDF7A6F860
:103700009DF82920052A51D9694890F810310733CE
:103710009A424BDA062A00F09F80069BFF2B4AD183
:10372000073A92B24FF4AA71D0F80801FEF730FAC6
:1037300080453BD0099B1BB990F91D30002B35DB30
:10374000059B0B9E41681E440368002B5BDA826870
:1037500023F000438A422CBFB6187618F61AC268C6
:1037600002F13D094B440893DAF800309E4216D925
:103770009D4238BF1D46079B0BEB0307189B1B7828
:10378000A34205D929463046FFF7BAF9B8423ED2DE
:10379000BDF82A30049ACAF8005093420BD2DDF8E3
:1037A00030909DF82970DDF820B03546189B1B78C5
:1037B000A3423FF67EAF9DF82930FF2B11D1DAF8F6
:1037C0000030DFF8F08036A7D7E900679D4238BFA8
:1037D0001D464FF00709189B1B78A3423ED8CAF834
:1037E0000050189B1C700FB0BDE8F08F934238BF9B
:1037F000134600224BE701210020FFF769F90D9BDA
:10380000022BF8D067E78B4238BF0B46A7E7294A5F
:1038100005EB0B03A3FB0201072202FB031120A30C
:10382000D3E90023FCF77CFD40F2E243B0FBF3F068
:10383000049B80B29842ADF82A000BD2199B022259
:1038400003EB44000DF12A010134FEF767F8E4B2FE
:10385000283593E700259BE70692A7E705EB0B03C6
:10386000A3FB080109FB031132463B46FCF758FD58
:1038700040F2E243B0FBF3F0049B80B28342ADF828
:103880002A000BD9199B022203EB44000DF12A01F7
:103890000134FEF743F8E4B228359CE700259EE7A3
:1038A00000CA9A3B00000000C12B0000AC050100DB
:1038B000340200208D49FD1A1FB50023039306230F
:1038C0008DF80B3090F91D30D0F8DC10002BBEBF06
:1038D0000246036F42F8E43F01910DF10B010091A4
:1038E000A8BF03AAB0F8C4300021FFF7BDFE05B0A1
:1038F0005DF804FB000000002DE9F043B0F8CE2095
:1039000089B004464048062305AEA2FB00018DF8AD
:103910000D3040F22313002503FB021138A3D3E935
:10392000002305957560B560FCF7FAFC08AA0DF157
:103930000D0142F8100DB4F8C43000910196012138
:103940002046FFF791FE04F1CE0704F1DA084FF6A6
:10395000FF79022239460DF10E00FDF7DFFF9DF8D9
:103960000D00BDF80E200023D9B2884211D80237CD
:103970004745EED1B5B9BDF8142040F2E2435343B8
:10398000C4F8843002223146D4F88C00FDF7C6FF1B
:1039900027E04A4504D036F81310914224D001257F
:1039A0000133E1E794F8743084F8753094F8C0304E
:1039B00084F8C130154B0022C3F88821D4F88C302C
:1039C00013F8052C42F0030203F8052C032203F838
:1039D000042C112203F8022C0F2203F8012C2022C0
:1039E0001A7009B0BDE8F08340F2E2435343C4F8D3
:1039F000843002220DF10E01C6E700BFAFF3008054
:103A00008D49FD1A070000000054CE093402002041
:103A10002DE9F04F8BB00024FF25DFF818918DF8C9
:103A20001F50804693461F4601F1040A1C6008940B
:103A300026460223099309AB02933B4B019308AB43
:103A400000930DF11F025B4641460020FEF7C2FFC6
:103A500002283CD0099B23B141F293313348FCF753
:103A6000F5FE9DF81F20FF2A56D0062AE1D999F8C5
:103A7000103107339A42DCDA073A92B24FF4AA7156
:103A8000D9F80801FEF784F80028D2D090F91D304B
:103A9000002BCEDB0368089AD0F804E0002B1ADA7A
:103AA000816823F0004371452CBF52187244D21A2A
:103AB000C168FF2D01F104010B4410D19DF81F5086
:103AC0001C461646B5E741460020FFF701F8099B62
:103AD000022BF8D0BEE7734538BF7346E8E731469E
:103AE000104605930492FFF70BF804EB0A01884295
:103AF000049A059BE2D90E483444A4FB0001072335
:103B000003FB041106A3D3E90023FCF709FC803072
:103B100038600BB0BDE8F08FFF2DECD1F9E700BFA6
:103B200000CA9A3B00000000C12B0000AC05010058
:103B30008D49FD1A3402002073B5164602AA1C46B0
:103B4000054642F8046D27310120FFF761FF236825
:103B50001BB3019B9B1B1B0204D541F2E7311448A8
:103B6000FCF774FE31460198FEF7CAFF0246114881
:103B70000723A2FB000103FB02110BA3D3E90023DF
:103B8000FCF7CEFB236818440028206005DB40F2D8
:103B9000E24068432368984201D302B070BD1B1A0B
:103BA0002360F7E7AFF3008000CA9A3B00000000F3
:103BB000AC0501008D49FD1A13B500F184030446DC
:103BC000D0F89020C168808CFFF7B6FF02A9D4F826
:103BD0008430D4F88C0040F2E242B3FBF2F30222CC
:103BE00021F8023DFDF79AFE02B010BD10B4054C5D
:103BF000024604F58273D4F8FC10B4F8F40010BC4B
:103C0000FFF79ABF3402002070B504780A78C4F335
:103C10008013B3EBD21F19D104F00F04012C01F172
:103C2000080600F1020508D0062231462846FDF7B5
:103C300060FEB0FA80F0400970BD06223146284689
:103C4000FDF757FE0028EFD1204670BD002070BD63
:103C500010B5174C94F8413194F842219A4204D19E
:103C600042F28A211348FCF7F1FD94F84121D4F87F
:103C70003C3153F8221094F8783108680B7094F8AE
:103C8000413194F840210133DBB29A4208BF00234E
:103C9000094A84F84131FDF7A0FF20B942F29E2184
:103CA0000448FCF7D3FDBDE8104006F009BB00BF97
:103CB00034020020AC0501008403002010B501206F
:103CC000FEF7C6FF044620B941F648010948FCF753
:103CD000BDFD4FF6FF73E3800623237104F10B0053
:103CE0001D220021FDF746FE3C23E372BDE8104093
:103CF000FFF7AEBFAC05010070B5D0F8B430044694
:103D00000E4600F1B40523B942F2BD311048FCF76C
:103D10009DFD238CA4F8BA300E4A84F8BC600723BA
:103D200084F8B83092F87831D4F8B40084F8B4301C
:103D300002F5A8722946FDF750FF20B942F2CD31B5
:103D40000348FCF783FDBDE8704006F0B9BA00BF38
:103D5000AC050100340200202DE9F04782460878C6
:103D600001F108080D46C009414691461E4609F07A
:103D70007DF80446D8B91C4FBAF1000F0ED12B784C
:103D800097F8E120DB09B3EBD21F13D1062241469D
:103D90001648FDF7AEFD68B9012012E097F8E23051
:103DA000DB07ECD5484608F011FE0028E7D0204696
:103DB000BDE8F08797F8E100C0F3011010F00200B1
:103DC00001D10446F3E795F90030002B09DA6B7B4B
:103DD00003F0C003402B04D1002EDDD00120307051
:103DE000EFE70020EDE700BF3402002018030020B9
:103DF0002DE9F843814603200F461646FEF728FFBB
:103E00000446A0B34FF6FF73C3801A4B93F8E1301A
:103E10005A0728D0C3F30203DAB2012A20D0042AB9
:103E20001FD040F2C1411448FCF710FD94F80980FE
:103E300004F1080508F10208B9F1000F15D009F0E6
:103E40000FFF00F07F0005F80800637A2B44DF7055
:103E5000637A1D442E71FFF7FBFE0020BDE8F88356
:103E600003232371E2E70223FBE77F20EBE7012036
:103E7000BDE8F88334020020AC0501000B4A92F83B
:103E8000803192F8811199420ED192F8803102EB83
:103E90004303A3F87A0192F880310133DBB2032B9C
:103EA00008BF002382F88031704700BF3402002031
:103EB00020B141F26F110248FCF7C8BC704700BF47
:103EC000AC05010001280A4B0AD1DA7C052A02D18F
:103ED0000022DA7470474FF48C510648FCF7B6BCE8
:103EE0005B7C052B02D141F28711F6E7704700BFDA
:103EF00034020020AC05010001280A4B0AD1DA7C0B
:103F0000062A02D10022DA74704741F2991106485C
:103F1000FCF79CBC5B7C062B02D14FF48D51F6E77D
:103F2000704700BF34020020AC05010040B1054BD2
:103F3000DB7C052B04D041F2A9110348FCF786BCB9
:103F4000704700BF34020020AC05010048B1054BAA
:103F5000DB7CC9B2994204D041F2B1110248FCF7AE
:103F600075BC704734020020AC050100044B5B7D3A
:103F700023B1012100220846FDF778BE704700BF3B
:103F800034020020062810B50C460AD9094BC21F7E
:103F900092B24FF4AA71D3F80801FDF7F9FD206041
:103FA00010BD052804D00628034818BF002010BD06
:103FB000024810BD34020020040300204C020020FF
:103FC00038B50F4B00241C700546B0B101280DD147
:103FD0000C4B002211462846FDF770FE78B141F2E5
:103FE0006B210948BDE83840FCF730BC41F2642140
:103FF0000548FCF72BFC2346EBE7044BE9E738BD0B
:1040000054040020D4450020AC050100C445002024
:10401000002208B51146064B1046FDF74FFE30B1A1
:1040200041F2DD110348BDE80840FCF70FBC08BDB4
:1040300004450020AC050100002208B51146064BDE
:104040001046FDF73BFE30B141F214210348BDE8B4
:104050000840FCF7FBBB08BDA4450020AC050100EF
:1040600010B5094C237823B941F2C1110748FCF778
:10407000EDFB20780138C0B2207018B9BDE81040BF
:1040800006F01CB910BD00BFF0030020AC05010014
:1040900038B1054A1378591C117023B9012006F074
:1040A0000DB9FFF7DDBF7047F0030020FFF7D8BF61
:1040B0001FB5544C48B1E37C052B04D041F6E20116
:1040C0005148FCF7C3FB04B010BD637C052B02D044
:1040D000A37C052B7AD104AB022243F8082D0022E1
:1040E00000930121494B1046FEF738FC022814D0FA
:1040F000029BFBB10298012840F08180237D002BB8
:1041000064D0434B04229A6000221146FDF7D6FD8D
:1041100000285BD041F6CB0155E001221146104644
:10412000FDF7A4FD029B022BE2D101210020FEF746
:10413000CFFCF7E702230393637C23B941F67701B1
:104140003148FCF783FB03AB0122002000931146AA
:104150002E4B6074FEF702FC022819D0039A22B39A
:104160000398012848D100222A4B1146FDF7A6FDED
:1041700020B141F6B1012448FCF768FB0022264B30
:1041800011460120FDF79AFD00B341F6B7011AE090
:10419000012211461046FDF769FD039B022BDDD17C
:1041A00001210020FEF794FCF7E7A369E16923F001
:1041B00000438B4216D2174B11460120FDF77EFDBE
:1041C00020B141F6A1011048FCF740FB0022134B3F
:1041D00011460120FDF772FD00283FF474AF41F64F
:1041E000F1016DE70C4B11460120FDF767FD00283A
:1041F000ECD041F6A801E6E741F6B901E3E741F664
:10420000D301E0E734020020AC050100C12B00001F
:104210005445002024450020E4450020F4440020BB
:1042200030B50468002C89B01FDA436885680690B1
:104230009D4224F0004434BFE41A641B0C4B0593E8
:10424000A4B20023049303930293184601940094AC
:10425000FEF736FB30F0020307D0064841F29D21FD
:1042600009B0BDE83040FCF7F1BA09B030BD00BF7D
:10427000E12B0000AC05010037B502AD104B45F84D
:10428000043D044609F078FB002009F0BDFB0D4811
:1042900009F03CFB0121204609F088FB284609F083
:1042A000D9FB620002F0FE022521082009F0EAFB9A
:1042B000054940F25B6009F087FC03B030BD00BFE8
:1042C000D6BE898EF97400005555550008B5084BC7
:1042D0000022986011461046FDF7F0FC30B141F223
:1042E00074510448BDE80840FCF7B0BA08BD00BFEF
:1042F00044450020AC0501002DE9F04F90468FB0F9
:10430000D8F800401A9A0C929B461B9A0B91002CED
:104310008146189B9DF864A00D92DBF8005003DAEB
:10432000AB4238BF2B461C46AC425A4F40F283800A
:1043300041F2A1530893584B05930021631B00934E
:1043400007974B4606910491039102910191012236
:104350000846FEF765FA30F0020304D041F2A3519B
:104360004E48FCF773FA00231A4619461846FFF721
:1043700063FE4B4E0B9BF36041F2CE5308930D9BB3
:10438000069300220C9B059307974B4604920392D9
:1043900002920192009411461046FEF741FA30F065
:1043A000020304D041F2D0513C48FCF74FFA0520FB
:1043B000FFF78CFFD6F884319D4228D0CBF800302F
:1043C000D8F800300597002BBCBF23F00043C8F895
:1043D0000030D8F80020D6F884118A4238BF0A4647
:1043E00041F2FC51A3B292B20691002102930192D4
:1043F00000920491039152460846FEF761FA30F0AC
:10440000020304D041F2FE512448FCF71FFAFF20BA
:10441000FEF78EFF234B012211460020C3F808A0AF
:10442000FDF74CFC90B31D4841F211610FB0BDE89F
:10443000F04FFCF70BBA22D200231A461946184651
:10444000FFF7E6FD41F2B653002108932C1B164BF3
:10445000059307974B4606910491039102910191B0
:10446000009401220846FEF7DBF930F0020304D085
:1044700041F2B8510948FCF7E9F92C4679E70023E5
:104480001A4619461846FFF7C3FD6CE70FB0BDE8A2
:10449000F08F00BFB13E000011400000AC050100EC
:1044A0003402002004460020394000007FB50D4C46
:1044B000637C05460E4623B141F286710A48FCF73B
:1044C000C5F9052363740193236A00930022074B07
:1044D0000392074A029231461A1F2846FFF70CFF43
:1044E00004B070BD34020020AC0501005002002071
:1044F000E94600007FB5204C637C05460E4623B19B
:1045000041F614111D48FCF7A1F9062363740193C9
:10451000D4F8D83000930022194B0392194A029222
:1045200031461A1F2846FFF7E7FED4F8003103B3DF
:10453000D4F8D030002B0CDAD4F8D810D4F8D4202A
:1045400023F0004391422CBFC3EB0103C3EB0203F2
:104550001D440D4B0122114600209D60FDF7AEFB6E
:1045600038B1064841F63B1104B0BDE87040FCF795
:104570006DB904B070BD00BF34020020AC0501006D
:1045800008030020C54700007445002007B505203A
:10459000FFF79CFE41F60713002100930522094B0B
:1045A0000846FEF7DBF930F0020307D0064841F673
:1045B000091103B05DF804EBFCF748B903B05DF8EE
:1045C00004FB00BFB1400000AC05010010B50C4B6E
:1045D0001A7C8AB901220B481A740AF0E3FC0446DB
:1045E00020B941F22A210848FCF730F9636801211B
:1045F0001B682046984700B910BDFEF7BFFAF5E7E3
:104600003402002030050100AC050100024B18689F
:10461000436800215B68184734020020F0B5484029
:1046200003274FEA102E082600240EF00105013E54
:1046300045EA440516F0FF06ECB24FEA5E0EF4D1EF
:1046400025022DB2C0B24FF0080E344600F001062C
:1046500046EA44040EF1FF3616F0FF0EE4B24FEACC
:104660005000F3D12C4304EB0414013F0C4417F029
:10467000FF07A0B2D5D125244140B1FBF4F004FBE3
:104680001010C0B2C40800F00705145D2C41E40707
:1046900007D45943C1F307411046BDE8F040FEF787
:1046A000A5BAF0BD70B514460E460546FEF726FACB
:1046B0002146FEF725FAC41C092C11D9094B1B7899
:1046C00013B10020FFF77CFC324600212846FFF79B
:1046D000A7FDAB681C44262C00D8AC60012070BD3F
:1046E000002070BD5404002070B5324C237D054677
:1046F00023B141F2E9713048FCF7A8F8637C052B3F
:1047000004D041F2EA712C48FCF7A0F894F8290093
:10471000A56000230126267500F0070063740523B9
:10472000A374FFF7A9FD94F8293094F82820C3F367
:10473000C20363F3020284F82820FEF72FFF08F07B
:10474000B5FB94F8293000B313F0C00F14BF304606
:10475000002008F0CDF9821C4178007809F098FA21
:10476000E26805F10901012009F0F6FA09F0BAFB47
:104770002A4605211148FFF795FF034650B104234F
:104780006375BDE8704009F0E3B913F0C00FE7D0DE
:104790003046DEE70A4A0146FEF75EF930F00203D2
:1047A00006D041F639010448BDE87040FCF74EB828
:1047B00070BD00BF34020020AC0501004C02002097
:1047C0006D3F0000F0B55C4C237D8DB0054623B1F4
:1047D00041F64E115948FCF739F8637C062B04D09A
:1047E00041F64F115548FCF731F802232375012398
:1047F000002663750623667494F8E100A37494F8A8
:10480000E030A56066F3410300F0070084F8E03073
:10481000FFF732FD94F8E030C3F38100421C62F3ED
:104820008303253084F8E030FEF792FE94F8E03000
:1048300003F00C020C2A08BF66F383034FF09600C6
:1048400008BF84F8E03009F07BFA002319461A46C5
:10485000184609F0E3F9D4F83C3194F8412153F8B3
:104860002200083009F040F909F0F0F908F01EFBC9
:1048700094F8E13040B3C3F3001008F039F906466C
:104880000DF12F0008F0B6F871780746B21C3078A9
:1048900009F0FEF939469DF82F0009F0F1FBE268B6
:1048A00005F10901002009F057FA09F01BFB062168
:1048B0002A462348FFF7F6FE014688B104236375B4
:1048C00009F046F90DB0F0BD13F0300FE7D001202C
:1048D00008F00EF9821C4178007809F0D9F9DEE77A
:1048E00041F6AA130893174B0793174B0593D4F877
:1048F000F030049004220933009306922B46039073
:1049000002900190FDF78CFF30F0020304D041F6D5
:10491000AD110A48FBF79AFF0023194618460B4AC7
:10492000FEF79AF830F00203CCD041F6B6110348F6
:10493000FBF78CFFC6E700BF34020020AC05010086
:1049400004030020B13E0000815C00006D3F0000C8
:1049500010B590F8F840D0F8402114F0800F18D12D
:10496000D0F83C31ABB1240713D4D0F84841A3426E
:1049700004BF1C68C0F8484192B91A680A601960FF
:10498000C0F84011C0F844110B680BB9C0F84C11C5
:1049900010BD2AB9D0F83C310B60C0F83C11EFE7EC
:1049A000D0F844311A680A601960EBE710B490F847
:1049B000F84024070A460FD5D0F8401131B9D0F895
:1049C0003C111160C0F83C2110BC7047D0F8443154
:1049D000196811601A60F7E710BCFFF7B9BF000053
:1049E000F8B5214F054607F5AE700E46FDF79BF86A
:1049F0000446B0B333797179D7F8142143F07F437B
:104A000043F47E0343F4435343F0100343EA01238A
:104A1000B17943EA0143D2F8A410C1F310010B406D
:104A2000C2F8A43092F8503043F0200382F850309E
:104A3000037943F003030371082209234371C3710F
:104A400000211044FCF796FFD5F8A43023721A0A0F
:104A50001B0C28466272A3722146FFF7A7FF0020B5
:104A6000F8BD0120F8BD00BF3402002010B5044697
:104A7000C9B90F48FDF757F8B8B1011D94F8F830DF
:104A800043F0200384F8F8300B7843F003030B70F5
:104A900001234B700623CB7040B101462046FFF73F
:104AA00057FF002010BD0020E8E7012010BD00BF27
:104AB0009003002070B504460B480E461546FDF7DE
:104AC00032F878B10379067243F0030303710323CC
:104AD00043711123C371457201462046FFF738FF29
:104AE000002070BD012070BD900300200000000078
:104AF0002DE9F04FC94D8FB01C466B7C0C9181465F
:104B0000174623B141F64D71C548FBF79FFE94F857
:104B100020300733DBB26B7494F91D30002B09DAB7
:104B2000636DE26D07FB03331344A26DE3659342AB
:104B300088BFE265228D94F874301744628CBFB24E
:104B40002785174494F875209A42BFB240F0A78198
:104B500094F8F8305E0700F18A8294F8C12094F846
:104B6000C0309A4200F094800520FFF7AFFBD5F8E3
:104B7000883113B19C4240F08B8094F8C23003F02E
:104B80000703052B00F24681DFE813F006006300FF
:104B90001A01820082008200A248FCF7C4FF064688
:104BA000002875D094F8C230042262F3020384F81E
:104BB000C230037943F003030371182343710F23B9
:104BC000C371B4F8C43003814381B4F8C630838123
:104BD000B4F8C830C38100230374C37403754FF065
:104BE000FF3343758375C375037643768376C37647
:104BF000037743778377A0F8117001462046FFF7CB
:104C0000A7FE2268B4F84230C5F88841002AA4F80B
:104C10004430C4F8E0900BDAA368616822F00042E7
:104C20008B422CBF4B4409EB01039B1AC4F8E030C4
:104C300013367D4BC4F8DC600122114600209C60D5
:104C4000FDF73CF820B341F6B7417548FBF7FEFD90
:104C50001EE094F8C36096B37248FCF764FF014607
:104C6000B0B1037943F0030303711123C37103232C
:104C700043710F23037294F8C33043722046FFF749
:104C800067FE94F8C03084F8C1300023C5F888313D
:104C900094F8F52094F8F4309A4200F0F980052059
:104CA000FFF714FB94F8F63003F00302032A00F236
:104CB0006881DFE812F0BB00ED00ED00070194F918
:104CC0001D30002B3BDB94F8741094F875308B4248
:104CD000DED194F8C230C4F88460052262F3020386
:104CE00094F8CA2084F8C230012384F88830B4F8DC
:104CF000C43022B193FBF2F3013313FB02F3A4F8A7
:104D00007A30B4F8C630A4F87C30B4F8C830A4F8CF
:104D10007E3094F87830022262F3010394F8C220C6
:104D200082F00802C2F3C00262F3820384F8783092
:104D30000139012384F8763084F87510A8E73948E2
:104D4000FCF7F1FE01460028A2D0037943F00303EB
:104D50000371182343711023C371B4F8C430038165
:104D60004381B4F8C6308381B4F8C830C38194F865
:104D7000CA300374B4F8CC30A0F81130B4F8CE3097
:104D8000A0F81330B4F8D030A0F81530B4F8D23011
:104D9000A0F81730B4F8D430A0F81930B4F8D630F1
:104DA000A0F81B30B4F8D830A0F81D302046FFF72B
:104DB000CFFD94F8C03084F8C130C5F8886167E74A
:104DC00094F8F83018073FF563AF0220FDF740FF75
:104DD00000283FF45DAF94F8C230032262F302036F
:104DE00084F8C230238CC38001230371037A1343F8
:104DF0000372182343720F23C372B4F8C430838143
:104E0000C381B4F8C6300382B4F8C8304382FEF7D9
:104E10001FFF3DE741F6705117E700BF3402002045
:104E2000AC0501009003002094450020B248FCF737
:104E30007AFE014660B394F8F63094F839600122A6
:104E400062F3010384F8F630DBB2C3F38200C3F3EC
:104E5000421394F8382063F3C50684F8396094F857
:104E6000F76060F3020266F3861284F838200A794C
:104E7000087242F003020A7103224A7116224B7231
:104E8000CA712046FFF764FDB4F84230A4F84430FC
:104E900094F8752094F874309A4200F0E880052068
:104EA000FFF714FA94F87630013B072B00F2AD853A
:104EB000DFE813F06D00D802370351048104AB051D
:104EC000DA04F40494F8F42084F8F520C3F38202A1
:104ED000910744D5022262F3840384F8F63094F8F3
:104EE000F6305A09900743D5022262F3471384F83B
:104EF000F63094F8F62094F83830C2F38201C3F308
:104F0000C2038B4294F8783014BF61F384036FF3CB
:104F1000840384F8783094F83A30520903F0070398
:104F2000934294F8783014BF62F347136FF347133A
:104F300084F8783094F8783094F8F72043F001033F
:104F4000C2F3400262F3410384F87830082384F806
:104F5000763094F87530013B84F8753098E7D607C1
:104F600001D50122B7E712F0040218BF0422B2E70C
:104F7000D10701D50122B8E712F0040218BF0422BC
:104F8000B3E741F6D2615D48FBF760FC80E7D5F8F6
:104F900088310BB9C5F8884194F8783013F00303D1
:104FA00000F0B4805448FCF7BEFD064600285ED0F1
:104FB00094F8783003F00303012B00F09B80022B60
:104FC00040F091804E4A94F878306FF3010384F8F2
:104FD0007830E38C06333B449BB2A4F880303179BF
:104FE00041F0030131710C2171710021F17194F8CC
:104FF00088103172D4F8841040F2E240B1FBF0F135
:10500000A6F80910B4F87A10A6F80B10B4F87C10C2
:10501000A6F80D10B4F87E10A6F80F10A6F81130FF
:105020002168C4F8909000290BDAA368606821F029
:10503000004183422CBF4B4409EB00035B1AC4F8C8
:10504000903006F10903C4F88C302E4BDA6001224F
:10505000114600209C60FCF731FE20B141F6FB11A7
:105060002648FBF7F3FB31462046FFF771FC94F826
:10507000B12094F8B0309A421ED00520FFF726F9EF
:105080001D48FCF750FD0146B0B194F8B03084F8EB
:10509000B130037943F00303037102234371C371F9
:1050A00094F8B23003722046FFF752FCE38F012BD5
:1050B00098BF0133A4F8443094F8E92094F8E8301C
:1050C0009A4200F0E5840520FFF700F994F8EA30F1
:1050D00003F00303032B00F2BB85DFE813F0990410
:1050E000D904D904F50441F633210448FBF7AEFB9B
:1050F000002268E7044A66E790030020AC0501003F
:10510000F938000084450020B93B0000B4F88080E5
:10511000A7EB08081FFA88F818F4004FA7D194F8F5
:10512000742084F8752094F8C01094F8C1208A4245
:1051300009D094F8C22002F00702052A04BF84F8BF
:10514000C110A4F84430D5F888210023944208BF48
:10515000C5F888316B74A28CB4F87A309A4214D1B5
:10516000B4F87C10E38C99420FD140F2E2435A43E9
:10517000B4F87E3042F2107101FB0323013B93FB34
:10518000F2F3E28F9BB29A421AD00220FDF760FD43
:10519000064620B941F66F21C748FBF757FB238C21
:1051A000F380082333710023F372B4F87A30B381AB
:1051B000B4F87C30F381B4F87E303382FEF748FDDA
:1051C00023686768002B0ADAA66823F00043BE4212
:1051D0002CBF4E4409EB07062360A6EB0309A38C02
:1051E000B4F87AB0B54913FB08F39BB2B3FBFBF2FA
:1051F0001FFA82FA1BFB0AF080B2834280F0128110
:10520000C01A40F223124243C31701FB0323A0FB41
:1052100001011944A6A3D3E90023FBF781F820F08C
:105220007F4000EB0906238DA3EB0803534423853D
:105230002368BB4238BF3B460C9394F91D3040F2C3
:10524000E249002BD4F884300B9309FB0BF780F272
:10525000FA80E26D636D9A4903FB182395F82021CB
:1052600031F8128094F85020C2F3820231F81220F3
:1052700094F88810904409FB01F107FB08F8616677
:1052800008F5742800218F4A216708F23F288E49CB
:10529000B8FBF2F87A0808FB0AF0963A0344C4F81F
:1052A0005480A265934294BFE365E265A0FB0101CF
:1052B0007FA3D3E90023FBF733F883490B9B361A0E
:1052C000B3FBF9F009FB00F079A3D3E90023A0FBBD
:1052D0000101FBF725F8A7EB080820F07F45B4F89B
:1052E0007E30B4F87C20E28442F2107101FB03733B
:1052F000013BB3FBF7F3E387744BA4F824B03B44C2
:10530000B3FBF7F3A4F84230714B3B44B3FBF7F720
:10531000931DB9B29942C4BFC2F57F43FA33A4F8D2
:105320004A10C8BFC91894F87830C8BF89B213F0C2
:10533000040308BFA4F84030A4F84610002001215F
:1053400008F00AFF0022012182461046FCF78EFC7D
:1053500094F8202041F6F923002107320093D2B2BD
:105360005C4B0846FDF7FAFA30F0020304D041F630
:10537000FB215148FBF76AFA534B94F82070A8FBC5
:10538000038940464AA3D3E900234946FAF7C8FFF8
:10539000514A20F07F4B072320F07F4000214343F8
:1053A00002FB0133A0FB0201B8EB0000194469EBDA
:1053B00001014FF47A720023FAF7B2FFE3680C9A06
:1053C00094F91DE0454902901A441346444A049357
:1053D00012EA2E0238BF0A4641F609310891073712
:1053E0003C490791FFB20021059233460694039190
:1053F0008DE820083A460846FDF712FA30F002031D
:1054000004D041F60B312C48FBF720FABAF1000F1B
:1054100000F057830122114600200FB0BDE8F04F85
:10542000FCF724BC0BFB123292B2A2FB010140F24A
:10543000231303FB02111EA3D3E90023FAF770FF25
:10544000A9EB0006EFE60B9908461F4918A3D3E91C
:105450000023A0FB0101FAF763FF20F07F40451C09
:10546000B8463CE794F87830002B3DD01D48FCF757
:105470005AFB064600283FF4FAAD002384F8783042
:10548000E38C06333B44A4F87E30037943F00303F6
:105490000371082343710123C371052204F17901CB
:1054A0000830FCF73BFAB4F87E30A6F80D30DAE5A8
:1054B0008D49FD1A07000000AC0501000054CE091B
:1054C0009C05010040420F0000CA9A3BFF5962024E
:1054D0007FC3C901B13E00008D49FD1A795C00000F
:1054E0007D5C000090030020B4F87E30FB1A1E049F
:1054F0003FF5BDAD94F8743084F8753004F11706AB
:10550000052204F179013046FCF708FA05213046FE
:10551000FCF7B4FC637F60F3050363770123237713
:10552000A5E594F87880B8F1000F7FF4A0ADD848D5
:10553000FCF7F9FA064600283FF499AD94F91D30BE
:10554000002B00F1040A4DDB04F1F90B5B464246E7
:1055500004F1940104F1840008F096F810225946F1
:1055600004F58D70FCF7DAF904F58971082204F26C
:105570003310FCF7D3F994F8113184F8098168F3FA
:10558000000384F8113194F8323184F80A8143F031
:10559000010384F8323194F8F83084F80B8143F039
:1055A000100384F80C8184F80D8184F80E8184F84E
:1055B0000F8184F81081A4F82A81A4F82C81A4F822
:1055C0002E81A4F8308184F8F83051462046FFF748
:1055D0004DFA31462046FFF7BBF994F8743084F851
:1055E000753044E594F8F83003F04803082B00F0D8
:1055F000A28094F87980B8F1000F20D0037943F0AD
:105600000303037194F85030980612D5D4F8A430EF
:1056100059070ED51123F3710323337286F80980DD
:1056200002237371737901337371002384F8793025
:10563000CFE70D23F37186F808800123F1E7944842
:10564000FCF771FA8246002800F00883037943F0E2
:10565000030303714FF0040B0D23437180F807B06F
:1056600000F108031946082268680D9309F07EFCD2
:105670000AF1100319465A4668680B9309F076FC44
:105680000D9B0822194604F19C00FCF747F95A4685
:105690000B9904F58B70FCF741F95146204604F153
:1056A000F90AFFF755F95346424604F1940104F113
:1056B000840007F0E9FF1022514604F58D70FCF7D5
:1056C0002DF9082204F5897104F23310FCF726F94C
:1056D00094F8113184F8098143F0010384F8113101
:1056E00094F8323184F80A8168F3000384F8323187
:1056F00094F8F83084F80B8143F0100384F8F83004
:10570000337984F80C8143F0030384F80D8184F825
:105710000E8184F80F8184F81081A4F82A81A4F8FE
:105720002C81A4F82E81A4F8308133710123737188
:105730000523F3714DE75146D5F81401FFF796F9AB
:10574000D5F8142192F8F83068F3820368F3C303A4
:1057500082F8F8303DE74E48FCF7E5F906460028A8
:105760003FF485AC94F8743084F87530494BC4F834
:10577000A430037943F0030303710923437194F9BF
:105780001D30002BACBF08230E230822C37100215B
:105790001044FCF7EFF8D4F8A43033721A0A1B0C4B
:1057A0007272B37231462046FFF7D2F8B4F8423035
:1057B000A4F844305BE494F8A830DA0724D43448E1
:1057C000FCF7B1F9014600283FF451AC94F874306D
:1057D00084F8753094F8A83043F0010384F8A830B9
:1057E000037943F003030371062343710C23C37150
:1057F000092303726FF00E034372052383724FF087
:10580000FF33C3720373CEE79B0727D594F8743038
:1058100084F875300220FDF71BFA064620B941F6E0
:105820004F411D48FBF712F8238CF380012333719D
:10583000337A43F003033372062373720C23F3723B
:1058400094F8A9303373B4F8AA30A6F80D30B4F840
:10585000AC30A6F80F30FEF7FBF908E441F66741DB
:105860000D48FAF7F3FF02E40948FCF75CF901463A
:1058700000283FF4FCAB94F8743084F87530037959
:1058800043F003030371012343711223C3718AE7B9
:1058900090030020FF490100AC05010094F8782036
:1058A000D60758D5BE48FCF73EF9064600283FF417
:1058B000DEAB94F878306FF3000384F87830DBB215
:1058C000C3F3820252EA53123FD194F8741084F861
:1058D00075109807A4F87A2020D50220FDF7B8F9B2
:1058E000804620B941F6F761AE48FAF7AFFF238C46
:1058F000A8F806300C2388F80430002388F80B3011
:1059000094F83830C3F3C20388F80C3094F83A3076
:10591000C3F3020388F80D30FEF79AF9337943F0A8
:1059200003033371052373711823F37194F87830EE
:10593000C3F38203337294F87830C3F34213737263
:10594000B4F87A307381FFF78EBBE38C06333B44A7
:10595000A4F87A30E2E7B4F87A30FB1A19043FF57C
:1059600086AB94F8743084F8753012F01C0F94F8FC
:10597000383094F83A1018BFC2F38206C3F3C2005D
:105980001CBF66F3C50384F8383012F0E00F01F055
:10599000070108D094F8783094F83A605B0963F313
:1059A000020684F83A6094F838301E46C3F3801338
:1059B00063F3C716930784F838600BD4F3B2C3F3CC
:1059C000C203834206D194F83A3003F007038B42B6
:1059D0003FF44DAB0220FDF73BF9064620B941F6F6
:1059E00037717048FAF732FF238CF3800C23337140
:1059F0000023F37294F83830C3F3C203337394F87E
:105A00003A30C3F30203737325E741F6B37127E716
:105A1000FDF708F90646D5F83001FCF7B3F806445F
:105A2000B6B2FF2E04D94FF4ED515E48FAF70EFFDF
:105A300095F83A31B3422BD15948FCF774F8014636
:105A400030B394F8EA30B4F8EE00A085012262F396
:105A50000103B4F8F220628684F8EA300B79888179
:105A600043F003030B7109234B711423CB711B23E8
:105A70000B7200234B726FF06F038B720A23CB7291
:105A8000CA812046FEF764FFB4F84230A4F84430DF
:105A900094F8203094F91D5043484449A268039477
:105AA000073311EA250138BF0146DBB28DE80C004F
:105AB0000291231D22460C9948460137FEF71CFC33
:105AC00067840FB0BDE8F08FFDF7ACF80646D5F857
:105AD0003001FCF757F80644B6B2FF2E04D941F660
:105AE000E1513048FAF7B2FE95F83A31B34204D0AA
:105AF00041F6E7512B48FAF7A9FE94F8E83084F80C
:105B0000E930D5F814310021A4F8441093F8F820B6
:105B100061F3C30283F8F820B4F8EC302386B4F8BC
:105B2000F030E386D5F80C01FCF72CF8D5F8CC3032
:105B30000BB1013080B2D5F800310BB1013080B229
:105B4000268E95F810310E36013026F00306984265
:105B5000B6B278D0B5F83831B34274D30220FDF72D
:105B600077F8054620B941F64A610E48FAF76EFE0D
:105B7000238CEB8001232B712B7A43F003032B72D0
:105B800009236B721523EB72238EAB81E38D2B827D
:105B9000E38EEB81A38E6B82FEF75AF878E700BFA5
:105BA00090030020AC050100DD610000E95C00000D
:105BB0000BB995F84031013B85F8423195F8422107
:105BC000D5F83C3153F8223041461868FBF7C5FF41
:105BD00095F8403195F85421013B9A4204DB41F697
:105BE00023615046FAF732FE95F85431013385F8B7
:105BF000543195F8423195F841219342D8D1238E02
:105C0000292B9ABF3423A5F83831A5F83861B5F8A7
:105C10003631B5F83821B3FBF2F3DBB285F83A310F
:105C200023B941F63A611048FAF710FED5F82C0175
:105C30000E4B95F83A21B5F83811FBF74DFF0420CB
:105C4000FDF790F88AE7DFF82C80DFF81CA0D0E79A
:105C500041F66C610448FAF7F9FD19E7044930464A
:105C6000FBF77BFFFFF703BAAC05010064030020DC
:105C7000900300207C030020FEF73ABFFEF738BFF8
:105C8000084A08B593601346002211461046FCF7F7
:105C900015F830B141F274510348BDE80840FAF7F5
:105CA000D5BD08BD44450020AC05010010B5044633
:105CB00007F062FE002007F0A7FE0A4807F026FE64
:105CC00004F1100007F0C6FE637DA17D1B0243EACC
:105CD0000143217D40F25B601943BDE8104007F0AD
:105CE00073BF00BFF97400002DE9F041694D1C46F7
:105CF0002B7D074623B142F21E016748FAF7A6FD45
:105D0000238C6A7C07339A4204D042F22101624814
:105D1000FAF79CFD03232B7501236B7594F8203053
:105D2000C5F814410026073385F8186185F8196114
:105D3000DBB26E74AB74238D638520462685AF601D
:105D4000FFF7B4FF962007F0FBFF94F8382094F893
:105D50003A00D3093146C2F3C20200F0070007F04F
:105D60005DFF95F84121D5F83C3153F822102046CB
:105D70000831FDF785FA637F13F0400F04F1170235
:105D800059D0608CE18B013803F03F0380B2FEF7FD
:105D900045FCFDF7DDFB236EE26D13440022E26556
:105DA000A26D2366934288BF2266A36E626E0026B0
:105DB0001344A366EA68666607F10901304607F0F6
:105DC000CBFF804608F05AF8304608F079F8A36E09
:105DD000206E03F1500606EB400694F83A000121CC
:105DE00000F0070007F097FE4644064494F83A0096
:105DF00000F0070002283ED004280CBF4FF4BC730B
:105E0000282301211E4407F088FE304408F018F8CA
:105E100094F8201007313A46C9B22046FEF742FCFA
:105E2000034650B304236B7507F092FE0220BDE8D1
:105E3000F041FDF77DBA618DA67F01FB0666E17F2B
:105E400025200E4496FBF0F100FB1166F0B2C1086C
:105E5000E077515C06F0070641FA06F6F10703F019
:105E60003F0396D4B0FBF3F103FB1101C9B2104616
:105E7000FCF7BCFE8DE71823C3E7084A0146FCF790
:105E8000EBFD30F00203D1D042F2A5010248FAF74F
:105E9000DDFCCBE734020020AC0501006D3F0000C3
:105EA00090F8F8C01CF0800F2DE9F04104460E4632
:105EB00009D1D0F83C1131B11CF0080FD0F840E105
:105EC00023D0714521D094F8F83043F0800384F852
:105ED000F83007F08FFE0378012262F301030022FD
:105EE0004270D4F83C210370DBB25AB143F0100386
:105EF000037003786FF347130370002383703060DF
:105F0000BDE8F08162F30413F2E794F8512194F8AC
:105F100050310D1DA81813B9437884F8503122B1BF
:105F2000AB5C012767F30103AB5494F8507194F80C
:105F30003980BF1AFFB24770AB5C6FF30413AB54E8
:105F400008F00708B8F1020FA38E29D0B8F1040FAA
:105F500029D0DB080A3B9BB21CF0200F18BF043B82
:105F6000B4F82EC018BF9BB2634528BF63469F425A
:105F700081BF4370AB5C43F01003AB540B681BB1A3
:105F8000AB5C43F01003AB54BEF1000FB1D1D4F8B9
:105F9000483199421CBFC4F84411C4F84011A8E725
:105FA0009B080B3BD7E794F838805FEAD81815BFF9
:105FB000A3F51473A3F5D7739B111B11023BCAE71A
:105FC000F0B58FB002230993FF2200237C4E7D4F52
:105FD0007D4D0A9304460B938DF823200C9309AB57
:105FE00002930CAB009301960DAB0DF1230201213E
:105FF0000020FCF7EFFC022825D0099B23B141F2D9
:10600000F3213846FAF722FC9DF82330FF2B04D009
:1060100095F8102107329342E1DA5A1FD2B2F92AD9
:106020006A4F05D8684A92F81021073293420EDB76
:106030003B7813B10120FDF7C3FF0FB0F0BD012184
:106040000020FCF745FD099B022BF8D0D5E70AA9F3
:10605000E0B2FDF797FF054620B941F203315948F8
:10606000FAF7F4FB2B686C689DF82300002BB8BF8F
:10607000AB689C4238BF1C46EB680BA91C44FDF77B
:1060800081FF054620B941F211314E48FAF7DEFB97
:10609000AE686B682A689E4238BF1E46002A05DA41
:1060A0000C9B22F0004233449B1A0C930C9A04F18F
:1060B000310393420BD23B7813B10120FDF780FFEF
:1060C0009DF8232001212846FEF7AAF8B5E73A7883
:1060D0005AB901203E4B38701146FBF7EFFD20B155
:1060E00041F24C213748FAF7B1FB2B68002B19DB42
:1060F0009E4217D29B1B00209BB23649059102930A
:106100009DF82320069504900390019000900121B2
:10611000FCF7D6FB30F0020304D041F23D312948B0
:10612000FAF794FB0A9E002E87D00B9D002D84D099
:10613000B38CAA8C9A4280D1274892B2A2FB00016C
:1061400040F2231303FB02111BA3D3E90023FAF748
:10615000E7F80C9B20F07F400022984218D302B150
:106160000C9396F91D20002A95F91D2013DA002AB8
:10617000FFF663AF14349C427FF65FAF3046FCF706
:1061800079FD02287FF459AF0B98FCF773FD54E7B3
:106190001B1A0122E1E7002ABFF64FAF14349C42DC
:1061A0007FF64BAF2846FCF765FD02287FF445AF2C
:1061B0000A98EAE7AFF300808D49FD1A0700000056
:1061C000C12B0000AC050100340200205404002063
:1061D000B4450020D52B00000054CE09F7B54F4D33
:1061E0001C462B7D074623B142F2C6014C48FAF704
:1061F0002DFB238C6A7C07339A4204D042F2C901FA
:106200004748FAF723FB04232B7594F82030C5F890
:1062100014410022073385F8182185F81921DBB2D3
:106220006A74AB74238D6385022022856875AF6024
:10623000FDF77EF801A92046FFF732FE019994F898
:10624000F8200B7862F3C303C2F3400262F38203C7
:106250000B702046FFF72AFD962007F071FD94F899
:106260003A0000F0070007F0CDFC01992046FDF749
:1062700043F9637F13F0400F04F1170221D0608CC3
:10628000E18B013803F03F0380B2FEF7C7F9FDF759
:106290005FF9EA6807F10901012007F05DFD07F0E9
:1062A00021FE94F8201007313A46C9B22046FEF785
:1062B000F9F9034628B304236B7507F049FC03B0D2
:1062C000F0BD618DA67F01FB0666E17F25200E44AF
:1062D00096FBF0F100FB1166F0B2C108E077515C6B
:1062E00006F0070641FA06F6F10703F03F03CED4A5
:1062F000B0FBF3F103FB1101C9B21046FCF776FCC9
:10630000C5E7084A0146FCF7A7FB30F00203D6D0E8
:1063100042F276110248FAF799FAD0E734020020E7
:10632000AC0501006D3F00002DE9F04FC67A85B045
:1063300004460D4600F10807192E01F2A980DFE896
:1063400016F01A007A00B600C500F3001B014001E8
:106350009B058801AD01D801010233029C029E0118
:10636000B4020404870470058A051F061F06F6069A
:10637000B807EF077408C74ED6F8145195F91D30C9
:10638000002B81F28580417A0020FCF7FBFB00287E
:1063900001F07E80B4F815106B8CCB1A1A0401F151
:1063A000938095F8743095F875209A4241F0878073
:1063B000D6F888210AB9C6F88851227B85F888204A
:1063C000B4F80D0040F2E2424243C5F88420207C3C
:1063D000E27B42EA0022A5F87A20A07C627C42EAB5
:1063E0000022A5F87C20E27C207DA5F8801042EAFE
:1063F0000022A5F87E2095F8782002F0FC026FF3C9
:106400008202013B85F87820012285F8762085F804
:10641000753095F8C02095F8C130934207D095F8B3
:10642000C23003F00703042B01D185F8C1200020FE
:10643000A5F8440038E0974BD3F8145195F91D3076
:10644000002B81F22580417A0120FCF79BFB00287C
:1064500001F01E80B4F811306A8C9B1A1B0401F104
:10646000338095F8742095F875309A4204D042F242
:1064700044418948FAF7EAF9052204F10C0105F1D3
:106480007900FBF74BFA637CA27C002043EA0223ED
:10649000A5F87E3085F87800022385F8763095F8E7
:1064A0007530013B85F8753005B0BDE8F08F417A55
:1064B0000220FCF767FB002800F0EA87754B227B7F
:1064C000D3F8143183F8B3200020EDE7714ED6F8ED
:1064D000147197F91D30002B80F2DA87417A03207E
:1064E000FCF750FB002800F0D387082204F11601C6
:1064F00007F19400FBF712FAD6F81401042204F114
:106500001E0100F58970FBF709FAD6F8143193F8EB
:10651000F82042F0040283F8F820B3F84220A3F8F0
:10652000442001232B70CFE75A4DD5F8146196F91A
:106530001D30002BC0F2AC87417A0420FCF722FB0F
:10654000002800F0A587082204F10C0106F19C0048
:10655000FBF7E4F9D5F81401042204F1140100F565
:106560008B70FBF7DBF9D5F8142192F8F83043F083
:10657000040382F8F830A7E7464DD5F8142192F8C5
:10658000740092F87510884208D092F87630032B88
:1065900004D040F6E8114048FAF758F9D5F81451FC
:1065A00095F91D30002BC0F27387617A0520FCF746
:1065B000E9FA002800F06C87002085F878000323B2
:1065C0006BE7417A0620FCF7DDFA002800F06087CF
:1065D000304E337D032B31D1D6F8143193F874103B
:1065E00093F87520914208D093F87630032B04D0AD
:1065F00040F601212848FAF729F9D6F8143100228B
:1066000083F87820032283F8762093F87520013AE6
:1066100083F87520D6F8142192F8F8305F0641BF50
:106620006FF3861382F8F8300923237101232B704E
:10663000D6F814310020A3F8440035E7D6F8142129
:1066400092F8F83003F0FB036FF3C30382F8F830DD
:10665000E0E7104BD3F8145195F91D30002B80F270
:106660001787417A0820FCF78DFA002800F0108780
:106670003946284605B0BDE8F04FFEF7B1B9054BE5
:10668000D3F8145195F91D30002BC0F20187417ADF
:106690000E20E8E734020020AC050100417A092011
:1066A000FCF770FA002800F0F386237B617BB0488A
:1066B00043F07F4343F47E0343F4435343F010031A
:1066C000D0F8142143EA0123A17B43EA0143D2F825
:1066D000A410C1F310010B40C2F8A43092F850305E
:1066E00043F0200382F8503001232B70D0F814318E
:1066F000A0E79F4ED6F8145195F91D30002B80F27B
:10670000C786417A0A20FCF73DFA002800F0C086CF
:1067100006F5AE70FBF707FA014608B90120C3E69B
:1067200095F8F83043F044036FF3041385F8F8301C
:10673000037943F003030371012343710B23C371F6
:10674000284627E0417A0B20FCF71CFA002800F0CD
:106750009F868748D0F8144194F91D30002B1CDB2C
:1067600000F5AE70FBF7DFF901460028D6D094F8AB
:10677000F83003F0DF0343F004036FF3041384F8ED
:10678000F830037943F003030371012343710B23B2
:10679000CB712046FEF7DCF896E694F8F8306FF3FC
:1067A000451384F8F8308FE6417A0C20FCF7EAF9BB
:1067B000002800F06D866E48D0F8146196F8A83075
:1067C00013F0010750D100F5AE70FBF7ACF90146AC
:1067D0000028A3D096F8A83043F0010386F8A8302B
:1067E000037943F003030371062343710C23C37140
:1067F000092303726FF00E034372052383724FF077
:10680000FF33C37203733046FEF7D0F896F8F830C2
:1068100043F0800386F8F83007F0ECF9037847700E
:10682000012262F30103D6F83C210370DBB2C2B14E
:1068300043F010030370237B86F8A930A27B637BAF
:1068400043EA0223A6F8AA30E37B227C43EA022330
:10685000A6F8AC3096F8A83043F0020386F8A830CA
:1068600032E662F30413E5E713F002037FF42CAE83
:10687000A6F8443001232B70DDE7417A0D20FCF7A8
:1068800081F9002800F00486394BD3F8142192F8DE
:10689000F83003F0FB036FF3C303002082F8F830F5
:1068A000A2F8440001232B70FEE5417A0F20FCF78B
:1068B00069F9002800F0EC852D4BD3F888111A46B1
:1068C00051B1D3F81401814206D020220F2105B026
:1068D000BDE8F04FFEF7EEB8D2F8140190F91D3084
:1068E00090F8C010002B90F8C130C0F2A6809942F9
:1068F00009D090F8C23013F0070302D0043B012BFB
:1069000001D82322E2E790F8741090F8753099428C
:1069100003D090F87630032B05D190F8F41090F85E
:10692000F530994201D02A22D0E7B4F80C804346D2
:10693000052B1BD9E789B7F5486F17D8B84515D887
:10694000B4F810C0BCF5FA7F10D2B4F812E0AEF182
:106950000A06B6B240F676494E4507D80CFB0771D9
:10696000B1EB8E0F02DA217D8F4203D21E22ADE7FA
:1069700034020020A0F8C480A0F8C6C0A0F8C8E087
:1069800080F8CA10A67D617D41EA0621A0F8CC10EE
:10699000267EE17D41EA0621A0F8CE10A67E617E2A
:1069A00041EA0621A0F8D010267FE17E41EA0621C7
:1069B000A0F8D210A67F617F41EA0621A0F8D4108A
:1069C000E17F94F8206041EA0621A0F8D61094F8FF
:1069D000211094F8224041EA0421A0F8D810D0F800
:1069E000C440416A8C420FD1848C40F2E241614341
:1069F00042F2107404FB0E13013B93FBF1F3C18FC1
:106A00009BB2994200F0928090F8F8301C0740F158
:106A1000878090F8C230022161F3020380F8C2300F
:106A200090F8C130013B80F8C130D2F88831002B9A
:106A30007FF44AADC2F8880146E5994203D090F848
:106A4000C23099077BD1B4F80C804346052B8DD911
:106A5000E789B7F5486F89D8B84587D8B4F810C02A
:106A6000BCF5FA7F82D2B4F812E0AEF10A06B6B2F3
:106A700040F676494E453FF679AF0CFB0771B1EB16
:106A80008E0FBFF673AF217D8F42FFF46FAFA0F87A
:106A9000C480A0F8C6C0A0F8C8E080F8CA10A67DDF
:106AA000617D41EA0621A0F8CC10267EE17D41EA15
:106AB0000621A0F8CE10A67E617E41EA0621A0F84C
:106AC000D010267FE17E41EA0621A0F8D210A67FF1
:106AD000617F41EA0621A0F8D410E17F94F820609C
:106AE00041EA0621A0F8D61094F8211094F822402B
:106AF00041EA0421A0F8D810D0F8C440416A8C4281
:106B00000ED1848C40F2E241614342F2107404FBE6
:106B10000E13013B93FBF1F3C18F9BB2994205D059
:106B200001232B7090F8C230032175E7002380F811
:106B3000C33090F8C230012103F0F7036CE740F650
:106B40004F31CB48F9F782FEBEE4CA4BD3F814515B
:106B500095F91D30002BC0F29B84417A1020FCF780
:106B600011F8002800F0948495F8C02095F8C13001
:106B70009A423FF4A9AC95F8C23003F00703042B06
:106B80007FF4A2ACB4F80CE01FFA8EF2052A1BD9F0
:106B9000E389B3F5486F17D89A4215D8278ABAB255
:106BA000B2F5FA7F10D2668AB0B2A0F10A0189B2BA
:106BB00040F6764C614507D802FB0332B2EB800FFA
:106BC00002DA227D934203D21E22102128467EE65D
:106BD0000020A5F84400A5F8C4E0A5F8C670A5F803
:106BE000C86085F8CA20A27D637D43EA0223A5F828
:106BF000CC30227EE37D43EA0223A5F8CE30A27E8C
:106C0000637E43EA0223A5F8D030227FE37E43EA85
:106C10000223A5F8D230A27F637F43EA0223A5F8BE
:106C2000D43094F82020E37F43EA0223A5F8D6303D
:106C300094F8222094F8213043EA0223A5F8D830B2
:106C400095F8C230012262F3020385F8C2302BE4CA
:106C5000417A1120FBF796FF002800F01984854F38
:106C6000D7F8146196F8F53096F8F4108B42237B30
:106C700027D0162B7FF428AC627B232A0ED096F8FF
:106C8000383086F8F51096F83910C3F3C20363F371
:106C90000201002386F83910A6F8443096F8F73040
:106CA0009B077FF511AC0C23E272237196F8383004
:106CB000C3F3C203237396F83A30C3F3020363733A
:106CC0002FE496F8C11096F8C020914275D00F2B92
:106CD0007FF4FAAB96F91D30002B637B3ADB1A2B5D
:106CE00038D196F8742096F875309A4204D040F264
:106CF00095715F48F9F7AAFD96F8C230052262F354
:106D00000203B6F8C420A6F87A20B6F8C620A6F882
:106D10007C20B6F8C820A6F87E2096F8782086F861
:106D2000C230012183F00803C3F3C00361F3010201
:106D300063F3820296F8753086F888100020013BD4
:106D4000C6F8840086F8782086F8761086F87530C4
:106D5000FFF7AABB232B18D0D7F888319E4204D066
:106D600040F2AC714248F9F771FD0023C7F8883151
:106D7000A6F8443096F91D3096F8C02086F8C12058
:106D8000002BBCBFD6F8E430336796F8C2301F073B
:106D90007FF59AAB08232371637BE372F28CB38C8B
:106DA000E281F28FA3815A437D2353434FF47A72D9
:106DB00093FBF2F32382FFF7B4BB96F8E82096F832
:106DC000E91091421AD0142B7FF47EAB96F8F8307C
:106DD00086F8E920002060F3C30386F8F830092321
:106DE000A6F8440063721523E372338EA381F38DFA
:106DF0002382F38EE381B38E638253E5032B7FF40A
:106E000063AB96F8F83003F0FB036FF3C303002085
:106E100086F8F830A6F844000D23E372637B2373F1
:106E200040E5417A1220FBF7ADFE002800F03083E8
:106E30001048D0F8144100F5AE70FAF774FE014620
:106E400000283FF46BAC037943F003030371012383
:106E5000437113239CE4417A1320FBF793FE00282F
:106E600000F01683034BD3F81431FFF7E3BB00BFE8
:106E7000AC05010034020020417A0720FBF782FEB6
:106E8000002800F00583C24FD7F8146196F8C1209E
:106E900096F8C0309A423CD096F8C23043F01003C6
:106EA00086F8C23096F91D30002B09DB96F8742065
:106EB00096F875309A423FF41FAF40F6BB3118E7A1
:106EC000D7F888319E4204D040F6D231B148F9F764
:106ED000BDFC0023C7F8883196F8C03086F8C13071
:106EE00096F8C23018077FF5EFAA082323711A23FA
:106EF000E372F28CB38CE281F28FA3815A437D233B
:106F000053434FF47A7293FBF2F3238201232B70E5
:106F100032E096F8E83096F8E9209A4208D086F8F0
:106F2000E93096F8F8306FF3C30386F8F830EDE7F0
:106F300096F8F43096F8F5209A421AD086F8F53093
:106F400096F8383096F83920C3F3C20363F302028F
:106F500086F8392096F8F72091070DD50C2222717A
:106F60000022E272237396F83A30C3F3020363738C
:106F7000CCE7237B122BC9D1D7F81431FFF75ABBCA
:106F8000417A1420FBF7FEFD002800F08182142EC8
:106F90002BD18148FAF7C7FD064600283FF4BEAB67
:106FA0007B49D1F8140190F8E97090F8E8E0038E7D
:106FB00000937745C38D0193828EC38EE77A8A460C
:106FC00015D1142F1FD0152F00F0898240F62811FB
:106FD000704803920293F9F739FC039A029B90469A
:106FE0009946019FDDF800B062E00026D8E790F8EE
:106FF000EA1001F003010129E3D90229E3D1A7F145
:1070000014010129DFD8A1891A2968D9878D8F42F7
:1070100028BF0F46218A1B29009938BF8B46E1897A
:1070200028BF4FF01B0BB1F5A47F5AD3B0F83280C4
:10703000884528BF8846B4F81290B9F5A47F52D38A
:10704000B9F5296F28BF4FF42969009959454CD0EB
:10705000FBF7E8FD0446DAF83001FAF793FD044443
:10706000A4B2FF2C04D940F6D1014A48F9F7EEFB4F
:107070009AF83A31A34240F02982DAF8143193F8B1
:10708000E820DF85013A83F8E92093F8EA20A3F8A5
:10709000ECB042F00302A3F8EE70A3F83480A3F83A
:1070A000F090A3F8F28083F8EA2003238AF81530E1
:1070B000002E3FF409AA3379DAF81401A6F808B0D3
:1070C00043F003033371092373711523F371B781FF
:1070D000A6F80A90A6F80E803146FFF75BBB019F29
:1070E00098E79046A7E79946AFE790F8F81080F840
:1070F000E9E04FF0000E6EF3C30180F8F81001993B
:10710000A0F844E0B94203D1424501D14B45CFD06C
:107110000123C785A0F83690A0F83480A4F80CB0FD
:107120002782A4F80E90A4F812802B70C0E7417A51
:107130001620FBF727FD002800F0AA811448037DE4
:10714000042B5ED1D0F8140190F8F53090F8F410CB
:107150008B420AD090F8F62002F00302013A022A8C
:1071600003D823221621FFF7B2BB90F8745090F891
:107170007520954203D090F87620032A05D190F827
:10718000C05090F8C120954208D02A22EAE700BFFB
:1071900034020020AC0501009003002090F8F62096
:1071A0008B4242F0030280F8F62016D1013B80F8B2
:1071B000F53090F8F73090F838206FF3410380F8FD
:1071C000F73090F8F63062F3840390F83920C2F378
:1071D000C20262F3471380F8F63090F8F630627B13
:1071E000C3F382010A4062F3840380F8F630227B05
:1071F000DBB202EA531262F3471380F8F630FFF76E
:1072000063B9D0F8145100F5AE70FAF78CFC014662
:1072100000283FF483AA95F8F630022262F30103B6
:1072200085F8F63095F8F52095F8F43093421AD1A8
:10723000013B85F8F53095F8F73095F838206FF375
:10724000410385F8F73095F8F63062F3840395F83A
:107250003920C2F3C20262F3471385F8F630B5F85D
:107260004230A5F8443095F8F630627BC3F38200D3
:10727000024062F3840385F8F630227BDBB202EA37
:10728000531262F3471385F8F6300B7943F003038A
:107290000B7103234B711723CB7195F83830C3F36F
:1072A00002030B7295F83930C3F3C2034B72FFF738
:1072B00047BA8F4ED6F8145195F91D30002BC0F205
:1072C000E780417A1720FBF75DFC002800F0E080A2
:1072D000337D042B7FF4F8A895F8F52095F8F43069
:1072E0009A423FF4F1A895F8F63003F00302022A1F
:1072F0007FF4EAA843F0030385F8F630627BC3F31A
:1073000082010A4062F3840385F8F630227BDBB207
:1073100002EA531262F3471385F8F630FFF787B895
:10732000734BD3F8146196F91D30002B80F2B080B6
:10733000417A1820FBF726FC002800F0A980277B63
:10734000627B47EA020010F0070025D196F8F4208E
:1073500096F8F53093423FF4B7A896F8F63003F06C
:107360000303022B7FF4B0A896F8F73086F8F520D7
:107370009A07A6F844007FF5A7A80C23E0722371B2
:1073800096F83830C3F3C203237396F83A30C3F348
:1073900002036373FFF786BAE089738CC31A1B0478
:1073A00000F19F8096F8741096F875308B4240F08B
:1073B0009D8096F8F44096F8F530A34214D096F8E4
:1073C000F63003F00303022B0ED196F8F73086F85F
:1073D000F54096F87840C3F3400363F3410400237B
:1073E00086F87840A6F8443096F87830A6F87A0007
:1073F00002F0070262F3840367F347136FF300039D
:1074000086F878300820013903F01C0386F87600EE
:1074100086F87510002B3FF457A896F8393062F3C0
:10742000020386F83930FFF74FB8314ED6F81451C1
:1074300095F91D30002B2BDB417A1920FBF7A2FBBD
:1074400030B395F8382095F83A3043EAD203227BDE
:1074500003F0070313423FF437A895F8742095F81A
:1074600075309A427FF430A8052206F58D7105F13A
:107470007900FAF753FA012385F87830022385F86A
:10748000763095F87530013B85F87530FFF71CB8FC
:107490001748E47AD0F8145100F5AE70FAF743FBC0
:1074A000014600283FF43AA90379047243F003032C
:1074B0000371022343710723C371FFF741B92A23E4
:1074C00085F8B330FFF700B82823F9E7002E3FF422
:1074D00025A908493046FAF740FBFFF71FB9904647
:1074E0007EE5282386F8B330FEF7EEBF2A23F9E7BE
:1074F00034020020900300202DE9F04F95B006F0F3
:107500004FFBC6B266B306F06BFBC7B206F0ECFBEE
:107510005FFA80F906F0F2FB5FFA80F806F0F4FDFE
:107520005FFA80FA06F0DEFD5FFA80FB06F0A6FB4C
:10753000C5B2B44C06F01EFB06F0F2FB06F0CCFB25
:1075400006F0D6FD06F092FB637D052B01F2E68383
:10755000DFE813F07D00D0000E00CA09CA09CA098D
:107560004FF0FF0B3546B246B1463746D846E0E706
:107570000123637506F0CEFC0546962006F0E0FB7D
:10758000237D013B032B00F2AF80DFE803F0022FE5
:10759000636300231A461946184606F03FFB06F0BF
:1075A0002DFB06F0A1FA06F0F1FA20B140F28D2190
:1075B0009548F9F74BF905F079FC38B112A805F0B8
:1075C00019FA01469DF8480006F05AFD00210846C8
:1075D00006F0A3FAC33500210544084606F099FADF
:1075E000281A06F02DFC06F07DFC30E000231A4638
:1075F0001946184606F012FB94F84121D4F83C31A4
:1076000053F82200083006F06FFA06F0BFFA20B1F6
:107610004FF42D717C48F9F719F905F047FC38B1A2
:1076200012A805F0E7F901469DF8480006F028FD8C
:107630000021084606F071FAC335002105440846CA
:1076400006F067FA281A06F0FBFB06F0FFFA15B001
:10765000BDE8F08FD4F8143193F8382093F83A004D
:107660000021D30900F00700C2F3C20206F0D6FAE7
:1076700094F84121D4F83C31D4F8140153F8221085
:107680000831FBF7FDFD06F081FA20B140F2E5215B
:107690005D48F9F7DBF8D4F8143193F83A0001218A
:1076A00000F0070006F039FAD4F8142192F83A30C5
:1076B00003F007039B35022B054413D0042B0CBFAA
:1076C0004FF4BC702820054492F83800C109C0F37B
:1076D000C20006F01EFA281A06F0B2FB0120FBF7E2
:1076E00027FEB4E71820EEE740F215314648F9F7D7
:1076F000ADF8ACE726B90323637506F029FAA6E7CF
:10770000237D013B032B01F2EB80DFE813F0040043
:107710009D02BB05BB05002FEDD0BAF1000F39D09B
:10772000584605F09FF98DF8480006F067FA94F87E
:10773000792006462B232721007811FB02330B9377
:10774000E51800F00F03032B0AD173780C2B07D137
:1077500094F829305F061FD594F82930580647D48D
:10776000307800F00F03052BC5D17378222BC2D1DE
:107770000B9BE35C03F00F03012B40F01E82B71C50
:1077800012AA3946C0F3801005F034FB00283DD121
:1077900000204BE0FF20C6E712AAB11CC0F3801006
:1077A00005F028FB0028D7D00B9B3278E35CC3F3AD
:1077B0008013B3EBD21FD3D1062206F10801A81C17
:1077C000FAF797F80028CBD10323637506F030FA57
:1077D00094F8C900272303FB00407B3006F08AF9A8
:1077E00006F0D4F900283FF432AF40F2BB317DE718
:1077F000B9F1000FD8D19DF8480005F05DF90028D7
:10780000D2D1ADE734020020AC0501003146284654
:10781000FCF7FAF90028BBD09DF84830FF2B00F0A8
:10782000B98194F82A00C11A4842484100F0010089
:1078300000283FF460AF94F8823133B194F880317E
:1078400094F881219A427FF456AFD4F8CC30002BC3
:107850003FF451AF0420FBF7FBF9074600283FF443
:107860004AAF4FF0040984F8159006F071F9D4F886
:10787000CC50D4F8081100234FF4AA722846C4F85B
:10788000CC30FAF788F905F1100A2884032206F1B2
:10789000120105F11400FAF741F805F117084A46FC
:1078A00006F10E015046FAF739F8052206F11E01DD
:1078B0004046FAF733F805214046FAF7DFFA6B7FC6
:1078C00060F305036B7796F82330C3F30403AB77BB
:1078D000338BAB8440F2E24808FB03F8F27EB37EC0
:1078E00043EA022351464A46EB8405F16C00FAF75D
:1078F00015F8B38BE98C42F2107202FB0383013B53
:10790000B3FBF8F3EB87C64B4344B3FBF8F3A5F89E
:107910004230C44B881D4344B3FBF8F39AB2824211
:107920001346C4BFC1F57F43FA33A5F84A20C4BF4C
:10793000D21892B22B8CA5F846203146FB8001224A
:107940000023FB723A7311F8082B0D934FF00609D0
:10795000C2F3C012BA7687F804904A4607F11B00BA
:10796000F9F7DCFF9DF8480007F10E03FF280C93A0
:1079700006F1020A07F1140B0D9B00F03D810C9AF1
:1079800007F10D0105F00CFA7B7B02337B734A464D
:1079900051465846F9F7C2FF338BA7F82130738B55
:1079A000A7F82330B38BA7F8253096F82330C3F31C
:1079B000421387F82730288CFCF760FAFCF748F967
:1079C0000320FBF745F9074620B94FF48861964834
:1079D000F8F73CFF2B8CFB800B233B71337813F0C3
:1079E00020030ED06A7C2B7CE97C43EA0223AA7C2C
:1079F00042EA0122697F534041F04001EB836977FD
:107A00000123FB72FCF724F996F8232095F85030F7
:107A10008649520962F3840385F8503094F8203186
:107A200031F8122031F81330134408FB03F303F547
:107A300074237F4A03F23F23B3FBF2F36B654FEAF3
:107A40005803963BAB65737D40F2E249002709FB82
:107A500003F3AB6639466F66384606F05CF8754945
:107A6000834600F252406CA3D3E90023A0FB01013E
:107A7000F8F756FCD4F884316B602722934238BF64
:107A8000134620F07F409A466B6D2A60E860AF6035
:107A9000A8EB030806F038FA0C90F08A394600FB90
:107AA0000999384606F035F80C9BA9F1300999443C
:107AB000A9EB0009A9EB0B030C9340F2864300935A
:107AC00005225D4BDFF86CB139463846FAF746FFC0
:107AD00040F28741FCF7F6F90B9BE35C03F00F03E0
:107AE000012B06D100973B46032239463846FAF768
:107AF00035FFA8FB0B8948A3D3E90023404649463C
:107B0000F8F70EFC95F82030A46806950733DBB231
:107B10000B9340F29E430893484B0793484B0593C1
:107B2000EB68484A53440646049320F07F400723FD
:107B30000021434302FB0133A0FB02121A44084612
:107B4000B8EB0000114669EB010100254FF47A7291
:107B500000230395F8F7E4FB0C9902902EA3D3E9D8
:107B6000002326F07F46A1FB0B010196F8F7D8FB16
:107B7000A4EB0A0420F07F40009023460B9A29468C
:107B80002846FAF74DFE30F002033FF460AD4FF4A3
:107B90009461ABE50B9BE25C3378C3F38013B3EBEA
:107BA000D21F7FF4F5AD0622394605F10800F9F73A
:107BB000A0FEB0FA80F0400938E694F82930DB09DD
:107BC0000DD094F82930DB093FF4E2ADB9F1000F94
:107BD0000DD19DF8480004F06FFF40B9D8E512AA16
:107BE000B11CC0F3801005F005F90028E9D031463A
:107BF0002846FCF709F819E619464A465846F9F7A7
:107C0000B9FE33780C98C3F380137B734A46514610
:107C1000C0E600BFAFF300808D49FD1A07000000E9
:107C2000FF5962027FC3C901AC0501009C05010038
:107C300040420F0000CA9A3BC53E0000B13E000022
:107C40007D5C00008D49FD1AB9F1000F1CD094F83D
:107C5000E1004146C0F3001004F0D6FE804647B173
:107C600094F8E130DA0619D594F8E130DB0600F13A
:107C7000DB810323637505F06BFF94F8E0306FF34D
:107C8000410384F8E030E2E4BAF1000F03D0584633
:107C900004F0E8FEE2E74FF0FF08E0E7B9F1000F7B
:107CA00005D04146504605F057F80028DCD00023A7
:107CB0008DF8483094F84121D4F83C3153F82290A3
:107CC000D4F8003109F10806002B00F0DB8194F8AC
:107CD000823133B194F8803194F881219A4240F096
:107CE000D18194F8E130C3F30010002800F0BC818A
:107CF00099F8080010F00F0040F03C8206F004F9FB
:107D0000D4F8DC3000F21627D1480722A3FB00018B
:107D100002FB0311CAA3D3E90023F8F701FBA0F586
:107D20009670874280F0AE810420FAF791FF0746F3
:107D300000289ED0042363750023D4F80061C4F8A2
:107D4000003105F05BFF037803F0D00343F0250317
:107D5000037099F808300278C3F3801363F3C712F5
:107D60002223437005460270404604F02FFE94F82B
:107D7000E2300146284613F0010F10F8023B00F0F4
:107D80000482002900F0018243F040032B70062298
:107D9000F9F7C4FD05F108031846062209F10A01A6
:107DA0000B93F9F7BBFD042206F1100105F10E005B
:107DB000F9F7B4FD032206F1140105F11200F9F7F9
:107DC000ADFD01236B75B4F8F43040F2E242534349
:107DD0000C9306F099F8E268D4F804B1002A00F593
:107DE000DB63D8BF00F2BA63BBF1000F40F0D8816B
:107DF00085F816B085F817B09B460021084605F0B7
:107E00007FFE0021ABEB000B084605F082FEABEBDA
:107E1000000000F11E030E93B4F8F4302B83B4F885
:107E2000F6306B83B4F8F830AB8306F11701052206
:107E300005F11E00F9F772FDB27F95F8233062F369
:107E4000040385F8233094F8202162F3471385F862
:107E5000233005F0EDFE284605F04CFE05F096FEB9
:107E600020B140F2CB517B48F8F7F0FC4FF4AA72F6
:107E7000D4F808113046F9F78EFE002329463084E5
:107E8000FB723B7311F8023BF880C3F380134FF091
:107E9000060BBB7687F804B05A4607F11B00F9F7CA
:107EA0003DFD07F10E030D9307F11403BAF1000F26
:107EB00000F08681B8F1FF0F00F082810D9A0F93D8
:107EC00007F10D01404604F06BFF7A7B0F9B0B9985
:107ED00002327A7318465A46F9F720FDB4F8F430A6
:107EE000A7F82130B4F8F630A7F82330B4F8F8300A
:107EF000A7F8253095F82330C3F3421387F82730CD
:107F0000308CFBF7BBFFFBF7A3FE0320FAF7A0FEC4
:107F1000054620B940F211614E48F8F797FC338CC2
:107F2000EB800B232B7199F8083013F020030ED04F
:107F3000727C337CF17C43EA0223B27C42EA012268
:107F4000717F534041F04001F38371770123EB725D
:107F5000FBF77EFE2723D4F884713360D4F8FC301D
:107F6000F360002540F23B63272F77604FF0060255
:107F7000B560294600932846374BDFF8E8A038BFA4
:107F80002727FAF7EBFC40F23C61FBF7B5FF2B46E5
:107F90000422294600952846FAF7E0FC0C9BA3FB37
:107FA0000A89A36896F820400696A3EB070B40F2D7
:107FB00053630893294B0793294B0593F368039563
:107FC0001F44404620A3D3E9002349460497F8F70D
:107FD000A7F9104619464FF47A720023F8F7A0F972
:107FE00019A3D3E90023029049464046F8F798F9CF
:107FF0000E99019014A3D3E90023A1FB0A01F8F71D
:108000008FF9073420F07F40E4B200905B462246AF
:1080100029462846FAF704FC30F002033FF417AB78
:1080200040F25561FFF762BBB9F1000F7FF43FAE3C
:10803000404604F041FD00283FF41BAE37E600BF88
:1080400000CA9A3B000000008D49FD1A070000009D
:108050008D49FD1AAC050100F93E0000B13E00005B
:10806000795C000000CA9A3BB8F1FF0F70D094F819
:10807000E300A0EB080EDEF1000040EB0E0000284C
:108080007FF436AE99F8080010F00F0002D00628F1
:1080900040F0C28094F8E1301F0740F1A780D4F887
:1080A0000021002A40F0A280BAF1000F14BF41461F
:1080B000FF212846FBF79CFE00287FF4DAAD05F08F
:1080C0009DFD0378032262F30303037099F80830DF
:1080D0000278C3F3801363F3C7120C234370054681
:1080E0000270404604F072FC94F8E23001462846E3
:1080F00013F0010F10F8023B6FD000296DD043F050
:1081000040032B700622F9F709FC062209F10A0147
:1081100005F10800F9F702FC94F8E03043F002039F
:1081200084F8E03096200223637505F009FE0020F4
:1081300005F068FD284605F0DDFC05F0D3FE05F0EE
:1081400025FD00283FF483AA4FF4D361FFF7CEBA90
:1081500099F80820C3F38013C2F3801293428ED1A2
:10816000062209F10A01CC48F9F7C3FBB0FA80F006
:10817000400984E701288AD1002342463146FBF7B3
:10818000EBFD00283FF47EAFB8E594F8E120C34949
:10819000D20962F386132B700622F9E50C9A9344F8
:1081A000BBF1000FFADB9B45F8D3ABEB030340F2C6
:1081B000E242B3FBF2F3EB826B7D01336B751CE69D
:1081C000062200211846F9F7D5FB2B780B990D985C
:1081D000C3F3C0137B7306227EE694F8E120AF4917
:1081E000D20962F386132B7006228CE7A0B999F8A6
:1081F0000930002B3FF43DADD4F80031002B7FF463
:1082000038ADBAF1000F9DF8482014BF4146FF2158
:108210002846FBF7EDFD2CE501280ED099F8083033
:1082200003F00B02022AE2D003F00F03072B0DD15B
:1082300094F8E1305807DAD11BE512AB42463146DB
:108240000020FBF789FD0028D1D1E7E7042B7FF45C
:1082500010AD94F8E03099077FF50BAD05F0CEFC3A
:1082600099F808300278C3F38013B3EBD21F7FF480
:1082700000AD062209F10A010830F9F73AFB00289F
:10828000B5D0F6E494F8183194F84121013384F81C
:1082900018310026D4F83C318DF8476053F822801D
:1082A000012388F80430002F00F0A782D4F814517D
:1082B00098F8081095F8F830C1F3800103F0010236
:1082C000914200F08D8182F0010262F3000385F893
:1082D000F830237D032B02BF95F8503043F00103A3
:1082E00085F8503095F8F8301A0600F17481D5F809
:1082F0003C6195F85111301D00EB010A9AF801908C
:10830000B9F1000F00F091809B060BD5D5F82AB18A
:10831000D5F82EC11BF101024CF10003C5F82A214A
:10832000C5F82E31435C03F00303032B7DD19AF88B
:108330000330023B162B78D8DFE813F017005B0000
:10834000B600770077007700770077007900840027
:108350007700BD007700770077007700770077001F
:10836000C7007700DF00E60011010323637505F005
:10837000EFFB05F00BFC20B140F2DA614848F8F75A
:1083800065FA9AF80410D4F81401132908BF1621CD
:10839000FBF7B2FC0125D4F8140190F8513199444F
:1083A00090F850315FFA89F94B4580F851911ED110
:1083B000D0F83C31D0F8401100228B4280F8502197
:1083C00080F8512140F0D2808EB1D0F84411D3F81A
:1083D00000E0C0F83CE18B4206BFC0F84021C0F885
:1083E0004421C0F840E12F493046F9F7B6FB00269A
:1083F000C5E008220AF10E0105F19400F9F78EFAA2
:10840000D4F8140104220AF1160100F58970F9F775
:1084100085FAD4F8143193F8F82042F0080283F872
:10842000F820B3F84220A3F844200025B3E795F8DC
:10843000F83043F0480385F8F830B5F84230A5F835
:108440004430F2E794F814A05FFA8AFABAF1040F04
:108450002AD1337943F00303337117237371032354
:10846000F371082205F17A010430F9F757FA95F80B
:108470008230337495F88330737406F11201082248
:10848000606806F073FD06F11A015246606806F056
:108490006DFD0026C9E700BF1E0300201803002061
:1084A000AC0501009003002095F8F83043F0080374
:1084B00085F8F830B9E795F8F83003F0FB036FF36F
:1084C000C30385F8F8300023B9E795F8E82095F85C
:1084D000E9309A42A9D095F8EA3003F00302012A64
:1084E000A3D195F8F82042F0080285F8F82002227E
:1084F00062F3010385F8EA3097E795F8F630022237
:1085000062F3010385F8F630237D032B8DD101231F
:108510008DF848308DF849308DF84B300222042315
:108520008DF84A208DF84C308DF84D308DF84E3056
:108530008DF84F3095F8383095F8F620C3F3C20324
:1085400043EA920303F0070314AA134495F8392071
:1085500013F8083C63F3020285F8392065E795F8C3
:10856000783095F83920C3F38203F3E7D0F8482137
:1085700093421B6808BFC0F84831C0F83C317DB356
:10858000D4F81401FAF722FF0023C4F8143105F0DF
:108590009DFC18B905F08EFC05F092FCD4F814315E
:1085A000002B3FF454A81EB13146188CFAF794FE04
:1085B0009DF84730002B3FF44AA8D4F81431188CAA
:1085C000FBF75CFCD4F814311B8CA8F80630FBF7E1
:1085D0003FFBFFF73CB86FF3C71385F8F830002670
:1085E000D4F8143198F8082093F8F830C2F3C00298
:1085F000C3F340039A4240F0D0800320FAF728FBEF
:10860000002800F0CA8094F8823193B3D4F84C313A
:10861000D4F85021934205D194F8802194F8811127
:10862000914226D0D4F85021934200F0B68094F8BD
:10863000803194F881219A4200F0AF8094F8803123
:1086400033B9D4F81431B4F87E211B8C9A4210D07F
:1086500094F88031002B00F0A08094F88031D4F899
:10866000141104EB4303B3F878210B8C9A4240F0C9
:10867000948098F80950002D00F09880D4F81431B7
:1086800093F8F85015F0100508D005F0D1FC20B98A
:1086900040F66551A048F8F7D9F80125D4F814310F
:1086A00093F8F830D9062CD4D4F8140198F808308F
:1086B00090F8F82012F0040F39D1002213F00303D0
:1086C000A0F84820A0F84C2004D0022B5ED801234B
:1086D0008DF84730D4F8143193F8F82082F0020274
:1086E00083F8F820002D58D0D3F80991D3F80DA1C4
:1086F00019F101004AF10001C3F80901C3F80D1195
:108700004BE005F0B3FC0028CED10323637505F0E0
:108710001FFA05F03BFA20B140F675517E48F8F794
:1087200095F83D21D4F81401FBF7E6FA28E703F0A9
:1087300003010329E9D190F91DE098F80B10BEF16F
:10874000000F02F0400215DB22B90229B5D0112931
:10875000DBD809E08A1ED2B2092AF8D840F2052EE9
:108760002EFA02F2D207A8D46C4A22FA01F1CA0703
:10877000CBD5A2E72AB902299FD01129C5D8684ACA
:10878000F3E78A1E012A98D90B29F5E70DF1470175
:108790004046FDF7C9FD00289CD0D4F814210023E1
:1087A00084F819311D46A2F840303DE0D4F8142178
:1087B00092F8F83013F0140F8CD0D08CB2F84A1025
:1087C000831D9942C4BF8B1F1B1AB2F84600CCBF51
:1087D0009BB20B4698421EBFA2F846300023A2F877
:1087E0004C30B2F84C30002B7FF474AFB2F8463006
:1087F000A2F84830A2F84C106CE794F8193113B97C
:10880000022384F8193194F81931D4F81421013B6A
:10881000DBB284F81931B2F84060B3FA83F56D0920
:1088200086BBD38FA2F84030D4F8140112A990F877
:10883000F890FDF735FB637D032B4FEAD91910D073
:1088400015BB37B198F80830D80602D4129B5B7874
:10885000D3B1D4F8143193F8B330002B0CBF0223FA
:108860000323032B63752DD1237D042B0ED1D4F864
:10887000143193F8F82069F3C71283F8F82005F053
:1088800067F984E60026CFE70323EAE705F0D0F98D
:108890001299D4F814010B7890F8F82062F3C3030E
:1088A000C2F3400262F382030B70FAF725FE05F073
:1088B0006DF900283FF46BAE40F65D611648F7F79E
:1088C000C5FF64E6962005F03BFAD4F8143193F81E
:1088D0003A0000F0070005F095F905F003FBD7E733
:1088E00040F62471FEF702BF227D042A00F21382B3
:1088F000DFE812F0050205005A00AB00AB00032BC5
:1089000010D194F8283059070CD0FAF747FE05F03B
:1089100019F9FEF768BE00BFAC0501006020020037
:108920004020020005F0CEF9637D032B6FD194F84F
:10893000285015F040056AD1012212A9606806F09E
:1089400015FB9DF84810A4480A23B1FBF3F203FB82
:1089500012120132D2B2D6B2A6FB0001E8238DF882
:10896000482003FB06119AA3D3E90023F7F7D8FCAC
:1089700040F65F730693994B0593049583B2039574
:10898000029501950095052229462846F9F798FF9A
:1089900030F002033BD0E37C052B38D040F6637106
:1089A0008F48F7F753FF32E0032B24D1962005F0D0
:1089B000C7F9002319461A46184605F02FF994F80E
:1089C0004121D4F83C3153F82200083005F08CF8EE
:1089D00005F03CF904F06AFA38B112A804F00AF87C
:1089E00001469DF8480005F04BFB0123637505F037
:1089F000A3F8FEF7F8BD05F065F9637D052B06D1F8
:108A000000230093042219461846F9F7A7FF002512
:108A100025756575A57405F007FA724B2A46294637
:108A20002846F9F74BF920B141F2F9116C48F7F7F4
:108A30000DFF2068436800215B68984701221146BA
:108A40000020F9F713F9FEF702BED4F8140100284C
:108A5000DDD090F8B31081B1237D032B03D090F8C3
:108A60005030DA0709D5FBF747F9D4F81401FAF7C3
:108A7000ADFC0023C4F81431C9E7B0F82AB094F86B
:108A800018710BF10106B6B2002F00F08480237D2F
:108A9000032B73D105F01AFA814605F01DFAD4F8BC
:108AA000147197F83A3003F00703022BA9EB000981
:108AB000386E52D0042B0CBF4FF4BC784FF028080E
:108AC00000F13003434499450B93DFF81CA140A308
:108AD000D3E9002344D8A0FB0A01F7F721FC0B9B44
:108AE00085B2A3EB09003AA3D3E90023A0FB0A0156
:108AF000F7F716FC00233B66BB66D7F83C311FFA3C
:108B000080F8ABB35B7913B997F851310BB10023FF
:108B10007B85D4F8143100229A87D4F81401B0F878
:108B20004030C3B19E4280F0B8809B1B9BB20022B4
:108B3000062BA0F84030428540F2B180237D032B04
:108B400009D1BBF1000F40F0AA80C76E7B0817F077
:108B500001074BD1C36600274BE04FF01808AFE781
:108B6000A9FB0A01F7F7DCFB85B208F13000BAE790
:108B700097F85030DB07CCD5FB8CC9E749B190F8AA
:108B8000503043F0010380F850304FF00008454664
:108B9000BFE78846FBE7858F85B1AE4204D2AD1BA7
:108BA00085873D46A846B8E73E21FBF7A5F8D4F8EF
:108BB0001401FAF70BFCC4F8147128E7B0F84080F0
:108BC000B8F1000FEED1C38FA0F840304546A4E7BE
:108BD0008D49FD1A070000000010A5D42D3F0000AC
:108BE000AC0501001445002000CA9A3B43F0004345
:108BF000C366B0F8443023B19E4252D29B1BA0F80A
:108C00004430B0F84C3023B19E424CD29B1BA0F8AC
:108C10004C30D4F81421B2F8483092F8741023B1D3
:108C20009E4258D29E1BA2F8486092F875308B4243
:108C300006D092F87630013B012B9CBF0023538570
:108C400017B9538D5B4558D0538D01339BB235B95D
:108C5000B8F1000F03D113B9002F3FF4D8AE92F84A
:108C60002020039307320021D6B22E4A05922B46CC
:108C70000696049702910191CDF80080324608468D
:108C8000F9F71EFE30F002033FF4C1AEE37C9E42D2
:108C90003FF4BDAE41F2D00182E60821E3E60127B0
:108CA000A7E72221DFE60023A0F84C300220F9F7E5
:108CB000CFFF814620B941F278011B48F7F7C6FD86
:108CC000D4F814311B8CA9F806300A2389F8043033
:108CD000FAF7BEFF9DE70023A2F84830B2F844300F
:108CE000002BA2D192F875308B42A2D1072382F8D3
:108CF00076304B1E82F8753097E73B46A7E7043B7A
:108D0000012B04D941F2EF010748F7F79FFD00233B
:108D10006375FEF79CBC41F2F60141E641F2521147
:108D2000FEF7E4BC4D3F0000AC0501002DE9F04129
:108D30003D4E0A9C9DF81CC0BDF82C50BDF820800B
:108D40009DF818E030604FF4AA7000FB034086F8ED
:108D50002011C6F8084161190CF10104E7B27260F4
:108D600008F103040EF103022A2CD2B298BF02EBE1
:108D70004204A6F8348188BF08F10E0886F8542111
:108D80008CBF28F0030802EB84020EF1040E0CF1F4
:108D9000020C5FFA8EFE8CBF18FB02F292005FFAA3
:108DA0008CFCA6F8362186F874C1C6F83C014FEA5F
:108DB000CC0C00EB8E00B6F83641C6F86C0160446E
:108DC0003422C6F870016044A6F83821C6F82C0198
:108DD000B4FBF2F220440EEB0304C6F8440100EBAE
:108DE000C400BDF82440C6F858010A3424F0030436
:108DF0004830A4B2A6F8684107FB0404641A86F858
:108E0000103186F840E186F83A21C6F8600103D0B7
:108E10002C442046BDE8F081012386F88231F9F721
:108E2000EDFF04F087FDF4E734020020014B1868E1
:108E3000704700BF3402002038B503210520FAF73F
:108E4000B7F804210620FAF7B3F8224C002594F86D
:108E50001021ABB29A4205F1010534D894F82830BC
:108E60006FF3C71384F8283094F8E030002060F3E3
:108E7000000384F8E0303422B4F83631B3FBF2F367
:108E800084F83A3194F8403184F84101013B84F888
:108E9000750184F8780184F8543194F88031C4F86D
:108EA000CC00C4F80001A4F8382184F8420184F809
:108EB000760184F8770184F8813104F02FFBBDE856
:108EC0003840F9F79BBFA81DFF21C0B2FAF770F830
:108ED000BDE700BF34020020004870475F02002059
:108EE00000487047AF020020024B93F82800C009E9
:108EF000704700BF34020020044B93F92820002A59
:108F0000BABF93F82900800900207047340200207E
:108F1000094A92F8E03092F8E100D2F80021C0F35B
:108F2000C000002A03F0010303FA00F314BF042079
:108F300000201843704700BF34020020054B93F80F
:108F4000E00010F001001CBF93F8E100C0F3011035
:108F5000704700BF340200202DE9F04FDFF8F481A4
:108F600085B0D8F80051019383468A46914646461B
:108F7000002D40F0F48108F5A470F8F7D4FD074601
:108F800050B108F58670F8F7CEFD044630B908F503
:108F9000A4713846F8F7E1FD0720C8E198F8E13000
:108FA0006BF38613062288F8E130514608F1EA0097
:108FB000F8F7B4FCBDF80430A8F8F6302946BDF83F
:108FC0003830A8F8F8302846A8F8F49004F098FD56
:108FD0005F4900F252405CA3D3E90023A0FB0101EA
:108FE000F7F79EF94FF6FF7320F07F40C8F8FC00BA
:108FF000238403F59443C4F8A43003230193019B15
:10900000013BDBB2042103A8019302F0CDFFDDF8A0
:109010000CC04FF0000A4FEADC711F23D1464FF01D
:10902000010B5246D046013BDBB2FF2B06D1BAF111
:10903000000F00F09580CDF80CC091E02CFA03F5FC
:1090400005F001058D4224D10BF1010E072B5FFACB
:109050008EFE68D8002900F084810132BEF1060F2F
:10906000D2B2404649460AD8BEF1060F4BD01C2B5F
:1090700049D819B11C2B46D0012944D12DB3012563
:109080009D40072B2CEA050C01D8013AD2B20025ED
:1090900027E009F101010E2BC9B200F2698108F144
:1090A0000100072BC0B200F26481002D40F07581F1
:1090B0004FF0010E052BD7D83AB1052BD4D0012A99
:1090C00038D9042BD0D0022ACED1072B4FF001057E
:1090D00005FA03F598BF013245EA0C0C98BFD2B2ED
:1090E0000125894503BF0131C9B24FF0010E494640
:1090F00018BFDE460E2B04D8804506BF0130C0B233
:1091000040464FF0010A182916D9BAF1000F01D0D4
:10911000CDF80CC0012203991344EDB99A40013AED
:109120000A4303921CE0BEF1060F00F23181404673
:10913000494699E70122C8E70B28E6D88946F34655
:10914000294680466FE700BF8D49FD1A07000000E1
:1091500000CA9A3B340200209A4053420B400393CA
:10916000039B83F00E4383F4090304A883F43E4376
:1091700083F0D60340F8083D0421F8F77FFE01286C
:1091800040F2DD80039B9AB2B2EB134F00F0D28025
:10919000042203A904F110000393F8F7BFFB032195
:1091A00004F1140002F000FF05227E4904F11700CB
:1091B000F8F7B4FB96F81F21637F62F305036FF3A2
:1091C0008613637706220023A277E377B6F822118D
:1091D000B6F8F4E0B6F8F600A1851B21E1852186FA
:1091E000B6F8241161864FF4A471B6F82651A18611
:1091F000E18694F83810638465F30201012565F374
:10920000C50101F0BF0163F3C71184F8381094F869
:109210003910238565F3020184F83910B6F828C1A6
:109220006385C9B26CF3C50184F8391094F83A101B
:10923000A28765F3020184F83A10617FA4F824E064
:1092400063F3C711E084617794F8501001F0DF01F7
:1092500063F3000184F8501040F2E24202FB0EF288
:10926000B6F8F810A4F84030551E42F2107606FB0E
:109270000151A4F84430B1FBF2F14B4BE1874B496B
:1092800013441144B3FBF2F3B1FBF2F19AB2A4F828
:109290004210811D8A42A4F84A205ADC94F8A83072
:1092A000A4F84620002503F0FE0365F3410384F88B
:1092B000A83094F8C230A4F84C5065F3041384F835
:1092C000C23094F8F830A4F8485003F0800365F3F6
:1092D000C71384F8F83084F8745084F8755084F813
:1092E000B05084F8B15084F8B350C4F8B47084F826
:1092F000C05084F8C15084F8E85084F8E95084F8EC
:10930000F45084F8F550C4F83C51C4F84051C4F806
:109310004451C4F84851C4F84C5184F8505184F871
:109320005151FBF753F9224B2846C3F8004105B0D1
:10933000BDE8F08FDAB2B2EB136F7FF429AF019B77
:10934000002B7FF45CAE41F2E7611A48F7F77EFA32
:1093500055E6C0F57F43FA331A4492B29EE70C20DB
:10936000E5E7BEF1060F404649463FF6AEAEA1E640
:109370004046002D3FF49CAE1C2BAE463FF6C3AEDC
:1093800078E6012199402CEA010C404649467EE6E8
:109390000029F6D14046494697E60132D2B2AE46A0
:1093A00062E600BF4E0300207FC3C901FF5962027D
:1093B00034020020AC0501002DE9F0410C46904636
:1093C0001D46BDF81860BDF81C70F9F7DBFD30B321
:1093D000002C4AD190F8C230D90607D490F850300A
:1093E0009A0641D5D0F8A4309B073DD490F91D30A2
:1093F000002B17DA1A20BDE8F0818B420FD090F8CD
:10940000C23003F00702032A09D164F30203DBB27E
:1094100043F0080380F8C38080F8C23021E00C20BC
:10942000BDE8F08190F8743090F875209A42F6D13A
:1094300090F87830A0F87A500124002164F30103F9
:1094400061F38203224480F88840C0F88410A0F8B9
:109450007C60A0F87E7080F8783080F8764080F8E4
:1094600074200020BDE8F0810124013C14F0FF04C9
:1094700090F8C03090F8C110BFD19942CFD190F888
:10948000C23080F8C34064F30203DBB243F0080348
:109490000131A0F8C450A0F8C660A0F8C87080F8E8
:1094A000C23080F8C010DCE72DE9F0411E4C0146C7
:1094B0000522054604F58D70F8F730FA04F58D7035
:1094C0000521F8F7DBFC84F81F0194F81041013CFA
:1094D000E4B201274FF00208FF2C02D10020BDE8C2
:1094E000F0812046F9F74EFD0646B8B190F91D30DF
:1094F000002B13DB90F8742090F875309A4210D14D
:10950000052229467930F8F709FA96F8743086F87A
:109510007870013386F8768086F87430013CE4B2C6
:10952000DAE70120BDE8F08134020020F8B50D46ED
:10953000F9F728FD044660B1002700F117062777E8
:10954000052231462846F8F7E9F9207F0028F6D1B0
:10955000F8BD0120F8BD70B50D461646F9F712FDAD
:10956000044608B9012070BD15B390F8F80010F05A
:10957000400010D194F8742094F875309342F1D1E2
:109580000133032284F8795084F8780084F8743029
:1095900084F8762070BD94F8B12094F8B0309342EE
:1095A000E0D1013384F8B25084F8B030002070BDAF
:1095B000102231468430F8F7B1F994F8742094F809
:1095C00075309342CED10322013384F8795084F868
:1095D000785084F8762084F87430E7E708B5F9F716
:1095E000D1FC68B190F8742090F87530934207D19F
:1095F0000133042280F8743080F87620002008BD02
:10960000012008BD08B5F9F7BDFC68B190F87420D9
:1096100090F87530934207D10133052280F87430F9
:1096200080F87620002008BD012008BD10B50C464A
:10963000F9F7A8FC60B190F8B12090F8B0309342EF
:1096400006D1013380F8B24080F8B030002010BD60
:10965000012010BD10B51446F9F794FC10B100209C
:10966000207010BD012010BD10B50C46F9F78AFC22
:1096700060B1838CB0F84A205A437D2353430020C5
:109680004FF47A7293FBF2F3238010BD012010BDDA
:1096900010B50C46F9F776FC70B1828C40F2E243CB
:1096A000534342F2107101FB0434013C94FBF3F488
:1096B000A0F84A40002010BD012010BD70B50E4634
:1096C0001546F9F75FFCD0B190F8742090F875302A
:1096D0009A4214D190F8E82090F8E93093420ED1E4
:1096E00090F8EA40A0F8EE6001336FF3010480F8CF
:1096F000E83080F8EA40A0F8F250002070BD012068
:1097000070BD0000034BB3F822210280B3F824316E
:109710000B80704734020020034BA3F82201A3F80A
:1097200024110020704700BF3402002010B51B2414
:1097300004804FF4296008801480188010BD38B56B
:109740000D461446F9F71EFC58B190F83830C3F3B3
:10975000C2032B7090F83A30C3F302032370002049
:1097600038BD012038BD0000034BA3F82601A3F843
:1097700028110020704700BF340200202DE9F84373
:10978000894690461F46F9F7FDFB20B390F87420F8
:1097900090F875309A421ED190F8F43090F8F55058
:1097A0009D4218D190F8F64090F8F76004F0FC0460
:1097B00069F3840446F0020168F300012246013592
:1097C00080F8F71067F3471280F8F45080F8F6201D
:1097D0000020BDE8F8830120BDE8F8832DE9F341BE
:1097E000054608461849D1F84C31D1F8502193422A
:1097F0000F461FD0D3F8048001F2771198F80020AB
:10980000F9F776FB0446E0B902AE97F8773106F82F
:10981000033D97F8782131460DF10600F9F768FB12
:1098200034B928B9C5F80080204602B0BDE8F081FF
:109830000446EEE791F8782101F27711F9F758FB29
:10984000044600232B60EFE7340200202DE9F041AD
:10985000164D174E0446006805F5867728B9206036
:10986000FF20BDE8F041F9F77DBA0279D0F8008019
:109870000C2A15D80123934041F67E7213420AD177
:109880001B060DD5C288D5F808014FF4AA71F8F768
:109890007FF9394600E00749F8F75FF94046DDE710
:1098A00042F6A5413046F6F7D1FFF7E73402002033
:1098B000AC05010064030020914210B5144B19D18E
:1098C000D3F85021D3F84C41944211D1002914BF50
:1098D0000A460322013AD2B203EB420483F8812103
:1098E00093F88021A4F87A0191420FD083F8811176
:1098F000012010BD29B9B3F87E31181A18BF012014
:1099000010BD03EB4103B3F87831F6E7002010BD3A
:109910003402002030B4144B93F882210D4602B378
:1099200093F88021D1B293F8812135B14FF6FF73BE
:10993000984216D030BCFFF7BFBFD3F84C01D3F824
:109940005041A0420DD191420BD0D3F8504183F841
:109950008111A04205D093F88001814208BF83F8AD
:109960008121002030BC7047340200200148F8F704
:10997000DAB800BF980300200149F8F7EEB800BF3D
:10998000980300202DE9F0412E4C94F8765194F87C
:109990007431013588B0EDB280460F46AB4208BF46
:1099A0000025F9F7EFFA0646002848D094F87531FB
:1099B0009D4244D0B4F868317A79073B9A4204D981
:1099C00042F62A512048F6F741FF94F87621D4F860
:1099D0006C3103EBC20123F832804F6084F876517A
:1099E00096F91D30002B03DB002008B0BDE8F081A4
:1099F000738D002BF8D096F8503013F00204F3D199
:109A000096F8202043F0020386F850300F4B059360
:109A1000073201230393069623460494029401948B
:109A20000094D2B203212046F8F74AFF30F0020337
:109A3000DAD042F63D510448F6F708FFD4E701209A
:109A4000D3E700BF34020020AC050100412D000027
:109A50002DE9F8430746884616469946F9F792FAE3
:109A6000054610B90120BDE8F88390F8742090F8FD
:109A700075309A42F6D1FFF779FF04460028F1D0FD
:109A80001022494605F18400F7F748FF95F8F830B1
:109A900013F0300324D1237943F0030323711723F8
:109AA000082263710323E3714146A018F7F736FFDC
:109AB0003378237473786374082104F1120002F080
:109AC00073FA042104F11A0002F06EFA21463846B6
:109AD000FFF758FF0126D0B12046FFF74DFFC1E741
:109AE000302BF9D10822414605F17A00F7F716FF2D
:109AF000337885F88230737885F88330237943F0A2
:109B000003032371012363710A23E371DEE7032357
:109B100085F8763095F8743085F87860013385F8EB
:109B20007430BDE8F88300002DE9F04FDFF884B30E
:109B30008FB0994602230D939BF928308DF82F2082
:109B4000002B824688465D4601DA0C209EE19BF898
:109B50007A202B23272717FB02371BF8073003F047
:109B60000F03012B00F24881DBF8CC60002EECD112
:109B70000BF5A470F7F7D7FF0A9058B10BF5867074
:109B8000F7F7D1FF0A9A044630B90BF5A4711046D5
:109B9000F7F7E3FF072079E14FF6FF73038403F53E
:109BA0009443C0F8A430437FC67766F386134377A7
:109BB000BBF8223183851B23C3850386BBF8243180
:109BC00043864FF4A4738386C386BBF8261190F8AE
:109BD0003830468461F30203012161F3C50366F363
:109BE000861366F3C71380F8383090F8393006854D
:109BF00061F3020380F839304685BBF82801E66539
:109C0000DBB260F3C50384F8393094F83A30266645
:109C100061F3020384F83A30637F43F08003637793
:109C20000623A38794F8503066F3451366F30003C8
:109C300066F3410384F85030266794F8A830A4F8FE
:109C4000406066F3000366F3410384F8A83094F89B
:109C5000C230A4F8446066F3041384F8C23094F868
:109C6000F830A4F84C6066F3000366F3410366F332
:109C7000820366F3C30366F3041366F3451366F3C6
:109C8000861366F3C713A4F8486084F8746084F8F8
:109C9000756084F8B06084F8B16084F8B360C4F88B
:109CA000B42084F8C06084F8C16084F8E86084F867
:109CB000E96084F8F46084F8F56084F8F830C4F85A
:109CC0003C61C4F84061C4F84461C4F84861C4F818
:109CD0004C6184F8506184F85161FAF777FCCBF855
:109CE000CC400EA895F8293010F8092D6AF302032C
:109CF00062F3C50369F3871385F829309DF8603056
:109D000085F82A30D5F88431EB612723AB61012136
:109D100000232B62F8F7B2F81BF8076006F00F0675
:109D2000012E6BD14FF42773584300F59C705C49AA
:109D300059A3D3E90023A0FB0101F6F7F1FAAF69BB
:109D4000EB6968629F4238BF1F46B8F1000F5DD1D2
:109D5000721E5342534195F82860DFF85C91DFF89A
:109D60005CB163F3861685F8286016F040060DF1A5
:109D7000340A53D0F8F7C2FE6B6ACDF820A01F4416
:109D800006460020CDF81C900690CDF814B004973C
:109D9000039002908DE88100334605220321F8F7F5
:109DA0003FFD022836D00D98C8B902230D933D4BD4
:109DB000059303224AF2FE330093CDF820A0CDF89C
:109DC0001C90069004900390029001903346114637
:109DD000F8F726FD022846D00D98002847D0002C21
:109DE0003FF4B3AED4F8B4002F49F7F7B6FE2F49CD
:109DF0002046F7F7B2FEA8E6002472E7022E0CBF59
:109E00004FF4297340F2FC53584390E70023A2E734
:109E1000F8F7B4FE0D9B022BFAD0C4E7F8F76EFEFC
:109E2000CDF820A0CDF81C900696CDF814B06B6A42
:109E30000A901F4803961FFA88F81F44A8FB0001E8
:109E4000912303FB081114A3D3E90023049702967E
:109E5000F6F766FA009601900A9B05220321304628
:109E6000B6E7F8F78BFE0D9B022BFAD0B4E795F816
:109E7000283043F0800385F8283095F8E03013F05F
:109E8000010403D1012003F06BF920460FB0BDE8B7
:109E9000F08F00BFAFF300808D49FD1A070000006E
:109EA00000CA9A3B8D4500007C030020400300203F
:109EB000002AE78434020020C12B0000AD440000DA
:109EC00070B503210520F9F773F80546E8B9104C81
:109ED00094F8282060F3C71284F8282094F8E02032
:109EE000D30701D403F03CF9D4F8CC605EB1002371
:109EF000C4F8CC300749D6F8B400F7F72EFE06496F
:109F00003046F7F72AFE284670BD0C25FBE700BF58
:109F1000340200207C0300204003002000000000E9
:109F20002DE9F047684C94F8E0508EB01F4615F0CC
:109F300001054FF002030E460B93114603D00C208F
:109F40000EB0BDE8F08794F8E13094F8E22060F3B9
:109F5000C303400860F302039DF8600060F3000251
:109F600084F8E2209DF8642084F8E32066F3C713A8
:109F7000062204F1E40084F8E130544EF7F7CEFCF9
:109F8000BDF858204FF09109A2FB060109FB021110
:109F90004BA3D3E90023F6F7C3F994F8E1309DF819
:109FA0005C20D4F88481C4F8F00062F30513BAB2DF
:109FB000A2FB066709FB027784F8E130272300F152
:109FC000090AC4F8D480C4F8D030C4F8D8503CA3EF
:109FD000D3E9002330463946F6F7A2F9A0F127036A
:109FE0009A4594BFC4F8DCA0C4F8DC30B8F1270F60
:109FF000814638BF4FF02708F8F780FDD4F80031CC
:10A000008246002B45D00C950C9831492CA3D3E9FE
:10A010000023A0FB0101F6F783F90BAB08932D4B4E
:10A0200007932D4B0593D4F8DC3020F07F40434458
:10A03000002582440493304621A3D3E90023394606
:10A0400006950395F6F76CF9104619464FF47A72A7
:10A050000023F6F765F98DE82002029053460622A8
:10A0600003212846F8F7DCFB022823D00B9D002DA6
:10A070007FF465AF94F8E03043F0010384F8E030FA
:10A0800094F92830002B02DB022003F069F82846FF
:10A0900056E7D4F8DC100D930DAA0CAB4144032015
:10A0A000F9F7B6FC0C9B002BAED0DDF834A0ABE783
:10A0B000F8F764FD0B9B022BFAD0D7E7AFF30080D3
:10A0C0008D49FD1A0700000034020020002AE784B1
:10A0D00000CA9A3BC12B0000F544000070B5042172
:10A0E0000620F8F765FF0546E8B9104C94F8E02023
:10A0F00060F3000284F8E02094F92820002A01DBB4
:10A1000003F02EF8D4F800615EB10023C4F80031EA
:10A110000749D6F8B400F7F720FD06493046F7F7AF
:10A120001CFD284670BD0C25FBE700BF3402002053
:10A130007C03002040030020034BD3F800310BB117
:10A14000FFF7CCBF0C2070473402002037B5404CDD
:10A1500002AA002342F8043DD4F8500104F5A67188
:10A16000F7F74AFD054620B942F602413948F6F7AD
:10A170006DFB39492846F7F7F0FC019B1A790C2A48
:10A1800007D80123934041F67E72134207D11A0685
:10A1900016D442F639412F48F6F758FB10E094F8F0
:10A1A000403194F85421013B9A4204DB42F62F419E
:10A1B0002848F6F74BFB94F85431013384F85431B6
:10A1C000019B1A79062A35D1DA7A3C2A11D01B7BF9
:10A1D00093BB94F8E030DB0704D442F650411D48AD
:10A1E000F6F734FB94F8E0306FF3000384F8E030C6
:10A1F00014E00023D4F8CC50C4F8CC3094F92830C3
:10A20000002B04DB42F64D411248F6F71FFB94F891
:10A2100028306FF3C71384F828307DB994F8E00034
:10A2200094F8283000F00100400050EAD31001D12A
:10A2300002F096FF03B030BD0025DFE7D5F8B4008B
:10A240000549F7F78AFC05492846F7F786FCE5E754
:10A2500034020020AC0501007C03002040030020F4
:10A2600038B50B4CD4F84021D4F8445122B1002029
:10A27000C4F84001F8F7C2FA2DB10023C4F8443104
:10A280000120F8F7BBFA0020BDE83840F7F764BDBD
:10A2900000B000400120F7F75FBD684620F00701DD
:10A2A0008D4601B5F7F7F4F903F028FBF7F7E2F96B
:10A2B000F7F798F8BDE80140854670477047000001
:10A2C000014B186805F071BB8424002010B5374B92
:10A2D00086B01860364804F065FE18B96FF01200B9
:10A2E00006B010BD436801211B689847314804F04F
:10A2F00059FE04460028F1D003F058F9F7F78CFC1A
:10A300002D4B08221A7003221A7202221A7600209C
:10A310002A4A187405922A4A04922A4A03922A4A1F
:10A3200002920D2201920093284A04231721F8F784
:10A330002DFA18B19D212648F6F788FA254804F031
:10A3400031FE0028CAD041F604230593224B049322
:10A350001B230393029307210623009322460191B6
:10A360001023FEF7E3FC0446E0B9012003F0D6F821
:10A37000224621460120F7F763F9224621460B20A9
:10A38000F7F75EF9224621461820F7F759F9012020
:10A39000F7F724F90B20F7F721F91820F7F71EF942
:10A3A00020469DE76FF00B009AE700BF8424002051
:10A3B000300501000C0501006424002085E2000046
:10A3C000F9E10000CDE10000F42100205C1E002036
:10A3D000E50501003B0501005804002008B50248CE
:10A3E000F7F732FB002008BD1C06010037B5838952
:10A3F000054623B3037D8BB1022B20D101A901F0C7
:10A40000B3F90446019808B1F7F750FB1CB9284688
:10A4100003F0F8FF0024204603B030BD00F096FBA7
:10A4200002460028F3D08368197813290AD801233B
:10A430008B4013F40C2F05D0F7F738FBE7E76FF0EC
:10A440001504E8E71046F7F727FBE0E713B501909E
:10A45000081E03DB022807DD032822D08A211648C4
:10A46000F6F7F4F900240DE001280EBF00214FF0AB
:10A47000FF310120F7F7FAFA044618B101460198B6
:10A4800001F028FA019B0021D888FFF743FA02A8BF
:10A49000002250F8043D1A60FFF7D8F9204602B0B8
:10A4A00010BD4FF0FF31F7F7E1FA0446014601987D
:10A4B00001F0B8F9E6E700BF30060100F7B5144D2A
:10A4C000144E0DF1020101A8FFF788F9044640B9C6
:10A4D000019BBBB1FFF73AFE0199304604F08EFFB5
:10A4E000EFE74FF0FF310120F7F7C0FA22460746A9
:10A4F000BDF8021001F024FD3846F7F7D7FA05F051
:10A5000015FADEE74FF0FF31284605F076FAD8E776
:10A510005847002070470020044B186828B159683C
:10A5200002681A60884208BF5A6070478C24002075
:10A5300010B5154886B0FFF7C9FE044600BB1348A6
:10A5400001F02AFD6FF0090303934FF4E072104B02
:10A550001049059404940294019400940E4805F067
:10A560003DFC6FF007030393059404940294019457
:10A5700000940A4B0A490B484FF4007205F02EFC78
:10A58000204606B010BD00BF584700203C460020C2
:10A59000BDA40000D0330020342C0020A9A5000069
:10A5A00090350020C42B00202DE9F74F6A4E374626
:10A5B0004FF0FF320221304605F074FE20B14FF417
:10A5C00098716648F6F742F9F36803F4F833B3F587
:10A5D000805F05D13269002393604FF000090AE0E3
:10A5E000336A03F4F833B3F5804FF6D10021706A73
:10A5F00004F028FF8146FA686FF31032FA603A6A75
:10A600006FF310323A62564A1568564ABFF35B8FB1
:10A6100052E8001F21F0010342E800300028F7D182
:10A62000BFF35B8FCA0748BF4F4A504C42BF00215F
:10A6300011605160002D06DC4FF0FF322260B9F14D
:10A64000000F21D16DE0DFF82CB1DFF82CA1DBF891
:10A650000020454BDAF800101B680193AA1A0A443F
:10A660002260002BEBD0184601F07EFC8046B9F149
:10A67000000F18D0022803D0032805D122681AB190
:10A6800000213B4805F0A0FE484601F06DFC216822
:10A690004B1C05464CD0344A1068032D53D8DFE8D4
:10A6A00005F047473443022808D0032804D0FC2192
:10A6B0002A48F6F7CBF803E0236893B3FFF72CFFA3
:10A6C00041460198FFF7C2FEDBF80030ED1ADAF8D8
:10A6D00000301D44244B25608146186858B101F0B4
:10A6E00043FC022803D0032805D123681BB10021B5
:10A6F0001F4805F069FEB9F1000F12D0B9F80C300F
:10A7000048462BB3F7F7C8F90BE00121216078B177
:10A710000021C9F80010516881B9C2F80490C2F84C
:10A72000009005F003F943E70028F1D10029EFD0AC
:10A7300048462946FFF78AFE8146DCE7C1F80090CB
:10A74000C2F80490EDE7B3210448F6F77FF8EFE78D
:10A7500003F058FEE5E700BF144600203006010074
:10A76000C42C0020CC2C00208C2400208824002025
:10A770003C460020C82C0020D02C0020C0F307232A
:10A780000870000C8870000A4B70C870704738B5AC
:10A7900008300D460221144603F062FE0570447035
:10A7A00038BD000038B505464FF0FF30F7F768F9BF
:10A7B000042204460F21FFF7EAFF042104F10800F8
:10A7C00003F04EFE01234370024B05701B8843804B
:10A7D000204638BD9424002070B504461546013249
:10A7E0000E460834D2B23E21FFF7D1FF01212046A8
:10A7F00003F036FE067029462046BDE8704003F09F
:10A800002FBE000038B504464FF0FF300D46F7F775
:10A8100037F9EA1C2060D2B20E21FFF7B8FF20689A
:10A820000321083003F01CFE01230370054B1B8835
:10A83000A0F80130206829460830BDE8384003F010
:10A840000FBE00BF942400200E4B70B51546D3E90F
:10A850000023002302F08002134304460E4610D06A
:10A86000042208212846FFF792FF042105F1080081
:10A8700003F0F6FDB4FA84F35B090470A0F80160FC
:10A88000C37070BD5046002070B504461846134B87
:10A890001646D3E90023002203F0005313430D466C
:10A8A0001BD00F4BD3E90023002302F0080213430F
:10A8B00013D00B220421FFF78FFF08220470A0F8A9
:10A8C0000160033024B9291DBDE87040F7F726B8B0
:10A8D0000021BDE87040F7F74DB870BD504600202C
:10A8E000584600202DE9F84F05461846464B1646B7
:10A8F000D3E9002340F201284FF0000902F4007A66
:10A9000003EA090302EA080213430C464FF0000B66
:10A9100077D0002D50D13D4A1368013313605AEAB5
:10A920000B0301F1030851D112220121FFF754FF5B
:10A930000570A0F801606378C370A37803710746BF
:10A94000062241460530F6F7E9FFE38AA7F80B3007
:10A95000238BA7F80D30638BA7F80F30237F7B7410
:10A96000BDE8F88F1E220A21FFF736FF1E2204469B
:10A970000021F6F7FFFF2570BDE8F88F637D03F037
:10A98000C003402B38D1062204F11001F6F7C6FFB0
:10A99000062204F1090107F11100F6F7BFFFE38A6F
:10A9A000A7F81730238BA7F81930638BA7F81B3053
:10A9B000237F7B77BDE8F88F5AEA0B03D2D11222AE
:10A9C0000121FFF709FF12220446D1E71E220A21C6
:10A9D000FFF702FF0570A0F801606378C370A378E9
:10A9E00003710746062241460530F6F797FFE37BE1
:10A9F00007F10B00002BC1D106220021F6F7BAFFA8
:10AA0000C6E7BDE8F88F00BF584600209824002014
:10AA10001FB5032807D8DFE800F0020A0C0E07492B
:10AA200001A8F6F74FFF002005B05DF804FB0449CC
:10AA3000F6E70449F4E70449F2E700BF83060100A2
:10AA40008A060100910601009B060100037807B504
:10AA500003F00F02072A15D142789AB18278910645
:10AA600010D0C278D2070DD5C3F38013011D062282
:10AA70000DF101008DF80030F6F750FF9DF8000051
:10AA8000FFF7C6FF03B05DF804FB0000F8B5224BEA
:10AA90004FF0FF321A60214B4FF0FF3641F6FF773F
:10AAA000C3E900671E4B00260027C3E900671D4B62
:10AAB0001F2600270C46C3E90067054638B1FEF79C
:10AAC000BBF901212046FFF79DFE00230370164BC2
:10AAD000164800241C60164B1C60164B2022214691
:10AAE0001C60F6F747FF144B1C609DB1BFF35B8FF2
:10AAF000124B53E8002F42F0010243E800210029E5
:10AB0000F7D1BFF35B8F0E4B21461868BDE8F840C4
:10AB100005F05ABCF8BD00BF9C2400205046002020
:10AB20002825002058460020C42C0020A42C0020FA
:10AB3000C82C0020D02C002098240020CC2C0020F1
:10AB4000302500200346006859687047F0B58189B8
:10AB500099B00025022904460D9502D8002019B0AD
:10AB6000F0BD8368B24E1A7858789B7842EA00228A
:10AB70008B423280F2D8032104F1080003F07FFCFD
:10AB80003388C3F309029B0A042B00F0228109D801
:10AB9000012B27D0032B3CD001210DA8FFF732FE5B
:10ABA00001235DE0082B00F0C8813F2BF4D1013A6E
:10ABB000092AF1D801A353F822F000BF81B50000A3
:10ABC000B1B50000DBB5000099AB000099AB000007
:10ABD00021B6000099AB0000F3B500002DB60000CF
:10ABE0009BB60000062A06D01D2AD5D1A368188876
:10ABF000FEF708FD04E0A36899781888FEF716FDB3
:10AC0000002814BF0C200020FFF7CCFD0D900D98FC
:10AC1000A5E7332A00F08A8024D8032A46D00DD82D
:10AC2000012AB9D1A068FFF78DFF824BC3E900016B
:10AC300001210DA8FFF7E6FD002311E02D2A46D0E3
:10AC4000312AA9D1A3687C4C1D7801210DA8FFF7FA
:10AC5000D9FD23681BB1794A1268002A4DD00C2314
:10AC60000370D4E7632A26D00AD8352A94D1724BD0
:10AC70001B68002B6BDC01210DA8FFF7C3FDEEE77D
:10AC80007B2A00F08F807C2A86D1A3681C88598893
:10AC9000A0B2FEF7FDFC054603210DA8FFF7B2FDAB
:10ACA000002D14BF0C23002303703FE30DA92046A1
:10ACB000FFF7ECFEABE7A068FFF744FF604BC3E98A
:10ACC000000101210DA8FFF79DFD05709FE7A36816
:10ACD00004210DA81D889F78FFF794FDAEB20446AD
:10ACE000C21C39463046FEF7B5FC002814BF0223CB
:10ACF00000232370A4F8015089E702701DB1012DD3
:10AD000010D01223ACE7002B81DB4E4B4E480021C4
:10AD100019604E4B20221960F6F72CFE23685B4227
:10AD2000236074E7002B3FF772AFEEE7A3680121C1
:10AD30000DA8B3F803401D88FFF764FD3E4B1A6869
:10AD4000002A8CD11A2DDCD964421C605FE73B4B92
:10AD50001B68E3B1A5683C4E2F7800231946BB421F
:10AD600009DB3A4A13680B441360394B0021186819
:10AD700005F02AFB4BE705EB8302B2F80140B2F87D
:10AD800003000F2C03D836F81420904204D9012177
:10AD90000DA8FFF737FDB4E7121A26F81420014476
:10ADA0000133DCE7A3681C880EA9A0B2FEF75CFCA7
:10ADB000052105460DA8FFF725FD002D14BF0C2326
:10ADC00000230370A0F80140BDF83830A0F803302C
:10ADD0001DE7013A082A3FF6DFAE01A353F822F03F
:10ADE00005AE000055AE000007AF000099AB0000B3
:10ADF00099AB000099AB000099AB000099AB000043
:10AE000023AF000009210DA8FFF7FCFC002303700D
:10AE10008370C3706FF00E034371052309228371A1
:10AE20004FF0FF3342700271C3710372EFE600BF4F
:10AE30009424002050460020C42C00209824002098
:10AE400028250020C82C0020A42C0020D02C002075
:10AE50003025002041210DA8FFF7D4FC0021044635
:10AE6000402200F8011BF6F785FDE3786278617FE8
:10AE700094F8210063F07F03E370A37963F03F034C
:10AE8000A371E37A63F01B03E372E37B43F02803CF
:10AE9000E373237C43F002032374E37D43F0040354
:10AEA000E375A37E63F00803A37642F02002FF233C
:10AEB000E3766270237794F8222084F8243094F8A3
:10AEC000283062F00F0241F07F0143F0040384F860
:10AED0002220617794F8232094F8251084F82830F4
:10AEE00094F8273040F0300041F0010162F0060292
:10AEF00063F07F0384F8210084F8251084F8232070
:10AF000084F8273083E609210DA8FFF77BFC002198
:10AF10000446082200F8011BF6F72CFD602363713C
:10AF200075E607210DA8FFF76DFC0146002301F827
:10AF3000013B1846F7F7E8FD69E6013A4D2A3FF66E
:10AF40002BAE01A353F822F081B000008BB00000BB
:10AF5000A3B0000099AB0000C7B000006DB10000C5
:10AF600089B600009DB10000A9B10000B5B1000094
:10AF7000D3B10000EBB100000BB2000035B200000D
:10AF8000D3B00000E9B00000FBB0000003B1000046
:10AF9000EFB2000095B20000CBB20000E5B20000B5
:10AFA0000BB1000031B100009DB20000B1B2000051
:10AFB000C1B2000047B1000037B5000045B5000040
:10AFC00055B5000009B3000033B3000041B30000E1
:10AFD00061B3000079B3000099AB000099AB0000A9
:10AFE0007DB400008BB4000093B40000A3B4000053
:10AFF000B5B40000D3B40000F1B4000007B5000000
:10B0000095B30000ADB3000003B4000021B400000C
:10B0100073B500007BB5000099AB000099AB000050
:10B0200099AB000099AB000099AB000099AB000010
:10B0300099AB000099AB000099AB000099AB000000
:10B0400099AB000099AB000099AB000099AB0000F0
:10B0500099AB000099AB000099AB000099AB0000E0
:10B0600099AB000099AB000099AB000099AB0000D0
:10B070001DB5000099AB000099AB000013B50000AE
:10B08000A068FFF75FFDB24BD0E504210DA8FFF7E4
:10B09000B9FB002303701B22837007234270C37027
:10B0A000B5E509210DA8FFF7ADFB002104460822F4
:10B0B00000F8011BF6F75EFCFF2363704923A370C1
:10B0C0000123E370A3E5A1680120F7F737FD0446EB
:10B0D000D8E002210DA8FFF795FB0023037004467A
:10B0E00001F012FD607092E501210DA8FFF78AFBC7
:10B0F000044601F00BFD207089E5A06801F0D4FD45
:10B10000E5E7A06801F022FDE1E7A06800230EAAB0
:10B1100000F1100102F0B8FA11210DA8FFF772FB3F
:10B12000002300F8013B10220EA9F6F7F7FB6EE5AD
:10B1300009210DA8FFF766FB002300F8013B082159
:10B1400000F032FF63E509210DA8FFF75BFB014624
:10B150000023024601F8013B6FF44000FFF70EFBAD
:10B1600040F2FF30511DFFF709FB50E5A0680021B8
:10B17000037902880A910991089107910691059136
:10B18000847B0494447B0394C41D029484790194C9
:10B1900040790090084600F02DFF98E7A368591CFD
:10B1A000187801F041F843E5A368591C187801F0BC
:10B1B00093F83DE5A368187801F0D4F8044601211E
:10B1C0000DA8FFF71FFB002C18BF0C2308BF00239E
:10B1D00046E5A4686379B4F80320B4F80110207838
:10B1E000A479009401F03CF9E8E7A268594B107883
:10B1F00040B1527832B100221A60574B1A6001F008
:10B200004FF9DBE74FF0FF32F8E7A468B4F81350CA
:10B2100063792279618820880495B4F811500395E8
:10B22000B4F80F500295257B01950634009401F087
:10B2300071F9E5E4FEF780FF064648BB4FF0FF31A9
:10B240000120F6F713FC454A0D90D2E90045002491
:10B2500005F0005554EA0502034604D03246314653
:10B260000220FFF73FFB0D9884894CB101210EA805
:10B27000FFF7C8FA002303700E98F6F717FCC6E430
:10B2800003F0C0F801210DA8FFF7BCFA0470BEE47A
:10B290000C24F7E7A068FEF707F98FE7A06800F134
:10B2A0000C0300F10A02811C0088FEF7D1FBA7E421
:10B2B000A26832F8024B0021A0B2FEF74CF9EAE492
:10B2C000A36800221C880621F6E7A36808210DA8C0
:10B2D0001D88FFF797FAAEB20446C11C3046FEF750
:10B2E00025F902E5A3681888FEF778F988E4A268D2
:10B2F0001189938810880191D2880092002211460A
:10B30000FEF75AF8C0B27FE4A268118914889388C6
:10B310000191D288009200220221A0B2FEF74CF8DF
:10B32000032105460DA8FFF76DFA0570A0F801404E
:10B330006DE4A3681C889A78002301930093EBE7DF
:10B34000A3681C889A885988A0B2FEF7B7F9A2E4CE
:10B35000584600209C240020A024002050460020B5
:10B3600005210DA8FFF74EFA0446C11C0130FEF777
:10B37000C9F9002323704AE4A36859881888FEF7A6
:10B38000CBF9044601210DA8FFF73CFA002C18BFA9
:10B390001E231BE709210DA8FFF734FA0446C31D3D
:10B3A000421DC11C0130FEF7C1F9E2E7A368052187
:10B3B0000DA81D88FFF726FAAEB20446021DC11C77
:10B3C0003046FEF7BCF9E278A4F80150002814BF1B
:10B3D0000C2300232370002A92FAA2F3B3FA83F31A
:10B3E000227908BF4FF0FF330133E370002A92FA4D
:10B3F000A2F3B3FA83F308BF4FF0FF330133237195
:10B4000005E4A3681A78D10744BF07215970920751
:10B4100044BF07229A7099785878FEF7A5F9B0E7EB
:10B42000A36899781888B3F80540CF0742BFDA7847
:10B4300042F00702DA708E0748BF1A79D97844BF04
:10B4400042F007021A711B7941EA030212F0F80F69
:10B4500002D01120FFF7D8BB4D0701D05A0702D107
:10B460001220FFF7D1BB14F003021CBF04F1FF341C
:10B4700004F00102FEF782F9FFF7C2BBA06800F1F9
:10B480001702C11D01F0A0FE21E6A06801F03EFFF9
:10B490001DE601210DA8FFF7B5F9044601F07AFE7B
:10B4A00029E602210DA8FFF7ADF9044601F070FE70
:10B4B00060705EE70722A1680EA8F6F72FFA072151
:10B4C0000DA8FFF79FF90446411C0EA801F0ACFF40
:10B4D00011E60722A1680EA8F6F720FA07210DA8A9
:10B4E000FFF790F90446411C0EA801F0BDFF02E6EB
:10B4F000A36801210DA81D78FFF784F904462846AA
:10B5000001F0CAFFF7E5A368188801F0D7FFFFF73D
:10B510008FBBA068C17901F0D9FFD8E503210DA840
:10B52000FFF770F90146002301F8023B0130F7F7FD
:10B5300021FBFFF76CBBA36800220121187801F002
:10B5400045F9C4E5A068012382784178007801F0CC
:10B55000D9F8BCE50EA801F061F903210DA8FFF7A9
:10B5600051F900230370BDF83830A0F80130FFF71F
:10B570004EBBA3689A785978E0E7A068C378E3E700
:10B580000D210DA8FFF73EF902224270C270012280
:10B5900082710D220023C2716322037083700371D4
:10B5A0004371037242728372C3720373FFF72FBB3E
:10B5B00041210DA8FFF726F900210446402200F89A
:10B5C000011BF6F7D7F9637863F058036370A3782B
:10B5D00043F00303A370FFF71ABB09210DA8FFF77F
:10B5E00011F9002100F8011B0822F6F7C3F9FFF753
:10B5F0000EBB5C4B0EAA03F1280615461868596865
:10B60000144603C40833B3422246F7D129210DA8BA
:10B61000FFF7F8F8002300F8013B2822294684E5CB
:10B62000A1680020F7F78AFAFFF702BB4FF08053BA
:10B63000D3F8A420013206D1D3F8A8304FF6FF7218
:10B640009BB2934220D04FF08055D5F8A030DB0755
:10B650001AD518210DA8FFF7D5F8002601230446B6
:10B6600043700670D5F8A400A11CFFF787F8D5F841
:10B67000A830A371C3F3072363F03F03E3711022E3
:10B68000314604F10800B0E702210DA8FFF7BAF82F
:10B69000002303704370FFF7BABA21210DA8FFF70A
:10B6A000B1F80346002203F8012B4FF08052044604
:10B6B000D2F8901001314BD0D2F89410013147D01C
:10B6C000D2F89810013143D0D2F89C1001313FD00C
:10B6D000D2F890001946FFF751F8611DD2F8940096
:10B6E000FFF74CF804F10901D2F89800FFF746F88B
:10B6F00004F10D01D2F89C00FFF740F84FF08052A2
:10B70000D2F88030013304F1110327D0D2F884102D
:10B71000013123D0D2F8881001311FD0D2F88C101B
:10B7200001311BD0D2F880001946FFF727F804F149
:10B730001501D2F88400FFF721F804F11901D2F8BD
:10B740008800FFF71BF804F11D01D2F88C000AE510
:10B75000102200211846F6F70DF9CFE7102200213C
:10B76000184642E7DB0601002DE9F84300230B6091
:10B770008389032B0646884603D86FF01500BDE881
:10B78000F88350F8083F04215F881D8802F077FE97
:10B79000B389BB42F1D3FEF7E9F84FEA1539044605
:10B7A000C5F30B05F0B91E4BD3E90023002302F0CB
:10B7B0000072134312D04FF0FF310120F6F756F913
:10B7C0000122C8F800001A21FEF7E1FFD8F80000B6
:10B7D0000121083002F044FE012303706FF03600AF
:10B7E000BDE8F8830379B9F1000F02D0B9F1020F77
:10B7F00013D1022262F3010323716771B1683A46E3
:10B80000E01DF6F78BF821462846FEF7BBF8002826
:10B81000E6D02046FEF7B0F8AFE70122EAE700BF26
:10B8200050460020037A03F00303013B012B70B55F
:10B8300004463CD801F10806C5880421304602F0D0
:10B840000FFE237A617A418003F00303022B0CBFC1
:10B8500045F4005345F480530380304602F000FE67
:10B86000627A04F10B01F6F759F8154B1A68002AB1
:10B8700024DD144C1449236809685B1A934204D3ED
:10B8800040F691311148F4F7E1FF23680F2D03F1E1
:10B890000103236004D940F696310C48F4F7D6FF33
:10B8A0000B4A32F81530013322F8153070BD40F6DE
:10B8B0009D310648BDE87040F4F7C8BF70BD00BFB9
:10B8C000C42C0020C82C0020D02C0020A50601008C
:10B8D000A42C00202DE9F04F0379C688012B87B0F6
:10B8E00004460D4600F1080700F06782023B0A2B70
:10B8F00000F25D82DFE813F00B00260126012A0129
:10B900005D017801BC01E101F9010E022902012368
:10B910008DF8113003238DF81230FF238DF813308A
:10B920008DF8153002238DF81630437A0344002138
:10B9300093F80B90037A8DF81010042258068DF8B6
:10B94000142005D504F10A034A46084601F04AFDD1
:10B95000BD4BD3E90023002203F00053134300F052
:10B96000AB80637A234493F80CA0B84BD3E900234F
:10B97000BAF1000F3DD102F002020023134300F0A0
:10B980009B80B34B1A68002A984654DBDFF8DCB280
:10B99000002604F10A03D8F8002096422CDBAD4EB5
:10B9A000DFF8B4B230680BEBC00019460622023053
:10B9B000F5F7B4FF3268237A0BEBC201C3F38013AF
:10B9C0004B70237A03F00F0101238B40D8F800104D
:10B9D0000BF832300F29D5BF0131013231603260AE
:10B9E0003268D8BFC8F80010102A24D10022326073
:10B9F00021E002F00B02C0E71846062259460393E5
:10BA0000F5F777FF039BF0B9217A1BF8010C0A4682
:10BA1000C1F38011814216D18F4810F8363002F000
:10BA20000F0223FA02F1C90746D4012101FA02F2FA
:10BA3000134300F83630237A627A03F00F03012BA8
:10BA400005D1002605E001360BF1080BA3E7961F90
:10BA5000F6B2224492F80A80C8F100084FFA88F83A
:10BA6000BAF1000F35D0012B04D04FF40B617B48A5
:10BA7000F4F7ECFE11220B212846FEF7ADFE012360
:10BA800003704370054601F083FB814505F1030017
:10BA900015D20246A91C484601F082F9AB78023360
:10BAA000AB7001236B72062207F1080105F10A0051
:10BAB000F5F734FF85F8108007B0BDE8F08F237AE2
:10BAC000C3F38013AB70062204F10A01F5F726FFD9
:10BAD000E7E706F10B02D2B202212846FEF77CFE10
:10BAE00001230370237A06AA03F00F0313440546CB
:10BAF00013F8083C4370637A234493F80B9001F0E9
:10BB000047FB814505F1030012D20246A91C4846B5
:10BB100001F046F9AB780233AB706E720A353246EB
:10BB200007F108012846F5F7F9FE05F80680C3E796
:10BB3000237AC3F38013AB70062204F10A01F5F7F0
:10BB4000EDFEEAE73846FEF781FFB5E73E4BD3E965
:10BB50000023002203F00053134300F10A0607D02C
:10BB60003A4BD3E90023002302F4802213430FD180
:10BB7000237A0622C3F3801331460DF111008DF8AC
:10BB80001030F5F7CBFE9DF81000FEF741FF93E76C
:10BB9000082213212846FEF71FFE00230370237A94
:10BBA000C3F380134370062231460230F5F7B6FE28
:10BBB00082E7C77A3FB900F1140300F10E01FF22BA
:10BBC000407B01F00FFC204BD3E90023002203F05F
:10BBD000005313433FF470AF2B46324604F10B0180
:10BBE0003846FEF77FFE67E7174BD3E900230023B3
:10BBF00002F0100213433FF45FAF042205212846F0
:10BC0000FEF7C5FD042105F1080002F029FC002320
:10BC10000370A0F80160237AC3700F2E04D940F698
:10BC2000D8110E48F4F712FE0D4A0E4932F81630BC
:10BC3000086803440B60002322F816300A4A136890
:10BC4000013B136038E700BF5046002058460020F3
:10BC50009C240020A0240020A4240020A50601008C
:10BC6000A42C0020D02C002098240020A624002002
:10BC7000AF4BD3E90023002203F0005313433FF4FA
:10BC80001BAFAC4BD3E90023002302F004021343A3
:10BC90003FF412AF092203212846FEF79DFDE37A07
:10BCA0000370A389A0F80160A0F80330E389A0F82D
:10BCB0000530238AA0F80730FEE69D4BD3E9002328
:10BCC000002203F4004313433FF4F6AE0322302175
:10BCD0002846FEF75CFD032105F1080002F0C0FBD9
:10BCE00000230370A0F80160E6E6934BD3E900233C
:10BCF000002302F4000213433FF4DEAE0222572178
:10BD00002846FEF744FD022105F1080002F0A8FBD9
:10BD10000680D1E6864BD3E90023002203F00053CE
:10BD200013433FF4C9AE834BD3E90023002302F44D
:10BD3000002213433FF4C0AE032214212846FEF72D
:10BD40004BFD0680E37A8370B6E6794BD3E9002396
:10BD5000002203F0005313433FF4AEAE754BD3E91A
:10BD60000023002302F4006213433FF4A5AE052232
:10BD70000C212846FEF730FDE37A0370A0F801603D
:10BD8000227B002A92FAA2F3B3FA83F308BF4FF0A2
:10BD9000FF330133C370627B92FAA2F3002AB3FA35
:10BDA00083F308BF4FF0FF330133037184E640F69D
:10BDB000AB216248F4F74AFD7EE6C37A033B122BBF
:10BDC00000F2B280DFE803F00AB0B02FA7B035B0C0
:10BDD000B03C5BB05FB0B0B0B0878700544BD3E9E4
:10BDE0000023002203F0005313433FF465AE514B90
:10BDF000D3E90023002302F0100213433FF45CAEAA
:10BE00000C2205212846FEF7E7FC0822054604F12E
:10BE10000C0120F8026BF5F781FD022204F11401F8
:10BE200005F10A00C2E60A4600203146FEF70CFD85
:10BE300042E60B46324639460020FEF725FD3BE63A
:10BE40003B4BD3E90023002302F4006213433FF489
:10BE500033AE08220C212846FEF799FC0821681809
:10BE600002F0FEFA00230370A0F80160237BC37088
:10BE7000B4F80D308380B4F80F30C3801CE60A4656
:10BE8000007B3146D2E72A4BD3E90023002203F09E
:10BE90000053134307D0274BD3E90023002302F0BC
:10BEA0002002134308D10023019300931A22022198
:10BEB0003046FDF781FAFFE50A2206212846FEF703
:10BEC0008BFC0680A3894380E3898380238AC38017
:10BED000638A0381F0E5164BD3E90023002203F0C7
:10BEE000005313433FF4E8AD124BD3E90023002382
:10BEF00002F0400213433FF4DFAD0A220721284637
:10BF0000FEF76AFC0680238A4380638A8380A389C4
:10BF1000C380E389DDE7037B0E2B7FF4CDAD0B46B9
:10BF2000324600211A2088E74FF4376141E700BF0D
:10BF3000504600205846002028250020A506010074
:10BF400070B506460D46144613210522FEF71FFC68
:10BF5000052106F1080002F083FA01230370A0F81E
:10BF60000150A0F8034070BD0379012B06D0023BBD
:10BF7000DBB20A2B0AD8074AD0567047037A03F07F
:10BF80000303032B0CBF0220032070474FF0FF3048
:10BF9000704700BF78060100024B00211860084678
:10BFA000FEF774BD30250020F7B507460E460C4657
:10BFB000351B3D448CB1F4F7E9FF032C019007D900
:10BFC00004220DEB02012846F5F7A8FC043CEFE73C
:10BFD000224601A92846F5F7A1FC002003B0F0BDD8
:10BFE00008B5002301F050FB002008BD0048704751
:10BFF000342500202DE9F04F87B0984600238DF8B6
:10C000001030062301248DF812300E46022307213A
:10C010008DF81330019315469DF840B09DF844A06B
:10C020009DF858908DF811408DF814408DF815103A
:10C03000FCF75AFF019B0746002840F0ED80784945
:10C04000087AB8F1040F64F3020008727DD916F083
:10C05000100F06F0030213D003208DF80E3006AB4C
:10C060008DF80C001A4404208DF80D008DF80F7027
:10C07000330712F80C8C68D5A0460023CB600EE085
:10C08000032A00F0CB8006F00C030C2B00F0C680D6
:10C090000B7A69F302030B724FF00508CD600B7841
:10C0A0009DF84C00019160F302039DF8500060F38D
:10C0B000C4030B70FCF710FF90F84F500199034632
:10C0C00006AA05EB8500C5EBC00502EB08005A5D2A
:10C0D00010F8080C60F303026FF304125A55D2B241
:10C0E00002F00F00012894BF42F020026FF34512C6
:10C0F0005A550A786BF346120A70D2B2500603EB17
:10C10000050409D56AF3C7120A70464812990193CB
:10C110000622F5F703FC019B5A5D0BF0010B6BF354
:10C1200086126FF3C7125A55D2B202F00F010129DD
:10C130000FD16AF3C7125A551299062204F108006A
:10C14000F5F7ECFB0C23637043E0B8F1010FA5D1C8
:10C1500093E707295BD1A17801F0C00166F387114D
:10C16000A170B0064FF0000104F1020304F10402D3
:10C17000E1700AD4A17811F0C00F06D1B9F1040F13
:10C180001EBF0122E27004F10A02710644BFE17889
:10C190000132A2EB030348BF41F04001DBB248BFCC
:10C1A000E170022B8ABFA178012303F1FF30637095
:10C1B000E37884BF60F30501A1705B0609D5159B88
:10C1C0001BB31B787F2B02D1159900230B7002F84B
:10C1D000013CFCF785FE90F84F2002EB8203C2EB96
:10C1E000C3020424835C64F3030303F0CF036BF303
:10C1F00086136FF3C713811883544B780BB906234A
:10C200004B70384607B0BDE8F08F159BDFE76378C9
:10C21000002BDED1062396E70C27F2E71227F0E782
:10C2200034250020362500202DE9F0410F46064632
:10C23000FCF752FE90F84F5005EB8502C5EBC202A9
:10C24000044610F802E00EF00F03012B00EB020190
:10C2500040D0072B3ED090F84E30AB4204D1013590
:10C26000EDB2022D08BF002505EB8503C5EBC30326
:10C2700004EB0308E05C6EF303006FF30410E0547A
:10C28000A05C14F803E0C0F3401060F3451E04F80E
:10C2900003E0A05C5FFA8EFEC0F3801060F3861EA0
:10C2A00004F803E0A25C5FFA8EF0D20962F3C710D3
:10C2B000E0540622023108F10200F5F72FFB324666
:10C2C000394608F108000636F5F728FB88F80160C2
:10C2D00084F84F50BDE8F0812DE9F04106460F4645
:10C2E000FCF7FEFD90F84F3090F84E209A4204463D
:10C2F00036D15D1CEDB2022D08BF002503EB830291
:10C30000C3EBC2022BB203EB8300C3EBC0034FF0BD
:10C31000040EE05C6EF3030000F0EF006FF34510D5
:10C32000E054A05CA118E25CC0F3801060F38612B8
:10C3300004EB03086FF3C712E254B31D88F8013011
:10C340000622023108F10200F5F7E8FA32463946D2
:10C3500008F10800F5F7E2FA84F84F50BDE8F081E3
:10C360001D46CBE72DE9F34720B902B0BDE8F04701
:10C37000FDF7A6BDFCF7B8FD8146002855D1FCF7B6
:10C38000ABFD0746FCF7ACFD97F84F40334D04EB8F
:10C390008403C4EBC30407EB04083B5D03F00F0206
:10C3A000072A10D198F80320D2070AD54946C3F3CB
:10C3B0008010F6F7A9FB0622014608F10400F5F704
:10C3C000ADFAFF2422E090F84F3003EB8306C3EB75
:10C3D000C603C6182878C0F3C10000F0EDFB28782A
:10C3E00010F0400A23D04A46A91CC00900F028FCDE
:10C3F000FF28044602D0484600F0BCFD41462046D6
:10C4000000F05CFD3146204600F058FD2A78287A7D
:10C41000A9890094C2F3C10300F0070002F00702EB
:10C42000FDF782FB02B0BDE8F0870020FAE7385D37
:10C430005146C0F38010F6F767FB0622014608F16B
:10C440000200F5F76BFA385D5146C0F38010F6F73D
:10C450005BFB06220146B01CB1E700BF342500207B
:10C460002DE9F8438146884617461E46FCF750FDE5
:10C4700088B90A4D2C79A5F8008069F30304224697
:10C4800066F3051213469DF820206F8062F3871330
:10C490002B71BDE8F8830C20BDE8F883442500200B
:10C4A000F0B585B020B905B0BDE8F040FDF716BE87
:10C4B000FCF72EFD064640BB154C2079800900F0A4
:10C4C0009DFB237913F0010506D013F0200503D05E
:10C4D000304600F04FFD0125267906F00F07C6F320
:10C4E000001600213046F6F70FFBFF220392227957
:10C4F0002388029592090192628800923146024691
:10C500003846FDF70DFD05B0F0BD0020FBE700BF8C
:10C51000442500202DE9F04F85B01E46BDF8483077
:10C5200003938046894615460E9F9DF83C40BDF812
:10C5300040A0BDF844B0FCF7EBFC039BA0BB00930C
:10C5400052465B4639463046FCF706FD68BB284636
:10C5500000F054FBDDB1FF27A31E012B22D80020E1
:10C5600000F008FD04F00104012600212046F6F742
:10C57000CBFA4346024621460020119710960F95AC
:10C58000CDF8389005B0BDE8F04FFDF7C9BC00F01C
:10C590008DFC0028DFD039462A46304600F050FB9B
:10C5A0000746D9E70026E0E70C2005B0BDE8F08F8C
:10C5B00070B501F0DFFA01F0B3FB1B4B1B4A197891
:10C5C0001378CB1ADB0701D4117070BD01F09CFC0D
:10C5D000064601F081FC361A01F096FC144B1978DE
:10C5E000144B0546187801F08BFA281A40F2712195
:10C5F000801B06F26934B4FBF1F401FB040401F082
:10C600008FFC01F093FCA0420BD801F011FB2146F6
:10C61000012001F001FC01F031FCBDE8704001F0A7
:10C6200061BC04F27124EEE7512500205025002062
:10C630004F2500204E25002038B501F0B1FAC4B2D4
:10C640008CB101F0CDFAC5B201F094FA01F068FBAB
:10C6500044B1064B187801F0D5FA1DB1044A13888D
:10C660000133138038BD2546EEE700BF4E2500207C
:10C670004C25002070B515460C46064600F0A4FF78
:10C68000FCF7D4FB436801211B68984701F074F95B
:10C69000284601F03BF9174D174B032C8DBF0422A0
:10C6A000012204F1FF342A7094BF02FA04F400223C
:10C6B0001A7098BF2C701978287801F077F99620B5
:10C6C00001F03EFB01F0A6F97000023001F0AAF97A
:10C6D0000A4801F0BFF90A4940F25B6001F074FAC0
:10C6E0002A78520002F0FE02FF21082001F0CAF968
:10C6F000002070BD4E2500204F25002004090100B8
:10C7000055555500072A2DE9F0410C46904651D861
:10C710005A1E032A4ED8284E3278002A4AD1274A78
:10C720001946FFF7A7FF054650BB254A137801338A
:10C73000137001F063FA08F1FF3307460230062B4D
:10C7400005D8DFE803F02025282B2E3134001D49C1
:10C750002246F5F7E3F8384687F800807C7001F050
:10C76000C9F901F065FA00F057FF0022C11C012051
:10C7700001F0F2FA01F082FB01F0B4FB0123337007
:10C780002846BDE8F08122460F21F5F7F3F8E2E7ED
:10C7900022465521F9E722460B49DAE72246FF21D6
:10C7A000F3E722460021F0E72246F021EDE722469A
:10C7B000AA21EAE70125E3E74A250020B1C50000E8
:10C7C00051250020020801000307010038B54B1E67
:10C7D000022B1AD80E4D2B78BBB90E4AFFF74AFF31
:10C7E000044680B901F00AFA01F07EF90A4B187884
:10C7F00001F008FA00F010FF2246C11C204601F0AB
:10C80000ABFA01232B70204638BD0124FBE700BFA3
:10C810004A25002039C600004E25002010B5154CD1
:10C82000237823B3144B15491A88028000221A80FA
:10C83000134A08781378DBB298420ED101F088F9D8
:10C8400001F0F2FAFCF7F2FA436800215B689847BE
:10C8500000F0C8FE0020207010BD0233DBB20B7068
:10C8600011788B42ECD020BF40BF20BFF8E70120F9
:10C8700010BD00BF4A2500204C2500205125002076
:10C88000502500202DE9F041884615460AB1FF23C6
:10C890001370144E002400F0010716F83430DA0744
:10C8A0001DD5C3F34003BB4213D106EBC4000622DF
:10C8B00041460230F5F71DF810B9E0B2BDE8F0814D
:10C8C0003DB116F83430DB0703D42B78FF2B08BFBB
:10C8D0002C700134082CE0D1FF20BDE8F081002D40
:10C8E000F3D1F6E77F2700202DE9F0411A4DDFF85C
:10C8F0007480AE1E0024374616F83430D90724D58C
:10C9000098F800305BB115F8012C072A07D82823C6
:10C910005343124AD35C5A0701D5DB0615D510489C
:10C9200017F83430012202FA04F102780A43027047
:10C93000C3F340034278A34013430622437002FB33
:10C94000040029460230F4F7E9FF0134082C05F110
:10C950000805D1D1BDE8F081812700200C260020F8
:10C96000BF2700204C27002008B5FCF7BDFA28B9E6
:10C97000FCF7CEFAB0FA80F0400908BD002008BDEF
:10C98000F8B5104E104D0024282707FB04F1735C06
:10C99000DA0713D5012202FA04F02A780243C3F31E
:10C9A00080132A706A78A34013430622013102FBE8
:10C9B0000450314402306B70F4F7B0FF0134082C9E
:10C9C000E3D1F8BD0C2600204D27002007280CD805
:10C9D00028235843064A135C1118C3F3C00028B13A
:10C9E000C3F3400010B1486A70470020704700BF91
:10C9F0000C260020024B1B7803700248704700BFD2
:10CA0000822500208B25002038B50C4698B10729D7
:10CA100003D9F1211048F3F719FF104D15F8342010
:10CA2000D20703D4F2210C48F3F710FF05EBC4043E
:10CA30006478204638BD072903D9F5210648F3F765
:10CA400005FF28236343064AD35CDB07F1D4F721B3
:10CA50000148F3F7FBFEECE7080901007F270020FF
:10CA60000C26002010B5104B1B788342044604D8D6
:10CA700040F201110D48F3F7E9FE0D4B1C5D072C48
:10CA800004D940F203110948F3F7E0FE2823634379
:10CA9000084AD35CDB0704D44FF482710348F3F7F0
:10CAA000D5FE204610BD00BF8225002008090100E8
:10CAB000832500200C260020072838B5054610D80D
:10CAC0002822094C4243A25CD30704D440F20F1140
:10CAD0000648F3F7BBFE28206843205CC0F34010F3
:10CAE00038BD002038BD00BF0C2600200809010019
:10CAF000034B044A002814BF10461846704700BF75
:10CB00004D270020BF2700200820704710B5FCF7F4
:10CB1000F3F9044610B10C24204610BDFCF70EFAC0
:10CB2000C307F8D4074A234612F833106FF3000105
:10CB300002F833100133082BF6D1034B00221A7090
:10CB4000EAE700BF7F270020E02C002038B505462B
:10CB5000FCF7D2F9044610B10C24204638BDFCF78E
:10CB6000EDF9C307F8D42878FF2802D10F4B1C70C9
:10CB7000F3E72246691CFFF785FE072813D80C4B04
:10CB800003EBC0025578072D06D8282209496A43CD
:10CB90008D5C64F345158D5413F830206FF300025B
:10CBA00003F83020D9E70224D7E700BFE02C0020AB
:10CBB0007F2700200C26002008B50D4B00221A709C
:10CBC0005A7028B1FCF7BAF9C30701D4FFF78CFEFD
:10CBD000084B00221A705A70074B1B7833B1FCF7D0
:10CBE00097F918B9BDE80840FFF7CABE08BD00BFF5
:10CBF000BF2700204D2700204C27002008B50D4BF3
:10CC000000221A705A70C30704D5FCF775F908B9E9
:10CC1000FFF76AFE084B00221A705A70074B1B7808
:10CC200033B1FCF761F918B9BDE80840FFF7A8BEB9
:10CC300008BD00BFBF2700204D2700204C27002043
:10CC40002DE9F0478A4614460AB1FF231370DFF836
:10CC50005480002500F0010928266E43EFB218F831
:10CC60000630DA071AD5C3F380134B450FD1701C79
:10CC7000062251464044F4F73CFE60B13CB118F83E
:10CC80000630DB0703D42378FF2B08BF277001355C
:10CC9000082DE1D1FF273846BDE8F087002CF2D1FE
:10CCA000F5E700BF0C2600202DE9F3410746FCF70D
:10CCB00023F9054620B10C25284602B0BDE8F081D5
:10CCC000FCF73CF9C307F6D43878FF2803D11F4B93
:10CCD00001221A70F0E707F101080DF10702414641
:10CCE000FFF7D0FD07282DD99DF80760072E2BD818
:10CCF000174C3A7814F8363004EBC60062F341035F
:10CD000041460622023004F83630F4F707FE2A4680
:10CD100041463878FFF794FFF300072823440ED8E4
:10CD2000587028230B4A5843135C43F020031354D4
:10CD300014F8363043F0010304F83630BCE7FF2224
:10CD40005A70F5E71225B7E70725B5E7E02C002074
:10CD50007F2700200C26002038B50E4B1B780D468F
:10CD6000ABB1072913D890B928220B4C4A43A25CD7
:10CD7000D20704D440F2C5110848F3F767FD282113
:10CD80006943605C430702D5C0F3001038BD012041
:10CD900038BD00BF4C2700200C26002008090100E8
:10CDA0000728F8B504460F46164604D94FF4E67135
:10CDB0000E48F3F74BFD28230D4D6343EB5CDB0777
:10CDC00004D440F2CD110948F3F740FD282101FBBE
:10CDD00004F301FB0451EB5CC3F380133B7030465A
:10CDE00006220131BDE8F840F4F798BD08090100BA
:10CDF0000C2600202DE9F0471A4B1B787BB31378E3
:10CE0000FF2B2CD1184E00244FF02808B64608FB03
:10CE100004F35FFA84FCF75C17F0010F06EB0305DF
:10CE20001AD0C7F38017874216D106334F1E3344FA
:10CE300015F801AF17F8019FCA450DD19D42F7D1F2
:10CE400028235C4382F800C01EF80400430706D57F
:10CE5000C0F30010BDE8F0870134082CD7D10120C1
:10CE6000BDE8F0874C2700200C26002070B40D4C44
:10CE70002478A4B1072A12D828250B4C05FB02F60A
:10CE8000A65D36070BD550B14B7903F0C003402B9C
:10CE900005D105FB0242D01D70BCF4F7ABBD0020EC
:10CEA00070BC70474C2700200C260020024B1878DD
:10CEB000003018BF012070474C2700202DE9F041B9
:10CEC00005460C4601F10208FFF790F8072D0646CB
:10CED00033D82822254F6A43BA5C11072DD5930712
:10CEE00004D44FF404712248F3F7B0FC237843F0E4
:10CEF00040032370282303FB05730622596A40462A
:10CF0000F4F70CFD237803F00F02012A2CD1072D32
:10CF100004F108001ED82822144902FB05F7CF5D52
:10CF20007F0717D502FB051143F08003237006220B
:10CF30001E31BDE8F041F4F7F1BC30782378C0F33E
:10CF4000411060F386132370414600F00100F5F7AD
:10CF5000DBFDD7E73146227811F8023BDB0963F3AA
:10CF6000C71222700622E4E7BDE8F0810C260020FB
:10CF7000080901002DE9F04F87B0804602F07AFDE4
:10CF8000CDE90001B8F1000F40F0C980654BD3E94D
:10CF900000014C1C08BFB0F1FF3F00F0C080DDE98C
:10CFA00000341B1A1846604B1A6864EB0104002316
:10CFB000904274EB0303ACBF012600265B4DDFF803
:10CFC00078A1A5F1070900244F462823634319F8E7
:10CFD0000330DA0741D50EB998073ED428236343BE
:10CFE000FB5C590718D52A7C514B03EB021303F164
:10CFF00010020DF1070112F8010D01F8010F934223
:10D00000F9D105F1170102A8F4F707FD20B140F2AC
:10D0100082214848F3F71AFC28236343FB5C1A0774
:10D0200015D502A92846F4F7F8FC20B140F2892171
:10D030004048F3F70BFC062202AB02FB04ABC5F839
:10D040001D3019465846F4F769FCC5F81DB0282371
:10D050006343FA5C42F00202FA540134082C05F1F1
:10D060002805B2D126B1DDE900122E4BC3E900122A
:10D07000B8F1000F50D0FBF737FF00284CD0FEF777
:10D08000B5FF03785B06804646D5FBF725FF90F891
:10D090004F4090F84E3004EB8402C4EBC202A3422E
:10D0A000054600EB020704D10134E4B2022C08BFAC
:10D0B000002404EB8403C4EBC303A95CE85C61F3C4
:10D0C00003006FF30410E854AA5CC1B2C2F340122B
:10D0D00098F8000062F34511E954002208F10201BA
:10D0E000C009EE18FFF7ACFD0728804604D940F2CE
:10D0F0004E211048F3F7AAFB31464046FFF7DEFE0B
:10D100007A7807F10801063A06F10800F4F706FC00
:10D110007B78737085F84F4007B0BDE8F08F01262B
:10D120004CE700BFD82C00200C2D00201326002037
:10D130008B250020080901005225002008B5012098
:10D14000FFF718FF034B04491A680448BDE808407C
:10D1500002F0A2BF0C2D0020E42C0020582D00204E
:10D16000074B1B7830B14BB1064B07491A6807488B
:10D1700002F092BF13B1044802F02ABF704700BF0B
:10D180004C2700200C2D0020E42C0020582D0020DE
:10D190000820704710B5FFF7E7FB78B10849002376
:10D1A000282404FB03F20133885C082B6FF3000092
:10D1B0008854F6D1034B0020187010BD0C2010BD10
:10D1C0000C260020822500202DE9F04F85B007466F
:10D1D00089469246FFF7C8FB002800F0868007F1D9
:10D1E00001080DF10F0241463878FFF729FD0728A5
:10D1F0007DD99DF80F50072D7BD805EB850B3E4C54
:10D200004FEACB0B28266E430BF101000622414664
:10D210002044F4F783FB3978A35DA21961F38613E8
:10D22000484610210192A355F4F7C9FCA35D1021D3
:10D2300060F382035046A355F4F7C1FCA35D019A45
:10D2400000F0010060F3C30313F0040FA35538D1BD
:10D2500058B10BF10700102251462044F4F75EFB51
:10D26000282303FB054300225A6228266E430BF154
:10D270001800062200212044F4F77CFBA35D03F094
:10D28000FD036FF30413A355002241463878FFF7DE
:10D29000F9FA0728A35D9DBF184A43F0200302EB6B
:10D2A000C0006FF34513A3554FF0280398BF457096
:10D2B0005D430020635D43F00103635505B0BDE8A5
:10D2C000F08F0F4B1978D1750E4A55544A1C1A70BD
:10D2D0000D4B03EB011309F11002013B12F8011D84
:10D2E00003F8011F4A45F9D1B2E70C20E6E7122006
:10D2F000E4E70720E2E700BF0C2600207F2700209C
:10D3000082250020832500208B2500202DE9F84F61
:10D310008146FFF729FB002853D009F1010A0022BA
:10D32000514699F80000FFF78BFC072880464BD840
:10D330004FF0280B264C0BFB00F3E218E35C5B0775
:10D3400024D5244E3578013D15F0FF051BD0D77D3F
:10D35000AF4218D02048102200EB051100EB071057
:10D36000F4F7DCFA00230BFB03F16218615C11F0A7
:10D37000010FD8B221D049071FD5D17DA9421CD1B8
:10D38000164BD775D8553378013B33700022514680
:10D3900099F80000FFF776FA07289FBF104B03EBC0
:10D3A000C000FF234370282000FB08F0235C6FF3CC
:10D3B000000323540020BDE8F88F0133082BD2D19D
:10D3C000E1E70C20BDE8F88F0220BDE8F88F00BF30
:10D3D0000C260020822500208B250020832500209C
:10D3E0007F27002070B55C7904F0C004402C1D46F6
:10D3F00017D119B10022FFF723FC0246072A10D8E3
:10D400002821084C01FB02F3E35CDB0709D5182057
:10D4100011FB0200204429460622BDE87040F4F7C3
:10D420007DBA70BD0C26002038B500220D46411C87
:10D430000078FFF705FC072801D9022038BD282411
:10D44000182314FB0030074C044406212046F4F74F
:10D45000B6FB0028F1D0062221462846F4F75EFAF2
:10D46000002038BD0C26002010B500220C46411CBF
:10D470000078FFF7E5FB07280AD8064B282202FBB5
:10D4800000300622416A2046F4F748FA002010BD19
:10D49000022010BD0C26002010B50446FFF764FAE8
:10D4A00040B11CB1012C01D0122010BD024B1C70E8
:10D4B000002010BD0C2010BD4C2700204FF47A73C3
:10D4C0005843014B186070470C2D002038B50546B5
:10D4D0000C46FFF749FAD8B10022691C2878FFF7FB
:10D4E000AFFB072816D81CB1012C0AD0122038BD7A
:10D4F0002823094A5843135C64F30413135400208F
:10D5000038BD2823044A5843135C43F01003F5E761
:10D510000C2038BD022038BD0C260020194A0023FB
:10D5200030B41370184A12F833106FF3000102F888
:10D5300033100133082BF6D1144A15490023137018
:10D54000144A1160144A15494FF0FF354FF0FF346B
:10D55000C2E90045282505FB03F201338C5C082B4A
:10D560006FF300048C54F6D10D4B00221A7020B1D9
:10D570000C490D4830BC02F01BBD0B4830BC02F01A
:10D5800027BD00BFE02C00207F2700204C27002073
:10D59000A0BB0D000C2D0020D82C00200C26002054
:10D5A000822500203DD10000E42C0020054B002204
:10D5B000C3F808254FF44032C3F84423C3F80423CA
:10D5C000704700BF00B00040044A1378591C117026
:10D5D000012013B9024A106018467047F127002055
:10D5E00000B0004010B5094C23781BB92D21084824
:10D5F000F3F72CF920780138C0B22070012310B95C
:10D60000044A136010BD184610BD00BFF12700206A
:10D610004609010004B00040014BD3F804057047EF
:10D6200000B0004000F5A870014B43F8201070478F
:10D6300000B00040F0B5124B124D01210026AE465D
:10D640001A462960C3F80405C3F80061C3F80461F1
:10D650001960D3F8004134B9D3F804411CB9D3F8A8
:10D660000445002CF5D1CEF80010D2F80441002C6E
:10D67000E7D1D2F80475002FE3D0C2F80445F0BD1D
:10D6800000E0004004E0004070B58CB00E46154646
:10D690000146102268461C46F4F782FA10220DEB70
:10D6A00002003146F4F77CFA6846FFF7C3FF25B164
:10D6B000102208A92846F4F773FA24B1102208A909
:10D6C0002046F4F72BF90CB070BD0000094A0A4B54
:10D6D000002814BF1846104603F5F03302F5E24265
:10D6E0003C32C3F810250122C3F81405C3F8042501
:10D6F000704700BF04100040001000402DE9F047C3
:10D70000754D764C2E78764FC4F8607533B24FEA7B
:10D71000C30E88460EF1804101F5F831C4F8641556
:10D7200006F10B04E4B2E4006E4904F180444FEAD0
:10D73000830C04F5F8346144C4F8101506F10807A9
:10D740000EF1040E002800F0AA80022A00F0878063
:10D7500049F6C4704AF65C09042A18BF8146B8F13C
:10D76000020F7FD042F2B84247F27420B8F1040FA2
:10D7700018BF104609F5FA795B4AC4F8142518F069
:10D78000040F48444FF47A7AB0FBFAF06DD042F2BD
:10D79000B84444F69041B8F1040F18BF21469C00EC
:10D7A00004F18044FAB204F510474944D7F84085A3
:10D7B0004E4FB1FBFAF1C7F84885D7F84885414587
:10D7C00036BFD7F848850121A8EB0101C7F84815F5
:10D7D000424FDFF824814449C7F89085C7F8941573
:10D7E00004F5F831D1F8004844F48034C1F8004819
:10D7F000D10001F1804101F5F8310EF1804202F5CE
:10D80000F832C1F81085C1F81425394AC7F89825AF
:10D8100002F5FD4270326244C7F89C254FF4802225
:10D82000C7F804259B0003F1804303F51043D3F8A8
:10D83000402582428BBFD3F840250122101AC3F83D
:10D84000402588BFC3F84005244B4FF49062C3F8CD
:10D850000425731C03F001032B70BDE8F08749F623
:10D8600040497CE741F2883084E79A0002F1804227
:10D8700002F5F832D2F8004824F48034C2F80048A7
:10D88000FAB2D20002F1804202F5F832C2F8101565
:10D890000EF1804101F5F831C2F81415C2E7154ABE
:10D8A000C4F81425FAB2D20002F1804202F5F8322F
:10D8B0002C20C2F810150EF1804101F5F831C2F8A4
:10D8C00014150CF1804202F5F832D2F8001821F458
:10D8D0008031C2F80018A5E7142A002000F00140AA
:10D8E0000C110040409100400010004000900040AA
:10D8F000501100400410004048910040024B1B684A
:10D9000003B11847704700BF102A0020064B18606B
:10D91000064B1022C3F80423054B0222C3F88021D2
:10D920000120F3F75BBE00BF102A0020001000406A
:10D9300000E100E04FF080434FF0FF320021C3F8D8
:10D94000002EC3F8042EC3F8081EC3F80C2EC3F82B
:10D95000101EC3F8142EC3F8182EC3F81C2EC3F8DB
:10D96000202EC3F8242EC3F8282EC3F82C2EC3F87B
:10D97000302EC3F8342E704708B50120F3F73EFE71
:10D98000084B0022C3F8FC2F0122C3F8FC2F064AE3
:10D99000136823F0807323F0010343F08073136056
:10D9A00008BD00BF00100040741700400228144B4F
:10D9B00010D0042814D01A6822F000421A60032103
:10D9C000104BC3F81015D3F8502642F00102C3F8EB
:10D9D000502670471A6822F000421A600421EFE7CF
:10D9E0001A6842F000421A601A6822F0FF0211F031
:10D9F000010F42F05C0214BF052106211A60DFE727
:10DA00003C17004000100040014BC3F80C05704764
:10DA100000100040024B0822C3F80C25704700BFDD
:10DA200000100040014BC3F808057047001000408B
:10DA3000074BC3F85405D3F8182522F00072C3F839
:10DA40001825D3F8182542F00072C3F8182570473E
:10DA5000001000400A4A0023C2F82C350123C2F806
:10DA60003035C378C2F82435437881781B0443EA03
:10DA70000163017843EA0123C2F81C35704700BFF7
:10DA80000010004002F00103C2F34202022A23D038
:10DA9000042A0CBF4FF0C74200220BB142F480129F
:10DAA000C0F108031B0400F00F0040F4807003F481
:10DAB0007023034313430A4AC2F81435D2F81805F9
:10DAC000084B0340C2F81835D2F8183543F44033F8
:10DAD0001943C2F8181570474FF08072DDE700BF98
:10DAE000001000400000F8FE014BC3F80405704729
:10DAF00000100040014BC3F80405704700100040BF
:10DB0000022804D004280CBF2B202920704728208D
:10DB100070470120704729207047022803D004284D
:10DB200003D00A2070470520704711F0010F14BF81
:10DB30001E20142070470000014B01221A6070471C
:10DB400004100040014B01221A6070470010004091
:10DB5000074A4FF49063C2F8083501235360D3603D
:10DB6000A2F5F0320021C2F800121361704700BF25
:10DB700000F00140044B0022C3F80021C3F80C213F
:10DB8000C3F81021704700BF00100040034BD3F8CA
:10DB90000001003018BF0120704700BF0010004096
:10DBA000034BD3F80C01003018BF0120704700BFB1
:10DBB00000100040034BD3F85005B0FA80F0400944
:10DBC000704700BF00100040044B40F20312C3F83E
:10DBD0003425C3F83805C3F83C15704700100040E1
:10DBE000034BD3F80004003018BF0120704700BF7A
:10DBF000001000400048704704290020004870478A
:10DC000008290020044B03220021C3F80022024609
:10DC10000846FFF773BD00BF00100040034B03210F
:10DC2000C3F8001201460120FFF768BD0010004054
:10DC3000054B0322C3F8002203F5F0334FF4906242
:10DC4000C3F80825704700BF00100040034AD2F80F
:10DC5000003243F48873C2F800327047001000406D
:10DC6000014BD3F84805704700100040024B0022DA
:10DC7000C3F81C21704700BF00100040034BD3F8CD
:10DC80001C01003018BF0120704700BF0010004089
:10DC900030B50024A30003F1804303F580531568D9
:10DCA000C3F8005601349588C3F82056082C02F1B9
:10DCB0000602EFD1024B40EA0120C3F8400630BD16
:10DCC00000100040034AD2F8403623F0FF03C2F8A8
:10DCD0004036704700100040024B0022C3F8142168
:10DCE000704700BF00100040034BD3F81401003010
:10DCF00018BF0120704700BF00100040014BD3F84F
:10DD00001004704700100040044BC3F86005D3F8BE
:10DD1000002242F04002C3F8002270470010004089
:10DD2000054B4FF48022C3F8482303F5A033034A80
:10DD3000C3F80825704700BF00B000407F200400F2
:10DD4000034B044A1B7803F5A87342F8230070477D
:10DD5000142A002000900040F8B5A2F57423274C47
:10DD6000DFF8B0E0A3F51073A34288BF02F1E872B8
:10DD7000234B244C82BF02F5D43201F1FF3102F56E
:10DD8000A5720125B2FBF4F40026022204271D60CF
:10DD9000C3F8F864C3F80475C3F8FC24C3F8344529
:10DDA000CEF848154FF48021CEF8441316490C3BA9
:10DDB0000EF5A47EC1F818E5C1F81C35C1F804259C
:10DDC000FFF784FC114B124A1560C3F80465C3F8D1
:10DDD0001075C3F808651D60A3F5FD43743BC1F8D9
:10DDE00048354FF41063C1F84C25C1F800384FF4A2
:10DDF0009053C1F804382046F8BD00BFBFBDF07F86
:10DE00000C80004040420F0000F0014000900040B4
:10DE10000C90004000B00040024BC3F84015FFF7E3
:10DE200055BC00BF00800040044A01231360D3604A
:10DE30000C3202F6F4721360D36070470480004025
:10DE40000C4B0D4AC3F8440503F5B833C3F8282535
:10DE500002F5DE424032C3F82C2502F58072C3F889
:10DE60003025A2F5E242343AC3F834251822C3F82B
:10DE70000425704700800040041100400B4B0C4A01
:10DE8000C3F8202502F5DE424032C3F82425A2F56E
:10DE9000DE423C3AC3F8282502F5DE424032C3F8A0
:10DEA0002C250C22C3F80425704700BF00F0014068
:10DEB00000110040014BD3F844057047008000403A
:10DEC000014B1860704700BF0C2A0020014B1868F6
:10DED000704700BF0C2A0020014BD3F84005704763
:10DEE00000800040064B074AC3F8382502F5DE42A1
:10DEF0003C32C3F83C252022C3F80425704700BFFC
:10DF000000F001400C110040014BD3F84805704768
:10DF100000800040014BD3F8480570470080004066
:10DF2000014B01221A6070474C800040014BD3F82E
:10DF30004C05704700800040214B10B50024C3F809
:10DF400000450224A142C3F8004503D0042924D08F
:10DF50001C4900E01C491A4BC3F80415C3F8080516
:10DF60001A48C3F80C05C3F81025194AC3F814253C
:10DF70000022C3F800221749C3F80421C3F808217E
:10DF8000154AC2F8401501F55F41C2F84415402119
:10DF9000C2F8041501221A6010BD0321C3F81C1534
:10DFA0000D4B0E49C3F8781501F55E41BC31C3F83D
:10DFB0007C154FF40051C3F804150949CBE700BFA5
:10DFC00000F00040010000010100010108290020CB
:10DFD000F82700200411004000F0014050110040DB
:10DFE0000100020110B50E4B00220224C3F80025E7
:10DFF000C3F800450B4CC3F80445C3F80805C3F843
:10E000000C1509480949C3F81005C3F81415012176
:10E01000C3F80012C3F80421C3F80821196010BD29
:10E0200000F000400000010108290020F82700202E
:10E030000C4B0222C3F80423D3F804216AB1022254
:10E04000C3F80823084A4FF40041C2F88011D3F8FE
:10E050000801B0FA80F04009704720BF40BF20BFE0
:10E06000EAE700BF00F0004000E100E0034BD3F816
:10E070000004003018BF0120704700BF00F00040CE
:10E0800038B5134C134D0323C4F80035C4F8040508
:10E09000C4F80815D5F80435013BC4F81035002143
:10E0A0000D4BC4F814354020C4F80011C4F8041115
:10E0B000C4F80811FFF728FE084B094AC5F82811D3
:10E0C000C3F840254022C3F84445C3F8042538BDB1
:10E0D00000F0004000100040F427002000F0014054
:10E0E00028110040014BD3F80004704700F00040B5
:10E0F000044A0023C2F8283102F56042C2F8003514
:10E10000704700BF00100040084BD3F8280160B1F1
:10E1100003F56043D3F8000138B1D3F8040120B10E
:10E12000D3F80801B0FA80F04009704700100040B1
:10E13000012910B5144603D01C210648F2F786FBCE
:10E1400018201CB1BDE81040F3F748BABDE81040F4
:10E15000F3F754BA8209010008B539B101290AD090
:10E1600031210648F2F772FB002008BD0B20BDE804
:10E170000840F3F757BA1820F9E700BF82090100F9
:10E1800088420AD018B94B1E58425841704701289E
:10E1900005D1B1FA81F04009704701207047002095
:10E1A0007047000029B1012909D054210548F2F730
:10E1B0004DBB4FF40062044BC3F8002170474FF091
:10E1C0008072F8E78209010000E100E0032810B541
:10E1D000044603D929210648F2F738FB054B1C5D9C
:10E1E0001CB92C210248F2F731FB204610BD00BFBC
:10E1F000C4090100C0090100023810B41C460328FC
:10E2000031D8DFE800F002101827032906D1174B98
:10E2100000219C60002010BCF3F750BD4B21144836
:10E2200010BCF2F713BB042903D1124B01219C60EF
:10E23000F0E76221F3E7032903D0042906D08821FF
:10E24000EDE70D4B00219C600120E4E70B4B012121
:10E250009C60F9E7042904D1094B01219C6003204B
:10E26000D9E7A021DBE7A621D9E700BF604600205F
:10E27000C40901007046002080460020904600201E
:10E28000A046002001460020FFF7CCB970470000EF
:10E290008279044B03EB4213DB69C01A024BC010B6
:10E2A00058437047A0470020ABAAAAAA10B5094B53
:10E2B000827903EB42130A689B695C6823689A427F
:10E2C00094BF0A600B60FFF7E3FF94E80C0002FBC9
:10E2D000003010BDA04700202DE9F3410546019113
:10E2E000164601F0A7FB07464FF02003EFF3118815
:10E2F00083F311886B8A002B3DD02A8A9A422AD94F
:10E300000021284601F09EF828B388F311880446BE
:10E31000019B002B3CD0731C012B06D901F08AFB1A
:10E32000C01BB04294BF361AB61BA3791E4F07EB31
:10E33000431332469B691B6801A91B682046984716
:10E340000546206128BBA079214607EB401001F06B
:10E350005AF82C4618E0688A431E6B8288F31188AD
:10E360002C8A241AE869182303FB04040E4BED1AC7
:10E370006D11A571CCE788F311883146284601F06C
:10E3800061F804460028C3D1204602B0BDE8F08100
:10E39000236101232371002323606371019AA38108
:10E3A0002369E281A360EFE7A047002083695B68EF
:10E3B0000A461968FFF790BF70B5064601F042F8AB
:10E3C000054628B10446637913F0010302D12360A6
:10E3D000284670BD0021304601F034F86379206092
:10E3E00023F0010363710446EDE710B40A46146894
:10E3F00014B910BC01F00CB8537943F00103537108
:10E400002246F4E7F8B5154D0446002604B9F8BDD8
:10E4100023792768013BDBB22371002BF7D12169F7
:10E4200059B163799B0707D4A37905EB43132046C1
:10E430009B691B689B6898472661A079A66005EBDD
:10E44000401326605B691BB1204698473C46DDE7D8
:10E45000214605EB401000F0D6FFF7E7A04700206B
:10E460008388026819448180D018704730B483884B
:10E4700004689D188580E01830BCF3F74FBA838894
:10E480005B1A83800368194401600846704708B529
:10E49000036801211A78FFF7F2FF104608BD0268F1
:10E4A0008168C3888088521A9B1A181A704770B501
:10E4B00004680E4615464CB1A3681D4204D063683B
:10E4C0002A462146304698472468F4E770BD10B5C7
:10E4D00004688068A46801292468C16904D14B409C
:10E4E000C4F80435002010BD003321FA02F118BF32
:10E4F000012301F001018B424FF0010303FA02F303
:10E5000014BFC4F80835C4F80C35EBE710B504683F
:10E510008068A468C0692468D4F81045012980EA9D
:10E5200004001CBFD04000F001001860002010BDA6
:10E530008368186872B108605A68196002B9596036
:10E540000020704710605868814208BF5A600DE093
:10E55000024600680028F3D08142F9D10868002AF9
:10E56000F0D15A681860914200D1586000230B60C6
:10E57000E6E702688368926899691268986810B53E
:10E58000D2F810455A691143DA680240D8691B690C
:10E59000584022EA0102604022EA000010BD00005B
:10E5A00008B5094B1A786AB90121197006200521AE
:10E5B000F3F746F80620F3F711F8044B4FF000424A
:10E5C000C3F80423002008BD402A0020006000405A
:10E5D0001F288ABF094B4FF0A04300F01F0003EB38
:10E5E0008000D0F8003723F44033C0F80037D0F86B
:10E5F000003743EA0141C0F800177047000300509C
:10E60000F7B5036886689B6801F01F040D464F4903
:10E610001B79D1F8042344EA4314D2B2002303F552
:10E62000A27051F82000C0F3052084426FD122FA75
:10E6300003F0C0076BD59A0002F1804202F5C04298
:10E64000D2F8100520F00100C2F81005012202FAEC
:10E6500003F3C1F8083320460021FFF7B9FFB06883
:10E66000E84010F0010050D0F068E84010F00100E0
:10E670004BD07069E84010F0010254D0B369EB4010
:10E68000DB0748D43369F169EB4021FA05F503F063
:10E69000010305F00105AB4214BF012502252B4EF5
:10E6A000002202F5A27356F8230010F0030034D1C3
:10E6B000930003F1804101F5C04103F58073D1F867
:10E6C000107527F44F3727F44077C1F810752402EE
:10E6D0009BB2D1F8107504F47C5403F1804303F528
:10E6E000C04344EA05453D43C1F810551860019008
:10E6F000019BD1F8103543F00103C1F81035D2B2B7
:10E70000012303FA02F2C6F8042303B0F0BD01337B
:10E71000082B84D19FE70325C1E70132082AC0D125
:10E720006FF01200F1E7316921FA05F3F16921FA7E
:10E7300005F505F0010503F001012046A94214BFCB
:10E7400002210321FFF744FF1046DEE7006000408E
:10E750002DE9F84F0746856803F47040B0F5804F07
:10E760001E463ED02ADCB0F5805F3ED0B0F5405F5B
:10E770003FD050BB06F44078B8F5807F3DD0A8F577
:10E7800000746342634106F0010E4FEA4E0801290E
:10E7900048EA0E0818BFD4B248EA0020DFF8FCA00F
:10E7A00012BFA1464FF01F09002440EA830806F07B
:10E7B000020BA14523D20020BDE8F88FB0F5E04F51
:10E7C00019D006DCB0F5A04F11D06FF01500BDE8F0
:10E7D000F88FB0F5404F06D0B0F5504FF5D1072077
:10E7E000C8E70220C6E70620C4E70120C2E70320ED
:10E7F000C0E70420BEE70520BCE70323C3E73B686E
:10E800009B681A7904F01F0343EA42131F2BC6BF0B
:10E8100003F01F0352464FF0A04203F5E07342F8A5
:10E8200023800123AA68A340BBF1000F33D0134318
:10E830006A69AB600123A34016F0200F14BF134395
:10E8400022EA03036B61AA690123A34016F0400F7B
:10E8500014BF134322EA0303AB612A690123A340D7
:10E8600016F0040F14BF134322EA03032B61EA6975
:10E87000012316F0800F03FA04F314BF134322EAB6
:10E880000303EB6121463846FFF7BAFE00289ED10C
:10E890000134E4B28DE722EA0303C9E70003005024
:10E8A00001292DE9F04118BFD4B28768064612BF8E
:10E8B00025461F2500244FF00108AC4202D9002054
:10E8C000BDE8F081FB6808FA04F223EA0203FB606A
:10E8D00021463046FFF794FE0028F1D10134E4B21E
:10E8E000EBE701292DE9F04118BFD4B2876806464D
:10E8F00012BF25461F2500244FF00108AC4202D963
:10E900000020BDE8F081FB6808FA04F21343FB60C5
:10E9100021463046FFF774FE0028F2D10134E4B2FC
:10E92000ECE70000F0B585B000232D4C0293039373
:10E930002368012B07D12B48FFF71BFE02902A48C2
:10E94000FFF717FE03900023284E01279E46D6F8B6
:10E95000042307FA03F111421ED09A0002F180420B
:10E9600002F5C2421168012916D103F5A2700DF11A
:10E97000100C56F82050C2F800E0C5F340300CEB04
:10E980008000C5F30425A940126850F8085C009285
:10E990002943009A40F8081C0133082BD7D1029A6A
:10E9A0001AB110498868FFF782FD039A2AB10D4B0E
:10E9B00003F10C015869FFF77AFD2368012B0CD194
:10E9C0000848FFF7D6FD05460748FFF7D2FD284364
:10E9D00001BF206023680193019B05B0F0BD00BF1B
:10E9E0007C6100401C470020284700200060004058
:10E9F000054B1B682BB9054B1878003018BF012058
:10EA000070470120704700BF1C2100408C2A002065
:10EA1000034B186818B1D3F85C03C3F85C03704764
:10EA200024210040024B0422C3F80423704700BF96
:10EA300000200040024B0422C3F80823704700BFA7
:10EA40000020004008B5FFF7D3FF08BD024B18684F
:10EA5000003018BF0120704708210040024B4FF4DE
:10EA60000072C3F80423704700200040024B4FF4AB
:10EA70000072C3F80823704700200040012070474F
:10EA8000024B1960024B1A60704700BF842A0020B5
:10EA9000882A0020034B1B6813B1034A10681847EB
:10EAA000704700BF842A0020882A0020034B802260
:10EAB000C3F808230122DA6000F09BBA002000406E
:10EAC00008B500F095FA0B4B01221A608022C3F8BA
:10EAD000FC224FF02002EFF3118382F31188064AE3
:10EAE00012781AB1054A0421C2F8001183F3118883
:10EAF00008BD00BF082000408C2A002000E100E093
:10EB000008B50C4BD3F8042312F0800F1A4605D138
:10EB1000D2F8040310F0040006D108BDFFF768FF27
:10EB20000028F5D0012008BD034B1868003018BF3D
:10EB3000012008BD0020004008210040F7B5002357
:10EB4000094C0A4F1E46D8B2151A002D02DD256861
:10EB500001330DB903B0F0BD266025680195019D14
:10EB6000D7F818550D54EEE708210040002000406A
:10EB700007B50C4A0023136012680192019A0A4AF1
:10EB800013700A4B01221A60C3F81415FFF730FF07
:10EB90000028FBD0064B012208461A6003B05DF83E
:10EBA00004FB00BF1C2100408C2A002008200040EC
:10EBB0000C200040084B1A6882B052B10020186047
:10EBC0001B680193019B054BD3F818350B7002B0FD
:10EBD00070474FF0FF30FAE7082100400020004066
:10EBE0002DE9F3410D4E0E4FDFF838800024E5B2D9
:10EBF000531B002B03DDFFF7FBFE013418B9284639
:10EC000002B0BDE8F08100233360306801900198C4
:10EC10003B704B5DC8F81C35E9E700BF1C21004084
:10EC20008C2A00200020004037B51F4A4FF40053C3
:10EC3000C2F808354FF0A04103F1804300240320BF
:10EC40001D25C2F83407C1F87447C3F814552D25A3
:10EC5000C3F80C554FF00045C1F80855C1F87C07C2
:10EC6000C2F830471F22C3F808252C22C3F810250C
:10EC700001214FF08052C3F86C15C3F824250422FB
:10EC8000C3F80025094A146012680192019A1960BC
:10EC9000074B224602201970F2F7D2FC0220F2F74D
:10ECA0009DFC204603B030BD000300500821004009
:10ECB0008C2A00202DE9F0418378C4781E1DA342E0
:10ECC0000A4406441FD8E41AE4B2A1423EBF641AC3
:10ECD000E7B20C462344A1EB040128BF0027DBB2B6
:10ECE000C9B23444A64209D183704378BB4282BF83
:10ECF000204B01221A600846BDE8F08116F8015B3E
:10ED000002F8015DEEE70578ED1AEDB2A9423FBFCA
:10ED1000671AED19EFB20D4638BF5B18A1EB05017C
:10ED200032BFDBB227460023C9B2964606EB050C7C
:10ED3000664519D1521B0029D6D0002CD4D08C4264
:10ED40008ABF0B462346641A00F10406A1EB0301B7
:10ED50008CBFE7B20027C9B2F418A642C4D016F897
:10ED6000015B02F8015DF8E716F8018B0EF8018DE2
:10ED7000DEE700BF00D0004030B5D0B1C2780578E2
:10ED80008478531CDBB2AB4208BF0023A34210D0EF
:10ED900061B10A490244D1F808151171C3700133F9
:10EDA000DBB29D4208BF0023A34205D06FF00F00E5
:10EDB00030BD6FF0360030BD002030BD00D00040C7
:10EDC00070B5846801221146204600F0E5FD04F18B
:10EDD00018000122002100F0DFFD042384F8313007
:10EDE0000C23002584F83D300521114B84F83010A8
:10EDF0000D2684F8335084F8325084F83C6084F84F
:10EE00003F5084F83E50D3F8042542F00102C3F885
:10EE100004250122C3F800513046C3F804231A60C8
:10EE20002A46F2F70DFC3046F2F7D8FB284670BDB3
:10EE300000D00040F8B5DD070E46144606D48068C1
:10EE40000A463C30E1B2FFF735FFF8BD7AB30D203A
:10EE5000F2F7D4FB194B1A4D0020C3F80001012230
:10EE6000D3F80413C3F804234FF400571A60224662
:10EE7000D3F800E1BEF1000F1BD0013A92B2D3F8F3
:10EE800008E506F802E0C3F80001C5F88071002A21
:10EE9000EED10C480122C907026058BFC3F808230D
:10EEA0004FF40053C5F880310D20F2F797FB204650
:10EEB000F8BD20BF40BF20BFDAE700BF00D0004050
:10EEC00000E100E004D0004038B5124BD3F8003127
:10EED000FBB18568012105F13C00FFF74DFF10F102
:10EEE000100F04460DD010F1370414BF002101218A
:10EEF00005F13000FFF740FF044605F1180000F06F
:10EF000054FD044B00221034C3F800211CBF012221
:10EF10005A6038BD00D000402DE9F84385680F469F
:10EF2000144605F1180814B92046BDE8F883FF2CF3
:10EF3000234628BFFF23E41ADEB2A4B205F130094C
:10EF40004FF0FF31284600F058FD31463A4648461A
:10EF5000FFF7B0FE0646284600F027FD002EE2D05F
:10EF60004FF0FF31404600F048FDE9E71346024804
:10EF70000A461946FFF79EBECC2A002038B5084B3A
:10EF800053F82040013053F820502046A84204F1A5
:10EF90000C0400D338BD54F80C3C5B689847F4E788
:10EFA000980A0100104B70B5104C05461E469C4255
:10EFB00004D10E4CB44209D1002412E062681AB1A7
:10EFC00022681268AA420CD00C34F0E763680BB9CF
:10EFD0000C34EFE7236828461968F2F77DFC002817
:10EFE000F6D1204670BD00BF58470020BC46002027
:10EFF00070477047431C03D0034B1B68984201DBEA
:10F00000F2F784B9704700BFB04600200F4D80B5BD
:10F010000F4F05F114064FF02002EFF3118382F336
:10F0200011886B69B3420AD04BB11C69631C08D0CC
:10F030003B68A34205DDEC61F2F75AFBEBE74FF0CA
:10F04000FF342046F2F744F9F5E700BF102D002009
:10F05000B04600200248034A0021121AF2F78ABC87
:10F0600000000020D82D00200248034A0349121A4C
:10F07000F2F754BCD044002000480020B40A01003C
:10F0800008B50220FFF77AFF0320FFF777FF00F0B3
:10F09000E3FEF1F72DFC034A137A23F00103137208
:10F0A00008BD00BF502B002080B586B006AFF2F738
:10F0B000ADF9304B83F308882F4B304D304E002490
:10F0C000E02283F82220DC771C765C769C765A6AF4
:10F0D00042F4E0225A62F2F779FAF2F703FB204693
:10F0E000FFF74CFF0120FFF749FF00F009FC012367
:10F0F00035624FF4007204930394029401940094D7
:10F10000204B2149284600F04FFE6B7A23F0040281
:10F1100013F01B0F6A72344602D16B6A013325D09B
:10F1200001231A4E04930F230393002302930193A8
:10F1300000934FF4A072164B1649304600F034FE8F
:10F14000737AE66023F004037372134B6361A36167
:10F15000124BA56023F00703114C0A4A83F3098878
:10F1600063B6002181F3118810462047284600F03D
:10F17000BBFAD5E7D042002000ED00E0502B002084
:10F18000102D002081F0000090370020E02A0020A0
:10F190000DF0000090390020242D0020903900202F
:10F1A0007D09000038B5074C074DAC4201D3002063
:10F1B00038BD04F114036361A3612046F1F71AFC22
:10F1C0001C34F2E758470020584700202DE9F04F43
:10F1D0001D1E85B006460C46174656DD00F03CFC69
:10F1E00080462B484FF4004E00214FF4A02200230C
:10F1F000CEFB0501F1F744F818EB0008254B264A31
:10F20000F31A9B1002FB03FA5FFA8AFA06F1140B59
:10F21000009403AB02AA39463046F1F738FC10F1EE
:10F220000B0F0BD1009403AB02AA39463046F1F71D
:10F230002EFC10F10B0F08BF6FF00B006379029AE0
:10F2400084F804A062F3030363716368039A62F3B2
:10F250001F336360B0B1ADB110F10C0F12D14FF09C
:10F260002003EFF3118083F311882A46594600F0FA
:10F27000F1FA6B1CCCD000F0EFFBB8EB0005C7D562
:10F280006FF00A0005B0BDE8F08F4FF00008B5E759
:10F29000FFFF040058470020B76DDBB670B5047857
:10F2A00002684178134EC4EBC404A400120B01F0B1
:10F2B0000F013019F1F7C5FC4FF02003EFF3118572
:10F2C00083F3118804F11400304400F009FB40B1CD
:10F2D000EFF305830D2B04D833B1074B5B681B0597
:10F2E00002D485F3118870BD2846BDE8704000F057
:10F2F000A5B900BF5847002000ED00E007B50A1D82
:10F3000004D200236946FFF761FF18B1002003B063
:10F310005DF804FB04220DEB02010098F2F7FEFAFF
:10F3200000980430F3E710B10438FFF7B7BF704717
:10F33000034B9B680146586E08B1FFF7DFBF70476B
:10F34000102D0020F8B505460F4614464FF0200258
:10F35000EFF3118682F31188A3B10820FFF7E8FFCD
:10F36000002834D0012344600360044623685FB959
:10F370002A6803F00303134323606B682C6073B99E
:10F380006C600CE02360F1E73A6832F0030203F0AE
:10F39000030314D16A6823605AB96C602C6004219D
:10F3A00005F1080001F004F8304600F047F90020AC
:10F3B000F8BD136803F0030323431360E0E713432E
:10F3C00023603A6802F0030214433C60E7E76FF001
:10F3D0000B00F8BD10B5044630B10268930703D0A6
:10F3E000446809B1FFF79FFF204610BD002303606A
:10F3F000436000F108038360C36070470A4600233E
:10F400004168FFF79FBF00230A461946FFF79ABFDE
:10F4100038B54FF02003EFF3118583F3118843686B
:10F4200053B9016042600421083000F0C1FF284652
:10F43000BDE8384000F002B91C6804F00304214321
:10F440001960EFE72DE9F041044686B00D464FF014
:10F450002003EFF3118783F31188026882B11368E8
:10F46000416823F003038A42036008BF436001211F
:10F470001046FFF7AFFF87F3118806B0BDE8F081B3
:10F4800019B987F311880020F7E787F31188042161
:10F4900003460DEB010000F0EFFE6A1C02D000F005
:10F4A000C9FA06460027049BEA1B6FF310330121BB
:10F4B00001A8049300F0F6FE08B10B30E3D14FF041
:10F4C0002003EFF3118883F31188206838B10368B3
:10F4D000626823F003039042236008BF6360012148
:10F4E000FFF778FF88F311880028C6D16B1CDAD0AB
:10F4F00000F0A0FA871BBD42D5DAC4E790E80C0003
:10F500001A600268536070470146006908B5431CE1
:10F510000ED0084B9B6999421FBF0A681369C01837
:10F5200010610846FFF7EAFF4FF0FF330B61002040
:10F5300008BD00BF102D00204FF02003EFF3118015
:10F5400083F31188704700000D4B194651F8242FA2
:10F550008A4200D002B9DA6870B9996861B1487A14
:10F56000C00609D1486A013006D148897F2803D9ED
:10F5700004480068814201D11A62704719627047DD
:10F58000102D0020B00A010090F90A0091F90A300C
:10F590009842ACBF002001207047000010B5014622
:10F5A000FFF7CAFF4B7A5A0604460DD50846FFF707
:10F5B000A5FF4B7A23F040034B72054B9868431A22
:10F5C00058425841FFF7C0FF84F3118810BD00BFB7
:10F5D000102D002008B50246FFF7AEFF13689A42CF
:10F5E00008BF002380F31188184608BD10B50146F6
:10F5F000FFF7A2FF04460846FFF780FF4B7A23F08F
:10F6000002034B7284F3118810BD10B50021FFF77F
:10F61000E1FF044628B1FFF7E9FF04F11400FFF70A
:10F6200073FF204610BD10B50446FFF7DFFF04F15D
:10F630001400BDE81040FFF767BF0000EFF305833B
:10F640000D2B09D81BB1084B5B681B0504D5074B74
:10F650009A681B6A9A4202D180F311887047044B62
:10F6600000221A60F1F7DEBE00ED00E0102D002050
:10F67000402D002010B5FFF75FFF0A4B9A68D37A40
:10F6800001330446D3720120FFF75EFF84F3118833
:10F690004FF02003EFF3118083F31188BDE8104091
:10F6A000FFF7CCBF102D002010B50368984208BFAB
:10F6B000002393B191F90A4093F90A20944206DAA3
:10F6C0005A684A600B605A681160596010BD426800
:10F6D000934202D01B68002BEBD1086043684B605B
:10F6E00043681960416010BD38B50446FFF724FF38
:10F6F000214605460648FFF7D7FF637A43F04003EB
:10F7000063720020FFF720FF85F3118838BD00BF2A
:10F71000342D0020427AD20604D1436A013301D14C
:10F72000FFF7E2BF7047000070B50B6104461D464D
:10F730008860CA6003BB4FF02003EFF3118683F3A8
:10F7400011884FF0FF330B6170B1CB6813B1FFF735
:10F750004DFF2562637A23F0040363722046FFF7AE
:10F76000D9FF86F3118870BD86F311884B692BB3DE
:10F770000846BDE870401847114A104650F8143F3B
:10F7800083420CD1086093694B6093691960916161
:10F7900070BD641B0C619469A342F3D01B68002BFD
:10F7A000F0D00C691D69AC42F3DC5A682C1B1C615B
:10F7B0004A600B605A681160596070BD70BD00BF2F
:10F7C000102D002038B50446FFF7B6FE054620464A
:10F7D000FFF794FE21460648FFF766FF637A43F081
:10F7E000400363720020FFF7AFFE85F3118838BD38
:10F7F000342D0020F8B5044616460D46FFF7CEFE20
:10F80000637A43F002036372731C19D04FF0200334
:10F81000EFF3118783F311880D484FF4004E002158
:10F82000CEFB06014FF4A0220023F0F729FD2A4663
:10F83000431C04F114012046FFF776FF87F311887B
:10F840002DB121462846BDE8F840FFF72DBFF8BD91
:10F85000FFFF040010B5064B04469868FFF7CAFF87
:10F86000044B00222046BDE810401A60F1F7DABDD3
:10F87000102D0020402D0020134B1B68002B10B5CD
:10F8800002461FDD43897F2B1CD8104B90F90A10CC
:10F890001B68994216DBFFF74FFE0D4951F8243FD4
:10F8A0008B4204460AD05BB192F90A0093F90A3000
:10F8B000C31A5842584184F3118810BD0020FAE75A
:10F8C0001846F8E7002010BD502D0020542D0020D0
:10F8D000102D0020014B00221A607047402D00209F
:10F8E00038B5054600202C68A54200D004B938BDC3
:10F8F0002046FFF798FE2046FFF70CFF0120F2E7B5
:10F90000064B03F124025A629A62054A00231360EF
:10F91000044A1360044A1360704700BF102D002092
:10F92000502D0020402D0020542D002038B5144CBF
:10F93000144BA2681B689A420FD0FFF7FDFD0546E5
:10F94000A068FFF7DBFDA16804F12400FFF7ACFE1F
:10F950000120FFF7F9FD85F31188226AA3689A4216
:10F960000CD04FF02003EFF3118083F31188064B86
:10F9700000221A60BDE83840F1F754BD38BD00BF21
:10F98000102D0020B00A0100402D0020014B986886
:10F99000704700BF102D002000F110038160C2608D
:10F9A0000060406003614361704770B504464FF0EA
:10F9B0002003EFF3118683F31188FFF726FE054637
:10F9C00060B1437ADB0602D1436A013312D00023CF
:10F9D000EB663046BDE87040FFF730BEA368E268D2
:10F9E0009A4218BF0133A360022104F1100000F015
:10F9F000DFFCEEE7FFF778FEE9E710B40A460446BD
:10FA00004FF02003EFF3118083F31188A36833B123
:10FA1000013BA36080F31188002010BC704721B91E
:10FA200080F311886FF00F00F7E7214610BCFFF755
:10FA300011BF0000074B10B5D3E900234FF47A74CF
:10FA4000A2FB0401002304FB031164220023F0F74E
:10FA500067FC10BD482D00204FF02002EFF311830A
:10FA600082F31188024AD2E9000183F311887047BA
:10FA7000482D002038B5FFF7EFFF4FF47A73A0FB55
:10FA8000034503FB01556422002320462946F0F775
:10FA900047FC38BD2DE9F34707464FF02003EFF34D
:10FAA000118083F311885949D1E90045E21945EBEA
:10FAB000E773C1E9002380F311886C46CDF800D0CC
:10FAC000CDF804D04FF02003EFF3118083F31188B9
:10FAD0004F4E3146024651F8143F8B4200D0EBB9ED
:10FAE00080F31188B068FFF7C7FEA0B1494A1368D8
:10FAF0001F44494B17601B689F420CDB00231360B7
:10FB00004FF02003EFF3118483F31188B068FFF7FF
:10FB100059FE84F3118802B0BDE8F08739464FF0F2
:10FB200000096FF0010E1D698D42AABFA5EB010C03
:10FB3000C3F81090C3F810C0491BB56918699D42FD
:10FB400014BF1D680025D0B993E80101C8F8000072
:10FB50001868C0F80480009883E8110000980093AA
:10FB60004360C3F810E082F311884FF02003EFF3F5
:10FB7000118283F311882B46002DD4D101E0002996
:10FB8000F1DC82F311880098A042ABD00028A9D004
:10FB9000019B984201D1002500E005684FF0FF3835
:10FBA0004FF0000984684FF02003EFF3118A83F3CC
:10FBB0001188C0F81080CCB1C36823B12046FFF78C
:10FBC00015FDC4F82090637A23F0040213F01B0F94
:10FBD000627202D1636A013313D08AF31188002D57
:10FBE00080D0019BAB4208D1002307E08AF3118843
:10FBF0004369002BF3D09847F1E72B6828461D4650
:10FC0000D0E72046FFF770FDE7E700BF482D002052
:10FC1000102D0020402D0020502D002008B54FF45D
:10FC200000724FF0FF330349034800F0A7F90020AA
:10FC300008BD00BFD0420020582D002003695A1C87
:10FC400011D00A4A926990421FBF01680A699B1845
:10FC50000B6190E80C001A60026853604FF0FF33AC
:10FC60000361002070471846704700BF102D002028
:10FC7000427AD20604D1436A013301D1FFF734BD81
:10FC800070470000F8B52E4E044600274FF40040A0
:10FC9000C0FB01674FF4A022002330463946F0F73D
:10FCA000EFFA461C4FF02003EFF3118583F3118820
:10FCB000002304F114076662E4612362D6B94FF0B1
:10FCC0002003EFF3118783F311884FF0FF33636252
:10FCD000236A1BB12046FFF789FC2662637A23F072
:10FCE000040363722046FFF7C3FF87F3118885F38F
:10FCF0001188F8BD134A114651F8143F8B4206D1C2
:10FD000061619369A36193691F609761EFE7002BBD
:10FD1000F6D0D2F818E0606A1E69B04208DC5A6872
:10FD2000301A1861A26163615A6817605F60DEE78C
:10FD3000801B73456062E3D01B68002BEBD1DFE7CB
:10FD4000FFFF0400102D0020EFF305800D2807D8D9
:10FD500038B1044B586880F40060C0F3C02070478D
:10FD60000120704700ED00E0024B9B68187A00F01C
:10FD700001007047102D002010B54FF02003EFF365
:10FD8000118483F31188437A590702D484F31188CC
:10FD900010BD23F004034372FFF76AFF2046BDE85D
:10FDA0001040FFF74BBC000030B587B004460E9DF5
:10FDB00004950D9D03950C9D02950B9D01950A9D43
:10FDC0000095F1F767FC044B9B6813B9636607B0B5
:10FDD00030BD5B6EFAE700BF102D002070B586B015
:10FDE00004460E9E04960D9E03960C9E02960B9E54
:10FDF0000F9D01960A9E0096FFF7D6FF6B1C03D05D
:10FE00002DB92046FFF7B8FF204606B070BD294641
:10FE10002046FFF737FFF7E7436D10B5044603B1FF
:10FE20009847637ADA0606D1626A013203D1204626
:10FE3000FFF7B4FB0BE09B0702D52046FFF7D6FB8C
:10FE4000636A013303D004F11400FFF7F7FE637A0D
:10FE500043F00803637210BDF0B5214F214D87B008
:10FE60003E46BD4205F12C0414D31F4B9A68D37A49
:10FE7000013BD3724FF02003EFF3118583F3118818
:10FE8000184CB4421FD385F3118807B0BDE8F04089
:10FE9000FFF7F0BB54F80C3C049354F8103C039368
:10FEA00054F8143C029354F8183C019354F81C3C49
:10FEB0000093A4F12C000FC8FFF776FF54F82C3CF8
:10FEC0001D652546CDE7616A4B1C03D0206819B932
:10FED000FFF752FF2C34D4E7FFF7D4FEFAE700BF58
:10FEE0005847002058470020102D0020037242720E
:10FEF00000234FF0FF328172C37242620362C3611A
:10FF00008362704700B501F10803BFF35B8F53E8CC
:10FF1000002F42F0010E43E800ECBCF1000FF6D1D7
:10FF2000BFF35B8FD30703D45DF804EBFFF766BA2A
:10FF30005DF804FBA0F10C018069FFF7E3BF10B589
:10FF400004464FF0FF312046FFF77CFA03460028B5
:10FF5000F7D008334268BFF35B8F53E8001F21F0EE
:10FF6000010E43E800ECBCF1000FF6D1BFF35B8F4C
:10FF7000CB0700D59047FFF7D9FCE2E7F0B587B093
:10FF800004461F460D461646FFF730FA002005903E
:10FF900004900290019003970094044B3246294646
:10FFA00004F11000FFF71AFF07B0F0BD3FFF00009B
:10FFB0004FF0FF320023C261044A03604160836056
:10FFC0008361436102624362704700BF35FF0000F6
:10FFD000F0B54FF02003EFF3118483F31188436AE7
:10FFE00023B984F311886FF01500F0BDBFF35B8F68
:10FFF0008368BFF35B8FDA0700F1080533D5426AE7
:020000021000EC
:1000000013680021002BECD0984227D10368576871
:1000100023F00303C9B9B842136000D153600368E9
:1000200003F00303036000234362BFF35B8F55E8D3
:10003000002F22F0010245E800210029F7D1BFF38B
:100040005B8F84F311881846F0BD0E6806F0030636
:100050003343B8420B6008BF5160E0E71E681946A1
:1000600026F00303CEE7C1694B1C00F10C02DAD085
:10007000084B9B699A421FBFC26813695B181361E2
:100080000369C2681A60C26853604FF0FF33C361EE
:10009000C9E700BF102D0020F8B506460C461746EC
:1000A0004FF02003EFF3118583F311884B6A23B1DE
:1000B00083420BD06FF02F000DE038B166626FB94C
:1000C00021463046FFF71EFF002004E02046FFF7E0
:1000D0007FFF0028F2DA85F31188F8BD25484FF438
:1000E000004E00210023CEFB07014FF4A022F0F7C1
:1000F000C7F80023471C04F10C06E7616361A361A4
:100100007FB94FF02002EFF3118382F311884FF093
:10011000FF32E26183F31188236A43B33046984784
:10012000D2E7154A114651F8143F8B4206D1E160DF
:100130009369236193691E609661C5E7002BF6D031
:10014000D2F818E0E0691F69B84208DC5A68381A2A
:1001500018612261E3605A6816605E60B4E7C01BF4
:100160007345E061E3D01B68002BEBD1DFE7184655
:10017000B1E700BFFFFF0400102D0020142330B5AD
:1001800003FB01000024002900DA30BD437B8460BA
:1001900003F00F03022B03D0042B01D0012B04D159
:1001A000436805681D6005686B6082F311884FF035
:1001B0002003EFF3118283F3118801391438E2E749
:1001C000836870B505460E46D3B100221C685A609C
:1001D000637A9A0714D5636A02331BD02046FFF76F
:1001E00022FA082E0CBF6FF003030023E366637A44
:1001F000DB0605D1636A013302D12046FFF774FAAA
:10020000EB68C3F30432164366F310330020EB604F
:10021000A86070BD6FF00A0070BDF8B50368984221
:1002200004460E46174606D13460636873606368FF
:100230001E606660F8BD4368002BF5D09B681168AE
:100240001868FFF7A1F90028EED12568AC42EBD081
:10025000002DE9D0AB6838681968FFF795F930B11F
:100260006B68736035606B681E606E60F8BD6368B4
:100270009D42D9D02D68EBE730B5457B036161F332
:1002800003054573C168002464F31031C160090C93
:1002900062F341018173C289846064F38F02C28179
:1002A00030BD00002DE9F04F404B85B09B680093B6
:1002B0000026012307468A469046019304464FF0E4
:1002C000FF35B146564510DB4FF02003EFF31186A2
:1002D00083F31188019C002C3FD1324629463846D1
:1002E000FFF74CFF86F3118840E04FF02003EFF357
:1002F000118B83F31188637B03F00F03022B03D070
:10030000042B04D0012B06D12269926801E02269F6
:100310001268002A3DD1B8F1000F14D0019A92B1B1
:10032000022B07D0042B13D0012B09D16A4621469A
:10033000206903E020696A4621461030FFF76DFF0F
:10034000C4F808D001358BF3118801361434B9E7AD
:1003500020696A4621460830F0E700230193B8F18E
:10036000000F07D186F311886FF00A04204605B00C
:10037000BDE8F08F02A94246304602910391FFF793
:1003800069FA04464FF02003EFF3118683F31188D6
:10039000A3E7E268C4F80890C2F304310B4363F3A7
:1003A0001032E260CDF80490CDE700BF102D0020A0
:1003B0000368984207D093E805001060186842600F
:1003C0001846FFF7FDBE704738B54FF02003EFF336
:1003D000118583F311880368C16098424FF00101D1
:1003E00081600DD093E805001060186842601846DF
:1003F000FFF7E6FE04462846FFF720F9204638BD01
:0A04000085F311880024F9E7704726
:02040A00FFFFF2
:08040C0044FFFE7F0100000027
:10041400F40401007506000000000000020701005A
:100424008D0D000000000000300501003D100000AB
:10043400000000003B0501003D100000000000002A
:100444004605010039130000000000000207010006
:10045400751800000000000002070100DDA3000081
:10046400000000003C0A0100A1E50000340A01007C
:10047400430A0100A1E500002C0A0100CA0401009E
:1004840029EC0000000000000C050100C1ED000093
:100494000000000002070100A5F1000000000000B8
:0C04A400020701001DFC00000000000029
:1004B0000C0802170D0101020909010106020918C1
:1004C00018030101090903030503554152545F3024
:1004D000000000001F000000C8310020040A0100D5
:1004E000D4040100040A0100EC0401004C000000E7
:1004F000883000206863695F7561727400464C4102
:1005000053485F30005352414D5F3000454E5452C6
:100510004F50595F3000000009110000000000003A
:100520000000000055100000DD0F0000000000007A
:10053000636C6B5F6B333273726300636C6B5F6D04
:100540003136737263007379735F636C6F636B0032
:10055000040A0100580501004C000000EC320020A4
:100560002F7573722F7372632F7A65706879722F8B
:100570007375627379732F626C7565746F6F7468CD
:100580002F636F6E74726F6C6C65722F7469636B1E
:1005900065722F7469636B65722E6300F401FA0053
:1005A000960064004B0032001E0014002F75737219
:1005B0002F7372632F7A65706879722F7375627307
:1005C00079732F626C7565746F6F74682F636F6ECB
:1005D00074726F6C6C65722F6C6C5F73772F6374C1
:1005E000726C2E63002F7573722F7372632F7A658E
:1005F000706879722F7375627379732F626C756589
:10060000746F6F74682F636F6E74726F6C6C657249
:100610002F6C6C5F73772F6C6C2E63006D0601007E
:10062000000000000000000031A50000EDA3000064
:100630002F7573722F7372632F7A65706879722FBA
:100640007375627379732F626C7565746F6F7468FC
:100650002F636F6E74726F6C6C65722F6863692F95
:100660006863695F6472697665722E6300436F6EBA
:1006700074726F6C6C65720001010101000202026C
:100680000202027075626C69630072616E646F6D64
:10069000007075626C69632069640072616E646FDA
:1006A0006D206964002F7573722F7372632F7A65E2
:1006B000706879722F7375627379732F626C7565C8
:1006C000746F6F74682F636F6E74726F6C6C657289
:1006D0002F6863692F6863692E63005A65706879B3
:1006E00072204F532076312E31332E3939204E6F00
:1006F0007620203120323031382032303A31373ACA
:100700003330000000000000000000000000000086
:1007100000000000000000000000000000000000D9
:1007200000000000000000000000000000000000C9
:1007300000000000000000000000000000000000B9
:1007400000000000000000000000000000000000A9
:100750000000000000000000000000000000000099
:100760000000000000000000000000000000000089
:100770000000000000000000000000000000000079
:100780000000000000000000000000000000000069
:100790000000000000000000000000000000000059
:1007A0000000000000000000000000000000000049
:1007B0000000000000000000000000000000000039
:1007C0000000000000000000000000000000000029
:1007D0000000000000000000000000000000000019
:1007E0000000000000000000000000000000000009
:1007F00000000000000000000000000000000000F9
:100800000000FFC1FBE84C90728BE7B3518963ABEA
:10081000232302841872AA612F3B51A8E53749FBB4
:10082000C9CA0C18532CFD45E39AE6F15DB0B61B1E
:10083000B4BE2A50EAE90E9C4B5E5724CCA1B759AE
:10084000B887FFE07D742648B9C5F3D9A8C4B1D5EF
:10085000911101420C39D5B0979D28D4F29BA4FD8B
:100860006465068C2996FEA2714DF3F82E58DB0DB7
:100870005A5F1528F57407CE25AF2B12E6D0DB2C76
:10088000DCC37FF03E3A13A4DCE2F96C54E2D8EA10
:10089000C8880021869C6AD8CB4E146AF94DD27E56
:1008A000B23203C6144B7FD1B8A6797C17ACED06E3
:1008B000ADAF0A947ABA03E792D7150973E86D16BB
:1008C000EEE13F781F9D09526EF17C362A716C75FE
:1008D00064448010434E35EC65270AB5FC26693F19
:1008E000599901638AA5BF685CD33CBE0BD6768359
:1008F000D657054A3DDD8173C9EB8A8439F4360B3E
:10090000F7000000294176712F7573722F7372639F
:100910002F7A65706879722F7375627379732F629D
:100920006C7565746F6F74682F636F6E74726F6C23
:100930006C65722F6C6C5F73772F6C6C5F66696C83
:100940007465722E63002F7573722F7372632F7A22
:1009500065706879722F7375627379732F626C7525
:1009600065746F6F74682F636F6E74726F6C6C65F3
:10097000722F68616C2F6E7266352F636E74722EE3
:1009800063002F7573722F7372632F7A65706879A5
:10099000722F7375627379732F626C7565746F6FE4
:1009A00074682F636F6E74726F6C6C65722F686100
:1009B0006C2F6E7266352F6D6179666C792E6300CF
:1009C000030400052F7573722F7372632F7A65709D
:1009D0006879722F7375627379732F626C756574A1
:1009E0006F6F74682F636F6E74726F6C6C65722FAB
:1009F00068616C2F6E7266352F7469636B65722E39
:100A000063000000ADE20000000000008DE2000085
:100A100051E70000CFE400000DE5000031E50000E3
:100A2000E3E80000A1E80000000000000000005022
:100A30000000000000030050010000004750494F33
:100A40005F31004750494F5F30000000B5EB0000B8
:100A500071EB000011EA0000E1EB00003DEB00004B
:100A6000C1EA0000ADEA000045EA000025EA000006
:100A700035EA000045EA00004DEA00005DEA0000AA
:100A80006DEA000001EB00007DEA000081EA000051
:100A900019EF000035EE0000BC4600201047002092
:100AA0001C4700204C47002058470020F5FFFFFF5F
:040AB000E02A002018
:100AB40002000000D844002000000000FD040100F2
:100AC40026000207000000200505010022000B118A
:100AD4000090D00300000000340400200000000057
:100AE400BD3C000000000000F403002001000000F1
:100AF4009140000000000000FC0300200000000002
:100B0400AD40000000000000C00300200000000011
:100B1400AD40000000000000C803002000000000F9
:100B2400AD4000000000000024040020000000008C
:100B34004532000000000000D00300200000000047
:100B44004532000000000000D8030020000000002F
:100B540045320000000000003C04002000000000BA
:100B6400ED3B0000000000004404002000000000F1
:100B740000000000000000004C0400200000000001
:100B8400B938000000000000040400200000000048
:100B9400C52B0000000000000C0400200000000031
:100BA400C52B000000000000140400200000000019
:100BB4000D460000000000001C040020000000009E
:100BC4000D46000000000000E003002000000000CB
:100BD4000D46000000000000E803002000000000B3
:100BE4000D460000000000002C040020000000005E
:100BF400C15F0000000000000000000000000000D1
:100C0400000100003C46002000000000000000003D
:100C14000000000000040000704700203C46002053
:100C24003C4600200000000000000000000000001E
:100C3400FFFFFFFFFF1F00001F0000000000000077
:100C440000000000182A002000000000471F0000D8
:100C540000000000202A002000000000F51F000012
:100C640000000000282A002000000000471F0000A8
:100C740000000000302A002000000000F51F0000E2
:100C840000000000382A002000000000F51F0000CA
:0C0C940003000000010000004701000008
:100CA0002004010000000000000000009804010082
:100CB00000000000000000005004010000000000DF
:100CC000000000002C0401001805010000000000D5
:100CD0003804010024050100000000008004010028
:100CE0004C0A0100000000008C040100900A010081
:100CF000902A0020440401000000000000000000D1
:100D000074040100100A0100442A00206804010054
:100D1000100A0100642A0020A40401000000000061
:100D2000000000005C040100000000000000000062
:0C0D30001404010000000000000000009E
:100D3C00584700205847002000000000FFFFFFFF2D
:080D4C00684700206847002001
:100D540000000000000000007847002078470020D1
:100D640000000000000000008847002088470020A1
:100D74000000000000000000984700209847002071
:100D84000000000000000000A8470020A847002041
:100D94000700070000000000DC04010020310020EF
:100DA4000000000000000000C8470020C8470020E1
:100DB4000200020000000000E4040100583000209A
:100DC4000000000000000000E8470020E847002081
:100DD400030003000000000050050100A4320020BD
:04000003000017FDE5
:00000001FF
